:100000000C94C22B0C94F32B0C94F32B0C94F32B29
:100010000C94F32B0C94F32B0C94F32B0C94F32BE8
:100020000C94F32B0C94F32B0C94F32B0C94F32BD8
:100030000C94F32B0C9433DB0C94F32B0C94F32BD8
:100040000C94F32B0C9464B90C94F32B0C94F32BB9
:100050000C94F32B0C94F32B0C94D6420C94F9D6FD
:100060000C94F32B0C9432B60C94F32B0C94F32BCE
:100070000C94F32B0C94F32B0C94F32B0C94F32B88
:100080000C94F32B0C94F32B0C94F32B0C94F32B78
:100090000C94F32B0C94F32B0C94F32B0C942BD487
:1000A0000C94F32B0C94F32B0C94F32B0C94F32B58
:1000B0000C94F32B0C94F32B0C94F32B0C94F32B48
:1000C0000C94F32B0C94F32B0C94F32B0C94F32B38
:1000D0000C94F32B0C94F32B0C94F32B0C94F32B28
:1000E0000C94F32B234331434D435B4375438343CC
:1000F0009D43A143A343A743AF437DD582D587D575
:1001000091D50AD69BD5A3D5ABD5B5D5BFD5C9D585
:10011000D8D5E2D50AD6ECD5F6D500D628D62BD63A
:100120001ED622D662D62FD633D639D63DD641D664
:1001300047D64BD64FD662D655D659D65DD6084A45
:10014000D73B3BCE016E84BCBFFDC12F3D6C7431EB
:100150009ABD56833DDA3D00C77F11BED9E4BB4C42
:100160003E916BAAAABE000000803F05A84CCDB20C
:10017000D44EB93836A9020C50B9918688083CA6ED
:10018000AAAA2ABE000000803F007C3C3E5E2B3DB8
:100190003F2F5B5D3B2C2A225C004572723A204D5A
:1001A000415854454D50204245440054656D70659A
:1001B000726174757265206865617465642062653A
:1001C00064207377697463686564206F66662E20A7
:1001D0004D415854454D502074726967676572658A
:1001E00064202121004572723A204D494E54454DFC
:1001F00050003A204578747275646572207377698F
:100200007463686564206F66662E204D494E5445C0
:100210004D502074726967676572656420210045DE
:1002200072723A204D415854454D50003A2045785D
:10023000747275646572207377697463686564208D
:100240006F66662E204D415854454D50207472699A
:10025000676765726564202100202D20496E7661F4
:100260006C6964206578747275646572206E756D52
:10027000626572202100504944204175746F747585
:100280006E652066696E69736865642120507574B7
:1002900020746865206C617374204B702C204B694E
:1002A00020616E64204B6420636F6E7374616E74A2
:1002B000732066726F6D2061626F766520696E745F
:1002C0006F20436F6E66696775726174696F6E2E19
:1002D0006800504944204175746F74756E652066DE
:1002E00061696C6564212074696D656F75740020A7
:1002F000403A006F6B20543A006F6B20423A005036
:100300004944204175746F74756E65206661696C2F
:100310006564212054656D70657261747572652025
:10032000746F6F206869676800204B643A20002072
:100330004B693A2000204B703A200020436C6173D7
:100340007369632050494420002054753A200020EE
:100350004B753A2000206D61783A2000206D696E5F
:100360003A200020643A200020626961733A20003C
:100370001000C90210012C01400122017001180176
:10038000B0010E01F00104015002FA00B002F000C9
:100390003003E600D003DC009004D2007005C800F2
:1003A000A006BE000008B400B009AA00D00BA0004F
:1003B000600E960060118C000015820020197800F4
:1003C000C01D6E00A0226400B0275A00902C50007F
:1003D00000314600E0343C0010383200903A2800EA
:1003E000603C1E00A03D1400803E0A00203F00003B
:1003F00070012C0190012701B0012201C0011D01F3
:10040000F00118011002130130020E01600209010F
:1004100090020401C002FF000003FA004003F5004F
:100420008003F000D003EB002004E6007004E1003C
:10043000E004DC004005D700C005D2004006CD0036
:10044000D006C8008007C3003008BE00F008B9001D
:10045000C009B400B00AAF00B00BAA00D00CA500D0
:10046000000EA000500F9B00C0109600501291008B
:1004700000148C00C0158700B0178200B0197D00F1
:10048000D01B7800001E730040206E00902269008F
:10049000F024640040275F0090295A00E02B5500AB
:1004A000102E500020304B0010324600E033410047
:1004B00090353C001037370070383200A0392D00DD
:1004C000B03A2800A03B2300603C1E00103D1900FC
:1004D000903D1400103E0F00703E0A00C03E050023
:1004E000003F0000686F77746F2E70727573613310
:1004F000642E637A00686F77746F2E707275736103
:1005000033642E636F6D00686F77746F2E70727531
:10051000736133642E636F6D00686F77746F2E7034
:100520007275736133642E637A00686F77746F2E0F
:10053000707275736133642E636F6D00666F7275D0
:100540006D2E707275736133642E637A00666F72FC
:10055000756D2E707275736133642E636F6D0066F6
:100560006F72756D2E707275736133642E636F6D6B
:1005700000666F72756D2E707275736133642E63D1
:100580007A00666F72756D2E707275736133642EAA
:10059000636F6D00707275736133642E637A0070DF
:1005A0007275736133642E636F6D00707275736161
:1005B00033642E636F6D00707275736133642E63E4
:1005C0007A00707275736133642E636F6D005779B2
:1005D000626F72206A657A796B612020202020206A
:1005E00020200043616D626961206C61206C656E42
:1005F000677561200053656C657A2E206C61206CF4
:10060000696E677561005679626572206A617A79F0
:100610006B6120202020202020200053656C656322
:1006200074206C616E677561676520202020200052
:10063000506F6C736B6900457370616E6F6C00492D
:1006400074616C69616E6F0043657374696E6100FB
:10065000456E676C697368004572726F7220696ECF
:10066000206D656E752073747275637475726500A4
:100670004572726F7220696E206D656E752073749D
:1006800072756374757265004572726F7220696E5F
:10069000206D656E75207374727563747572650074
:1006A0004572726F7220696E206D656E752073746D
:1006B00072756374757265004572726F7220696E2F
:1006C000206D656E75207374727563747572650044
:1006D000446F737461766F76616E69205A0041646D
:1006E0006A757374696E67205A0041646A75737421
:1006F000696E67205A00446F737461766F76616E1D
:1007000069205A0041646A757374696E67205A00E3
:10071000426162797374657070696E672059004236
:100720006162797374657070696E67205900426107
:1007300062797374657070696E67205900426162F6
:10074000797374657070696E6720590042616279CF
:100750007374657070696E672059004261627973C5
:1007600074657070696E67205800426162797374B5
:10077000657070696E6720580042616279737465B4
:100780007070696E67205800426162797374657099
:1007900070696E6720580042616279737465707089
:1007A000696E6720580020746F6F206C6F6E672031
:1007B000657874727573696F6E2070726576656E98
:1007C0007465640020746F6F206C6F6E67206578AD
:1007D00074727573696F6E2070726576656E74657C
:1007E000640020746F6F206C6F6E67206578747280
:1007F0007573696F6E2070726576656E74656400DE
:1008000020746F6F206C6F6E6720657874727573DB
:10081000696F6E2070726576656E74656400207411
:100820006F6F206C6F6E6720657874727573696F77
:100830006E2070726576656E7465640020636F6CFF
:100840006420657874727573696F6E207072657656
:10085000656E7465640020636F6C642065787472E3
:100860007573696F6E2070726576656E746564006D
:1008700020636F6C6420657874727573696F6E2085
:1008800070726576656E7465640020636F6C6420B9
:10089000657874727573696F6E2070726576656EB7
:1008A0007465640020636F6C64206578747275737E
:1008B000696F6E2070726576656E74656400656E32
:1008C0006473746F7073206869743A2000656E6495
:1008D00073746F7073206869743A2000656E647376
:1008E000746F7073206869743A2000656E64737465
:1008F0006F7073206869743A2000656E6473746F5A
:100900007073206869743A20005374657072617462
:100910006520746F6F20686967683A2000537465BA
:10092000707261746520746F6F20686967683A201F
:1009300000537465707261746520746F6F2068690C
:1009400067683A2000537465707261746520746F33
:100950006F20686967683A2000537465707261742B
:100960006520746F6F20686967683A200043616E84
:100970006E6F7420656E746572207375626469723F
:100980003A200043616E6E6F7420656E746572204C
:100990007375626469723A200043616E6E6F7420F1
:1009A000656E746572207375626469723A200043E3
:1009B000616E6E6F7420656E74657220737562640B
:1009C00069723A200043616E6E6F7420656E7465C3
:1009D00072207375626469723A20006572726F7278
:1009E0002077726974696E6720746F2066696C6520
:1009F000006572726F722077726974696E67207415
:100A00006F2066696C65006572726F72207772691B
:100A100074696E6720746F2066696C650065727218
:100A20006F722077726974696E6720746F206669CF
:100A30006C65006572726F722077726974696E6797
:100A400020746F2066696C65004E6F7420534420DB
:100A50007072696E74696E67004E6F742053442023
:100A60007072696E74696E67004E6F742053442013
:100A70007072696E74696E67004E6F742053442003
:100A80007072696E74696E67004E6F7420534420F3
:100A90007072696E74696E67005344207072696E7B
:100AA00074696E6720627974652000534420707207
:100AB000696E74696E672062797465200053442002
:100AC0007072696E74696E67206279746520005374
:100AD00044207072696E74696E6720627974652053
:100AE000005344207072696E74696E672062797475
:100AF00065200057726974696E6720746F2066699B
:100B00006C653A200057726974696E6720746F20B3
:100B100066696C653A200057726974696E67207463
:100B20006F2066696C653A200057726974696E6758
:100B300020746F2066696C653A2000577269746989
:100B40006E6720746F2066696C653A200046696C98
:100B5000652073656C65637465640046696C652027
:100B600073656C65637465640046696C65207365C4
:100B70006C65637465640046696C652073656C65BB
:100B8000637465640046696C652073656C656374A5
:100B90006564002053697A653A20002053697A65BC
:100BA0003A20002053697A653A20002053697A651B
:100BB0003A20002053697A653A200046696C652026
:100BC0006F70656E65643A200046696C65206F70D1
:100BD000656E65643A200046696C65206F70656ECD
:100BE00065643A200046696C65206F70656E6564C7
:100BF0003A200046696C65206F70656E65643A2026
:100C0000006F70656E206661696C65642C204669B2
:100C10006C653A20006F70656E206661696C656472
:100C20002C2046696C653A20006F70656E20666105
:100C3000696C65642C2046696C653A20006F7065AC
:100C40006E206661696C65642C2046696C653A208B
:100C5000006F70656E206661696C65642C20466962
:100C60006C653A2000776F726B446972206F706513
:100C70006E206661696C656400776F726B4469729F
:100C8000206F70656E206661696C656400776F72B5
:100C90006B446972206F70656E206661696C656473
:100CA00000776F726B446972206F70656E206661A9
:100CB000696C656400776F726B446972206F706550
:100CC0006E206661696C65640053442063617264E0
:100CD000206F6B0053442063617264206F6B00537C
:100CE000442063617264206F6B005344206361721F
:100CF00064206F6B0053442063617264206F6B004B
:100D00006F70656E526F6F74206661696C65640008
:100D10006F70656E526F6F74206661696C656400F8
:100D20006F70656E526F6F74206661696C656400E8
:100D30006F70656E526F6F74206661696C656400D8
:100D40006F70656E526F6F74206661696C656400C8
:100D5000766F6C756D652E696E6974206661696C5D
:100D6000656400766F6C756D652E696E69742066BA
:100D700061696C656400766F6C756D652E696E696E
:100D800074206661696C656400766F6C756D652EA4
:100D9000696E6974206661696C656400766F6C7554
:100DA0006D652E696E6974206661696C65640053B7
:100DB0004420696E6974206661696C00534420693F
:100DC0006E6974206661696C00534420696E6974B1
:100DD000206661696C00534420696E697420666105
:100DE000696C00534420696E6974206661696C0007
:100DF00043616E6E6F74206F70656E2073756264F0
:100E000069720043616E6E6F74206F70656E20733F
:100E100075626469720043616E6E6F74206F7065F5
:100E20006E207375626469720043616E6E6F742028
:100E30006F70656E207375626469720043616E6ED7
:100E40006F74206F70656E207375626469720048FC
:100E50006F74656E64206F6666736574733A0048DC
:100E60006F74656E64206F6666736574733A0048CC
:100E70006F74656E64206F6666736574733A0048BC
:100E80006F74656E64206F6666736574733A0048AC
:100E90006F74656E64206F6666736574733A006F75
:100EA00070656E006F70656E006F70656E006F70BC
:100EB000656E006F70656E00545249474745524554
:100EC000440054524947474552454400545249470B
:100ED000474552454400545249474745524544000E
:100EE000545249474745524544005265706F7274E9
:100EF000696E6720656E6473746F702073746174BB
:100F00007573005265706F7274696E6720656E64E8
:100F100073746F7020737461747573005265706FB1
:100F20007274696E6720656E6473746F7020737479
:100F300061747573005265706F7274696E672065B5
:100F40006E6473746F70207374617475730052658E
:100F5000706F7274696E6720656E6473746F702051
:100F6000737461747573007A5F6D61783A20007AEA
:100F70005F6D61783A20007A5F6D61783A20007A7F
:100F80005F6D61783A20007A5F6D61783A20007A6F
:100F90005F6D696E3A20007A5F6D696E3A20007A63
:100FA0005F6D696E3A20007A5F6D696E3A20007A53
:100FB0005F6D696E3A2000795F6D61783A20007943
:100FC0005F6D61783A2000795F6D61783A20007931
:100FD0005F6D61783A2000795F6D61783A20007921
:100FE0005F6D696E3A2000795F6D696E3A20007915
:100FF0005F6D696E3A2000795F6D696E3A20007905
:101000005F6D696E3A2000785F6D61783A200078F4
:101010005F6D61783A2000785F6D61783A200078E2
:101020005F6D61783A2000785F6D61783A200078D2
:101030005F6D696E3A2000785F6D696E3A200078C6
:101040005F6D696E3A2000785F6D696E3A200078B6
:101050005F6D696E3A2000496E76616C6964206547
:101060007874727564657200496E76616C6964208B
:10107000657874727564657200496E76616C696436
:1010800020657874727564657200496E76616C696A
:101090006420657874727564657200496E76616C5F
:1010A000696420657874727564657200416374695F
:1010B00076652045787472756465723A20004163E4
:1010C000746976652045787472756465723A20009B
:1010D0004163746976652045787472756465723A07
:1010E0002000416374697665204578747275646583
:1010F000723A200041637469766520457874727590
:101100006465723A2000556E6B6E6F776E20636F68
:101110006D6D616E643A202200556E6B6E6F776E56
:1011200020636F6D6D616E643A202200556E6B6EA8
:101130006F776E20636F6D6D616E643A202200558B
:101140006E6B6E6F776E20636F6D6D616E643A20AB
:101150002200556E6B6E6F776E20636F6D6D616EE2
:10116000643A202200526573656E643A200052652D
:1011700073656E643A2000526573656E643A2000B0
:10118000526573656E643A2000526573656E643A09
:1011900020005072696E7465722073746F70706590
:1011A000642064756520746F206572726F72732E8F
:1011B0002046697820746865206572726F722061BC
:1011C0006E6420757365204D39393920746F207233
:1011D0006573746172742E202854656D7065726138
:1011E000747572652069732072657365742E20535F
:1011F0006574206974206166746572207265737409
:10120000617274696E6729005072696E746572202C
:1012100073746F707065642064756520746F2065E9
:1012200072726F72732E204669782074686520652B
:1012300072726F7220616E6420757365204D39394A
:101240003920746F20726573746172742E20285473
:10125000656D706572617475726520697320726561
:101260007365742E205365742069742061667465FB
:10127000722072657374617274696E6729005072AE
:10128000696E7465722073746F7070656420647524
:101290006520746F206572726F72732E20466978B4
:1012A00020746865206572726F7220616E642075AB
:1012B0007365204D39393920746F207265737461FC
:1012C00072742E202854656D706572617475726534
:1012D0002069732072657365742E205365742069CC
:1012E00074206166746572207265737461727469CA
:1012F0006E6729005072696E7465722073746F7026
:101300007065642064756520746F206572726F72F9
:10131000732E2046697820746865206572726F723A
:1013200020616E6420757365204D39393920746FE2
:1013300020726573746172742E202854656D706517
:101340007261747572652069732072657365742E9D
:10135000205365742069742061667465722072651B
:101360007374617274696E6729005072696E746576
:10137000722073746F707065642064756520746F7B
:10138000206572726F72732E2046697820746865CA
:10139000206572726F7220616E6420757365204DD6
:1013A00039393920746F20726573746172742E201C
:1013B0002854656D7065726174757265206973205B
:1013C00072657365742E205365742069742061669C
:1013D0007465722072657374617274696E67290036
:1013E0005072696E7465722068616C7465642E2039
:1013F0006B696C6C28292063616C6C6564210050FA
:1014000072696E7465722068616C7465642E206BFD
:10141000696C6C28292063616C6C656421005072D2
:10142000696E7465722068616C7465642E206B69E6
:101430006C6C28292063616C6C65642100507269B2
:101440006E7465722068616C7465642E206B696CC3
:101450006C28292063616C6C656421005072696E90
:101460007465722068616C7465642E206B696C6CA5
:1014700028292063616C6C6564210020436F756EC0
:101480007420583A200020436F756E7420583A201B
:101490000020436F756E7420583A200020436F750A
:1014A0006E7420583A200020436F756E7420583AAD
:1014B00020004649524D574152455F4E414D453AF5
:1014C0004D61726C696E2056312E302E323B2053A6
:1014D0007072696E7465722F6772626C206D6173D1
:1014E00068757020666F722067656E3620464952B7
:1014F0004D574152455F55524C3A68747470733A77
:101500002F2F6769746875622E636F6D2F70727507
:10151000736133642F50727573612D69332D506C74
:1015200075732F2050524F544F434F4C5F564552C6
:1015300053494F4E3A312E30204D414348494E4594
:101540005F545950453A5072757361206933204594
:10155000585452554445525F434F554E543A3120EA
:10156000555549443A30303030303030302D3030FD
:1015700030302D303030302D303030302D30303074
:101580003030303030303030300A004649524D571C
:101590004152455F4E414D453A4D61726C696E2036
:1015A00056312E302E323B20537072696E74657244
:1015B0002F6772626C206D617368757020666F7240
:1015C0002067656E36204649524D574152455F555A
:1015D000524C3A68747470733A2F2F676974687547
:1015E000622E636F6D2F707275736133642F50724A
:1015F0007573612D69332D506C75732F2050524FC8
:10160000544F434F4C5F56455253494F4E3A312E3B
:1016100030204D414348494E455F545950453A505A
:1016200072757361206933204558545255444552B0
:101630005F434F554E543A3120555549443A303066
:101640003030303030302D303030302D30303030A0
:101650002D303030302D3030303030303030303090
:1016600030300A004649524D574152455F4E414D78
:10167000453A4D61726C696E2056312E302E323BE8
:1016800020537072696E7465722F6772626C206D80
:10169000617368757020666F722067656E362046CC
:1016A00049524D574152455F55524C3A68747470D7
:1016B000733A2F2F6769746875622E636F6D2F7090
:1016C0007275736133642F50727573612D69332D98
:1016D000506C75732F2050524F544F434F4C5F56F0
:1016E000455253494F4E3A312E30204D41434849DF
:1016F0004E455F545950453A5072757361206933B5
:101700002045585452554445525F434F554E543A24
:101710003120555549443A30303030303030302D5A
:10172000303030302D303030302D303030302D30C2
:1017300030303030303030303030300A00464952AE
:101740004D574152455F4E414D453A4D61726C696E
:101750006E2056312E302E323B20537072696E74DB
:1017600065722F6772626C206D6173687570206698
:101770006F722067656E36204649524D574152457B
:101780005F55524C3A68747470733A2F2F676974BE
:101790006875622E636F6D2F707275736133642F7D
:1017A00050727573612D69332D506C75732F2050F5
:1017B000524F544F434F4C5F56455253494F4E3A48
:1017C000312E30204D414348494E455F54595045D4
:1017D0003A5072757361206933204558545255440C
:1017E00045525F434F554E543A3120555549443A7E
:1017F00030303030303030302D303030302D3030EF
:1018000030302D303030302D3030303030303030DE
:10181000303030300A004649524D574152455F4EF4
:10182000414D453A4D61726C696E2056312E302E15
:10183000323B20537072696E7465722F6772626CEE
:10184000206D617368757020666F722067656E36F3
:10185000204649524D574152455F55524C3A6874A3
:101860007470733A2F2F6769746875622E636F6D99
:101870002F707275736133642F50727573612D69A7
:10188000332D506C75732F2050524F544F434F4C93
:101890005F56455253494F4E3A312E30204D414309
:1018A00048494E455F545950453A5072757361200E
:1018B00069332045585452554445525F434F554E65
:1018C000543A3120555549443A3030303030303078
:1018D000302D303030302D303030302D3030303011
:1018E0002D3030303030303030303030300A00532E
:1018F000746F6C696B204F4B2E0042617365206CD6
:101900006973746F2E0050696174746F206661741E
:10191000746F2E00426564204F4B2E004265642098
:10192000646F6E652E0047727A616E69652073740C
:101930006F6C696B612E2E00426173652043616C90
:10194000656E74616E646F0050696174746F2072AB
:10195000697363616C64616D2E005A6168726976A7
:10196000616E69206265642E2E2E004265642048F7
:10197000656174696E672E0047727A616E696520D1
:101980004F4B2E0043616C656E74616E646F206C0A
:101990006973746F2E0052697363616C64616D6565
:1019A0006E746F20666174746F2E005A616872697C
:1019B00076616E69204F4B2E0048656174696E67D1
:1019C00020646F6E652E0047727A616E69652E2EF7
:1019D0002E0043616C656E74616E646F2E2E2E0056
:1019E00052697363616C64616D656E746F2E2E2E27
:1019F000005A6168726976616E692E2E2E00486504
:101A00006174696E672E2E2E004D31303920496E7B
:101A100076616C6964206578747275646572200003
:101A20004D31303920496E76616C69642065787477
:101A3000727564657220004D31303920496E7661CF
:101A40006C696420657874727564657220004D312C
:101A5000303920496E76616C6964206578747275DE
:101A600064657220004D31303920496E76616C69B1
:101A70006420657874727564657220004E6F2074FE
:101A80006865726D6973746F7273202D206E6F209C
:101A900074656D7065726174757265004E6F207447
:101AA0006865726D6973746F7273202D206E6F207C
:101AB00074656D7065726174757265004E6F207427
:101AC0006865726D6973746F7273202D206E6F205C
:101AD00074656D7065726174757265004E6F207407
:101AE0006865726D6973746F7273202D206E6F203C
:101AF00074656D7065726174757265004E6F2074E7
:101B00006865726D6973746F7273202D206E6F201B
:101B100074656D7065726174757265004D32323135
:101B200020496E76616C69642065787472756465AD
:101B30007220004D32323120496E76616C6964202A
:101B4000657874727564657220004D3232312049B7
:101B50006E76616C69642065787472756465722054
:101B6000004D32323120496E76616C6964206578AF
:101B700074727564657220004D32323120496E7680
:101B8000616C696420657874727564657220004DBB
:101B900032313820496E76616C69642065787472E0
:101BA0007564657220004D32313820496E76616C63
:101BB000696420657874727564657220004D3231F5
:101BC0003820496E76616C6964206578747275643A
:101BD000657220004D32313820496E76616C69643F
:101BE00020657874727564657220004D323138203A
:101BF000496E76616C69642065787472756465728B
:101C000020004D32303020496E76616C6964206569
:101C10007874727564657220004D32303020496EE0
:101C200076616C69642065787472756465722000F1
:101C30004D32303020496E76616C6964206578746D
:101C4000727564657220004D32303020496E7661C5
:101C50006C696420657874727564657220004D3219
:101C6000303020496E76616C6964206578747275D5
:101C700064657220004D31303520496E76616C69A3
:101C80006420657874727564657220004D3130355A
:101C900020496E76616C696420657874727564653C
:101CA0007220004D31303520496E76616C696420B8
:101CB000657874727564657220004D313035204945
:101CC0006E76616C696420657874727564657220E3
:101CD000004D31303520496E76616C69642065783D
:101CE00074727564657220004D31303420496E760F
:101CF000616C696420657874727564657220004D4A
:101D000031303420496E76616C6964206578747274
:101D10007564657220004D31303420496E76616CF7
:101D2000696420657874727564657220004D313085
:101D30003420496E76616C696420657874727564CC
:101D4000657220004D31303420496E76616C6964D3
:101D50002065787472756465722000456E64206633
:101D6000696C65206C69737400456E642066696CEB
:101D700065206C69737400456E642066696C65202B
:101D80006C69737400456E642066696C65206C69CB
:101D9000737400456E642066696C65206C697374A9
:101DA00000426567696E2066696C65206C697374B2
:101DB00000426567696E2066696C65206C697374A2
:101DC00000426567696E2066696C65206C69737492
:101DD00000426567696E2066696C65206C69737482
:101DE00000426567696E2066696C65206C69737472
:101DF00000446F6E65207072696E74696E6720664C
:101E0000696C6500446F6E65207072696E74696EEE
:101E1000672066696C6500446F6E65207072696E3C
:101E200074696E672066696C6500446F6E6520702A
:101E300072696E74696E672066696C6500446F6EC6
:101E400065207072696E74696E672066696C6500E2
:101E50004E6F204C696E65204E756D6265722077FD
:101E600069746820636865636B73756D2C204C61C1
:101E70007374204C696E653A20004E6F204C696E79
:101E800065204E756D62657220776974682063689D
:101E900065636B73756D2C204C617374204C696E97
:101EA000653A20004E6F204C696E65204E756D625C
:101EB0006572207769746820636865636B73756DFC
:101EC0002C204C617374204C696E653A20004E6F73
:101ED000204C696E65204E756D626572207769745D
:101EE0006820636865636B73756D2C204C61737437
:101EF000204C696E653A20004E6F204C696E65205B
:101F00004E756D62657220776974682063686563D9
:101F10006B73756D2C204C617374204C696E653A3F
:101F200020004E6F20436865636B73756D20776981
:101F30007468206C696E65206E756D6265722C2008
:101F40004C617374204C696E653A20004E6F2043DB
:101F50006865636B73756D2077697468206C696E52
:101F600065206E756D6265722C204C617374204C17
:101F7000696E653A20004E6F20436865636B737528
:101F80006D2077697468206C696E65206E756D626E
:101F900065722C204C617374204C696E653A200088
:101FA0004E6F20436865636B73756D207769746845
:101FB000206C696E65206E756D6265722C204C61B7
:101FC0007374204C696E653A20004E6F204368653B
:101FD000636B73756D2077697468206C696E65201A
:101FE0006E756D6265722C204C617374204C696E45
:101FF000653A2000636865636B73756D206D697366
:102000006D617463682C204C617374204C696E653B
:102010003A2000636865636B73756D206D69736D3D
:10202000617463682C204C617374204C696E653A4E
:102030002000636865636B73756D206D69736D61F6
:102040007463682C204C617374204C696E653A206F
:1020500000636865636B73756D206D69736D617482
:1020600063682C204C617374204C696E653A2000C3
:10207000636865636B73756D206D69736D617463FF
:10208000682C204C617374204C696E653A20004CBA
:10209000696E65204E756D626572206973206E6F82
:1020A00074204C617374204C696E65204E756D62AE
:1020B00065722B312C204C617374204C696E653A2B
:1020C00020004C696E65204E756D626572206973E3
:1020D000206E6F74204C617374204C696E65204EC5
:1020E000756D6265722B312C204C617374204C69C4
:1020F0006E653A20004C696E65204E756D626572A2
:10210000206973206E6F74204C617374204C696E6B
:1021100065204E756D6265722B312C204C61737495
:10212000204C696E653A20004C696E65204E756DD5
:10213000626572206973206E6F74204C6173742025
:102140004C696E65204E756D6265722B312C204C8A
:10215000617374204C696E653A20004C696E65208D
:102160004E756D626572206973206E6F74204C61CC
:102170007374204C696E65204E756D6265722B31EB
:102180002C204C617374204C696E653A2000446FBA
:102190006E6520736176696E672066696C652E00D6
:1021A000446F6E6520736176696E672066696C6541
:1021B0002E00446F6E6520736176696E67206669D4
:1021C0006C652E00446F6E6520736176696E6720C2
:1021D00066696C652E00446F6E6520736176696E6A
:1021E000672066696C652E006F6B006F6B006F6B0C
:1021F000006F6B006F6B002020506C616E6E65721B
:1022000042756666657242797465733A20002020D3
:10221000506C616E6E657242756666657242797465
:1022200065733A20002020506C616E6E65724275B5
:102230006666657242797465733A20002020506C9E
:10224000616E6E6572427566666572427974657319
:102250003A20002020506C616E6E65724275666691
:10226000657242797465733A200020467265652074
:102270004D656D6F72793A20002046726565204D7C
:10228000656D6F72793A20002046726565204D6554
:102290006D6F72793A20002046726565204D656D3C
:1022A0006F72793A20002046726565204D656D6F2A
:1022B00072793A2000204C61737420557064617407
:1022C00065643A2000204C61737420557064617419
:1022D00065643A2000204C61737420557064617409
:1022E00065643A2000204C617374205570646174F9
:1022F00065643A2000204C617374205570646174E9
:1023000065643A2000207C20417574686F723A2021
:1023100000207C20417574686F723A2000207C2078
:10232000417574686F723A2000207C204175746892
:102330006F723A2000207C20417574686F723A20D9
:102340000020536F667477617265205265736574FF
:102350000020536F667477617265205265736574EF
:102360000020536F667477617265205265736574DF
:102370000020536F667477617265205265736574CF
:102380000020536F667477617265205265736574BF
:1023900000205761746368646F67205265736574C9
:1023A00000205761746368646F67205265736574B9
:1023B00000205761746368646F67205265736574A9
:1023C00000205761746368646F6720526573657499
:1023D00000205761746368646F6720526573657489
:1023E000002042726F776E206F757420526573659E
:1023F00074002042726F776E206F7574205265737F
:102400006574002042726F776E206F75742052657C
:10241000736574002042726F776E206F757420525E
:1024200065736574002042726F776E206F7574203B
:102430005265736574002045787465726E616C2016
:102440005265736574002045787465726E616C2006
:102450005265736574002045787465726E616C20F6
:102460005265736574002045787465726E616C20E6
:102470005265736574002045787465726E616C20D6
:10248000526573657400506F776572557000506FB8
:10249000776572557000506F776572557000506F98
:1024A000776572557000506F776572557000656E74
:1024B000717565696E67202200656E717565696E5C
:1024C00067202200656E717565696E672022006560
:1024D0006E717565696E67202200656E717565693C
:1024E0006E672022007770726F772E207A6D696197
:1024F0006E007061726120746F6D61722065666537
:1025000063746F0020706572206D6F7374726172F6
:102510006520692063616D622E002070726F2070EB
:10252000726F6A6576656E69207A6D656E002066E9
:102530006F722074616B6520656666656374005216
:10254000657374617274206472756B61726B69007B
:102550005265696E6963696172206C6120696D7092
:102560002E005269617676696F206C612073746108
:102570006D702E0052657374617274756A74652093
:102580007469736B61726E75005265626F6F74204F
:10259000746865207072696E746572004D6F642096
:1025A0005B7720777964616A6E6F73635D004D6F4E
:1025B000646F205B6D617320667565727A615D0082
:1025C0004D6F646F205B70697520666F727A615D14
:1025D000004D6F6420205B7679732E2076796B6FC7
:1025E0006E5D004D6F6465205B6869676820706F81
:1025F0007765725D004D6F64202020202020205BD5
:1026000063696368795D004D6F646F20202020202E
:102610005B73696C656E63696F5D004D6F646F20FD
:10262000202020205B73696C656E7A696F736F5D23
:10263000004D6F64202020202020205B7469636897
:10264000795D004D6F646520202020205B73696CEC
:10265000656E745D0057796D69616E612066696CA5
:10266000616D656E74750043616D6269616E646F62
:102670002066696C2E21004D757465766F6C65203F
:1026800066696C2E210056796D656E612066696CF5
:10269000616D656E747521004368616E67696E6770
:1026A0002066696C616D656E7421005770726F777A
:1026B00061647A2066696C616D656E7400496E7341
:1026C000657274612066696C616D656E746F004936
:1026D0006E7365726972652066696C616D656E7492
:1026E0006F00566C6F7A74652066696C616D656EFB
:1026F0007400496E736572742066696C616D656EF5
:1027000074004E616369736E696A2070727A7963CE
:1027100069736B00592070756C736520656C206D52
:10272000616E646F00592070756C736520656C2054
:102730006D616E646F004120737469736B6E6574B4
:102740006520746C616369746B6F00416E64207006
:102750007265737320746865206B6E6F62005779C1
:102760006D69616E61206F6B210043616D6269610B
:1027700072206269656E210043616D6269612E207D
:10278000726975736369746F21005A6D656E61209B
:1027900075737065736E6121004368616E676520B3
:1027A000737563636573732100437A79737A637A0F
:1027B0002E206B6F6C6F72750043617267616E647F
:1027C0006F20636F6C6F720043617267616E646F3C
:1027D00020636F6C6F720043697374656E69206269
:1027E00061727679004C6F6164696E6720636F6C0B
:1027F0006F720050726F737A6520637A656B6163E4
:102800000045737065726100417370657474610096
:1028100050726F73696D2063656B656A74650050F3
:102820006C656173652077616974005770726F77AA
:102830002E2066696C616D656E7475004361726708
:10284000616E646F2066696C2E0043617267616E11
:10285000646F2066696C2E005A61766164656E69EA
:102860002066696C616D656E7475004C6F6164699A
:102870006E672066696C616D656E74004B6F6C6F7E
:1028800072207A616E6965637A79737A2E00436F7C
:102890006C6F72206E6F20636C61726F00436F6C9F
:1028A0006F72206E6F20636C61726F00426172768E
:1028B00061206E656E6920636973746100436F6C9B
:1028C0006F72206E6F7420636C656172004272617A
:1028D0006B2066696C616D656E74750046696C2E5F
:1028E000206E6F206361726761646F0046696C2EB1
:1028F000206E6F206361726761646F0046696C616E
:102900006D656E74206E657A61766564656E0046ED
:10291000696C616D656E74206E6F74206C6F61649C
:102920006564004E6965004E6F004E6F004E650095
:102930004E6F0054616B00536900536900416E6F24
:10294000005965730057796D69616E61206F6B3F47
:102950000043616D626961646F20636F72726563C9
:102960002E3F0043616D626961746F20636F727204
:102970002E3F0056796D656E61206F6B3F00436896
:10298000616E67656420636F72726563746C793F12
:1029900000506F6D6F6300537570706F72740053E9
:1029A0007570706F727400506F64706F7261005355
:1029B0007570706F7274004E6167727A656A206418
:1029C00079737A65210050726563616C2E20657899
:1029D000747275736F7221005072657269732E2064
:1029E0007567656C6C6F210050726564656872650F
:1029F0006A746520747279736B7521005072656812
:102A000065617420746865206E6F7A7A6C65210048
:102A1000424C41443A004552524F523A00455252BC
:102A20004F523A0043485942413A004552524F52A0
:102A30003A00526563747261637400526563747224
:102A400061637400526563747261637400526563FC
:102A500074726163740052656374726163740057C9
:102A600070726F7761647A2066696C616D656E74EF
:102A700000496E74726F64756369722066696C6177
:102A80006D656E746F004361726963617265206683
:102A9000696C616D656E746F005A61766573742040
:102AA00066696C616D656E74004C6F616420666967
:102AB0006C616D656E740057796A61632066696C3C
:102AC000616D656E740053616361722066696C614B
:102AD0006D656E746F005363617269636172652026
:102AE00066696C2E0056796A6D6F75742066696C24
:102AF000616D656E7400556E6C6F61642066696C03
:102B0000616D656E740047727A616E69650050721E
:102B10006563616C656E7461720050726572697391
:102B200063616C646100507265646568726576000B
:102B30005072656865617400557374617769656E7C
:102B4000696100416A7573746500496D706F7374D3
:102B5000617A696F6E69004E6173746176656E6942
:102B60000053657474696E6773004B616C696272BF
:102B70006F776163205A0047726164756172205AF1
:102B80000043616C696272617465205A004B616C2C
:102B90006962726F766174205A0043616C69627277
:102BA000617465205A004175746F646F7374726F3D
:102BB0006963205A3F004175746F204D6963726FDD
:102BC0007061736F205A3F004175746F20726567A2
:102BD0006F6C617265205A203F004175746F2064EC
:102BE0006F6C61646974205A203F004175746F20D6
:102BF00061646A757374205A203F00456E64737473
:102C00006F702061626F727400456E6473746F70D0
:102C10002061626F727400456E6473746F7020611E
:102C2000626F727400456E6473746F702061626FBE
:102C3000727400456E6473746F702061626F727499
:102C400000446F7374726F6A656E6965206F737983
:102C5000205A004D6963726F7061736F205A004291
:102C600061627973746570205A00446F6C616465A9
:102C70006E69206F7379205A004C69766520616413
:102C80006A757374205A00426162797374657020AA
:102C90005900426162797374657020590042616223
:102CA000797374657020590042616279737465703C
:102CB0002059004261627973746570205900426145
:102CC000627973746570205800426162797374652B
:102CD0007020580042616279737465702058004218
:102CE000616279737465702058004261627973740F
:102CF00065702058005A204F6666736574005A202C
:102D00004F6666736574005A204F6666736574007B
:102D10005A204F6666736574005A204F6666736565
:102D20007400486F6D6520582F59206265666F7278
:102D300065205A00486F6D6520582F5920626566DE
:102D40006F7265205A00486F6D6520582F592062B8
:102D500065666F7265205A00486F6D6520582F595F
:102D6000206265666F7265205A00486F6D65205855
:102D70002F59206265666F7265205A005A20707262
:102D80006F6265206F75742E20626564005A207032
:102D9000726F6265206F75742E20626564005A2020
:102DA00070726F6265206F75742E20626564005AC0
:102DB0002070726F6265206F75742E2062656400EA
:102DC0005A2070726F6265206F75742E2062656480
:102DD0000056796D656E6974205344004368616ED6
:102DE00067652053442063617264004368616E67C5
:102DF0006520534420636172640056796D656E6985
:102E000074205344004368616E6765205344206317
:102E100061726400496E69632E20534400496E69F3
:102E2000742E205344206361726400496E69742ECD
:102E3000205344206361726400496E69632E2053FD
:102E40004400496E69742E2053442063617264000B
:102E500057796D69656E69632066696C616D656E31
:102E6000740043616D626961722066696C616D65B1
:102E70006E746F0043616D62696172652066696C92
:102E8000616D656E746F0056796D656E697420664C
:102E9000696C616D656E74004368616E676520667C
:102EA000696C616D656E74004175746F5265747202
:102EB0002E004175746F526574722E004175746FE7
:102EC000526574722E004175746F526574722E00D3
:102ED0004175746F526574722E00556E5265742080
:102EE000205600556E52657420205600556E52656E
:102EF0007420205600556E52657420205600556E81
:102F0000526574202056005320556E5265742B6D07
:102F10006D005320556E5265742B6D6D0053205516
:102F20006E5265742B6D6D005320556E5265742B77
:102F30006D6D005320556E5265742B6D6D00556E8E
:102F4000526574202B6D6D00556E526574202B6D8B
:102F50006D00556E526574202B6D6D00556E526577
:102F600074202B6D6D00556E526574202B6D6D00B5
:102F7000486F70206D6D00486F70206D6D00486F58
:102F800070206D6D00486F70206D6D00486F70206F
:102F90006D6D005265747261637420205600526535
:102FA0007472616374202056005265747261637498
:102FB00020205600526574726163742020560052BE
:102FC00065747261637420205600537761702052DB
:102FD000652E6D6D00537761702052652E6D6D000A
:102FE000537761702052652E6D6D005377617020AC
:102FF00052652E6D6D00537761702052652E6D6D98
:103000000052657472616374206D6D005265747254
:10301000616374206D6D0052657472616374206D1C
:103020006D0052657472616374206D6D0052657439
:1030300072616374206D6D0053544F505045442E9F
:1030400020005041524144410041525245535441A5
:10305000544F200053544F505045442E2000535499
:103060004F505045442E20004B494C4C45442E2097
:103070000050415241444120444520454D4552476E
:103080002E0055434349534F20004B494C4C454477
:103090002E20004B494C4C45442E20004E6F206D95
:1030A0006F76652E0053696E206D6F76696D696568
:1030B0006E746F004E657373756E204D6F76696D1B
:1030C000656E746F004E6F206D6F76652E004E6FCB
:1030D000206D6F76652E004472756B2070727A6574
:1030E0007277616E79005072696E742061626F72DE
:1030F000746564005374616D70612061626F7274F5
:10310000697461005469736B2070726572757365C0
:103110006E005072696E742061626F727465640033
:10312000577A6E6F7769656E6965206472756B7525
:1031300000526573756D69656E646F20696D70729C
:10314000652E0052697072656E6469205374616DFA
:103150007061004F626E6F76656E69207469736B83
:103160007500526573756D696E67207072696E7453
:10317000005761697420666F7220757365722E2E18
:103180002E004573706572616E646F206F726465A6
:103190006E657300417474656E6469205574656E64
:1031A00074652E2E2E005761697420666F7220752B
:1031B0007365722E2E2E005761697420666F72201F
:1031C000757365722E2E2E00536C6565702E2E2E33
:1031D000005265706F736F2E2E2E00536F737065E3
:1031E0006E73696F6E652E2E2E00536C6565702EA2
:1031F0002E2E00536C6565702E2E2E004272616B70
:10320000206B61727479205344004E6F206861799D
:10321000207461726A657461205344004E6F2053BC
:1032200044204361727461005A61646E61205344AA
:10323000206B61727461004E6F2053442063617291
:1032400064004472756B207A205344004D656E759E
:10325000206465205344004D656E7520534420431F
:1032600061727461005469736B207A20534400507A
:1032700072696E742066726F6D205344005A6174D7
:10328000727A796D6163206472756B004465746550
:103290006E657220696D70726573696F6E00417240
:1032A0007265737461207374616D7061005A61732B
:1032B0007461766974207469736B0053746F702045
:1032C0007072696E74004B6F6E74796E756F776192
:1032D00063005265616E7564617220696D7072651C
:1032E000732E0052697072656E6469207374616D2B
:1032F000706100506F6B7261636F7661740052652C
:1033000073756D65207072696E740050727A6572A3
:10331000776163206472756B005061757361722010
:10332000696D70726573696F6E00506175736100CD
:10333000506F7A61737461766974207469736B007D
:103340005061757365207072696E74004E6173749C
:10335000726F696300416A757374617200416461E0
:10336000747461004C616469740054756E6500503A
:103370007269707261766100507265706172650089
:103380005072657061726500507269707261766129
:10339000005072657061726500496E666F726D6192
:1033A000636A65004D6F6E69746F72697A6172004D
:1033B00047756172646100496E666F726D61636525
:1033C00000496E666F2073637265656E004F626EB2
:1033D0006F7669740052656672657368005265663F
:1033E00072657368004F626E6F766974005265662D
:1033F00072657368004F626E6F76697420767963C8
:10340000686F7A6900526573746F726520666169CE
:103410006C7361666500526573746F7265206661D6
:10342000696C73616665004F626E6F7669742076B1
:103430007963686F7A6900526573746F726520668C
:1034400061696C7361666500556C6F7A6974207090
:10345000616D6574004C6F6164206D656D6F72798C
:10346000004C6F6164206D656D6F727900556C6FF3
:103470007A69742070616D6574004C6F6164206DB1
:10348000656D6F72790053746F7265206D656D6F35
:1034900072790053746F7265206D656D6F7279007B
:1034A00053746F7265206D656D6F72790053746F20
:1034B0007265206D656D6F72790053746F7265204F
:1034C0006D656D6F7279004C434420636F6E74724A
:1034D000617374004C434420636F6E747261737443
:1034E000004C434420636F6E7472617374004C43EC
:1034F0004420636F6E7472617374004C43442063A4
:103500006F6E74726173740046696C2E2044696139
:103510002E20330046696C2E204469612E20330032
:1035200046696C2E204469612E20330046696C2E5A
:10353000204469612E20330046696C2E2044696165
:103540002E20330046696C2E204469612E20320003
:1035500046696C2E204469612E20320046696C2E2B
:10356000204469612E20320046696C2E2044696136
:103570002E20320046696C2E204469612E203200D4
:1035800046696C2E204469612E20310046696C2EFC
:10359000204469612E20310046696C2E2044696107
:1035A0002E20310046696C2E204469612E203100A6
:1035B00046696C2E204469612E2031004520696ED9
:1035C000206D6D33004520696E206D6D3300452000
:1035D000696E206D6D33004520696E206D6D33007E
:1035E0004520696E206D6D330046696C616D656EB6
:1035F000740046696C616D656E740046696C616D3E
:10360000656E740046696C616D656E740046696C28
:10361000616D656E7400506F687962004D6F7469FA
:103620006F6E004D6F74696F6E00506F6879620045
:103630004D6F74696F6E0054656D7065726174755D
:1036400072610054656D70657261747572610054C9
:10365000656D7065726174757261005465706C6F30
:1036600074610054656D70657261747572650045B2
:1036700073746570732F6D6D004573746570732F6F
:103680006D6D004573746570732F6D6D00457374B7
:103690006570732F6D6D004573746570732F6D6D5C
:1036A000005A73746570732F6D6D005A7374657072
:1036B000732F6D6D005A73746570732F6D6D005AA2
:1036C00073746570732F6D6D005A73746570732F0A
:1036D0006D6D005973746570732F6D6D005973743F
:1036E0006570732F6D6D005973746570732F6D6DF8
:1036F000005973746570732F6D6D00597374657024
:10370000732F6D6D005873746570732F6D6D005855
:1037100073746570732F6D6D005873746570732FBB
:103720006D6D005873746570732F6D6D00587374F0
:103730006570732F6D6D00412D72657472616374D5
:1037400000412D7265747261637400412D7265745D
:103750007261637400412D7265747261637400411B
:103760002D7265747261637400416D61782000414F
:103770006D61782000416D61782000416D61782095
:1037800000416D617820005654726176206D696E3B
:10379000005654726176206D696E005654726176DF
:1037A000206D696E005654726176206D696E005608
:1037B00054726176206D696E00566D696E00566DAB
:1037C000696E00566D696E00566D696E00566D69C2
:1037D0006E00650065006500650065007A007A008E
:1037E0007A007A007A00790079007900790079000E
:1037F00078007800780078007800566D61782000B5
:10380000566D61782000566D61782000566D6178A4
:103810002000566D6178200056652D6A65726B0038
:1038200056652D6A65726B0056652D6A65726B0070
:1038300056652D6A65726B0056652D6A65726B0060
:10384000567A2D6A65726B00567A2D6A65726B0026
:10385000567A2D6A65726B00567A2D6A65726B0016
:10386000567A2D6A65726B005678792D6A65726B8F
:10387000005678792D6A65726B005678792D6A65E5
:10388000726B005678792D6A65726B005678792DC7
:103890006A65726B00416363656C00416363656CCC
:1038A00000416363656C00416363656C0041636361
:1038B000656C005049442D43005049442D4300504D
:1038C00049442D43005049442D43005049442D4361
:1038D000005049442D44005049442D44005049446F
:1038E0002D44005049442D44005049442D4400507B
:1038F00049442D49005049442D49005049442D491F
:10390000005049442D49005049442D490050494434
:103910002D50005049442D50005049442D50005026
:1039200049442D50005049442D50004F6666004FC9
:103930006666004F6666004F6666004F6666004F1B
:103940006E20004F6E20004F6E20004F6E20004F03
:103950006E20004175746F74656D70004175746FF1
:1039600074656D70004175746F74656D700041759C
:10397000746F74656D70004175746F74656D70005F
:1039800020022046616374002002204661637400B7
:1039900020022046616374002002204661637400A7
:1039A00020022046616374002002204D61780020CF
:1039B00002204D6178002002204D61780020022015
:1039C0004D6178002002204D6178002002204D6971
:1039D0006E002002204D696E002002204D696E00AD
:1039E0002002204D696E002002204D696E004B6F51
:1039F0006E74726F6C6100436F6E74726F6C004313
:103A00006F6E74726F6C004B6F6E74726F6C6100CE
:103A1000436F6E74726F6C00507275746F6B2032EE
:103A200000466C6F77203200466C6F772032005072
:103A30007275746F6B203200466C6F7720320050C5
:103A40007275746F6B203100466C6F7720310046C1
:103A50006C6F77203100507275746F6B20310046A7
:103A60006C6F77203100507275746F6B2030004698
:103A70006C6F77203000466C6F7720300050727585
:103A8000746F6B203000466C6F7720300050727A74
:103A900065706C797700466C756A6F00466C75735B
:103AA000736F00507275746F6B00466C6F770050C7
:103AB0007265646B6F73632077656E742E00566554
:103AC0006E74696C61646F720056656E746F6C61C0
:103AD00000527963686C6F73742076656E742E0083
:103AE00046616E2073706565640053746F6C696B1A
:103AF00000426173650050696174746F00426564CF
:103B00000042656400547279736B6133004E6F7AC2
:103B10007A6C6533004E6F7A7A6C65330054727933
:103B2000736B6133004E6F7A7A6C6533005472792F
:103B3000736B6132004E6F7A7A6C6532004E6F7A29
:103B40007A6C653200547279736B6132004E6F7A11
:103B50007A6C6532004479737A61004675736F72CE
:103B6000005567656C6C6F00547279736B61004E21
:103B70006F7A7A6C6500507265646B6F7363005680
:103B8000656C6F63696461640056656C636974C3D6
:103B9000A000527963686C6F73740053706565643C
:103BA00000506F73756E6F7574206F2031306D6DBE
:103BB000004D6F76652031306D6D004D6F7665205C
:103BC00031306D6D00506F73756E6F7574206F209E
:103BD00031306D6D004D6F76652031306D6D005068
:103BE0006F73756E6F7574206F20316D6D004D6F42
:103BF000766520316D6D004D6F766520316D6D00FD
:103C0000506F73756E6F7574206F20316D6D004D40
:103C10006F766520316D6D00506F73756E6F7574C2
:103C2000206F20302E316D6D004D6F766520302E67
:103C3000316D6D004D6F766520302E316D6D005009
:103C40006F73756E6F7574206F20302E316D6D003F
:103C50004D6F766520302E316D6D0045787472752C
:103C6000646572330045787472756465723300451B
:103C70007874727564657233004578747275646522
:103C800072330045787472756465723300457874D8
:103C9000727564657232004578747275646572324B
:103CA0000045787472756465723200457874727577
:103CB00064657232004578747275646572320045CD
:103CC00078747275646572004578747275736F727A
:103CD000004573747275736F726500457874727500
:103CE0006465720045787472756465720050727A0A
:103CF0006573756E6163205A004D6F766572205A48
:103D0000004D756F7669205A00506F73756E6F7530
:103D100074205A004D6F7665205A0050727A657390
:103D2000756E61632059004D6F7665722059004DA4
:103D3000756F7669205900506F73756E6F757420BA
:103D400059004D6F766520590050727A6573756E13
:103D500061632058004D6F7665722058004D756F75
:103D60007669205800506F73756E6F757420580017
:103D70004D6F766520580052756368206F73690037
:103D80004D6F76657220656A6573004D756F766953
:103D9000204173736500506F73756E6F7574206F7B
:103DA0007375004D6F766520617869730052657494
:103DB0007261637400526574726163740052657459
:103DC0007261637400526574726163740052657449
:103DD00072616374004578747275646F7661740003
:103DE0004578747275646500457874727564650011
:103DF0004578747275646F76617400457874727575
:103E00006465005A61706E6F7574207A64726F6AAF
:103E10000053776974636820706F776572206F66EE
:103E2000660053776974636820706F776572206FDE
:103E30006666005A61706E6F7574207A64726F6A7C
:103E40000053776974636820706F776572206F66BE
:103E500066005679706E6F7574207A64726F6A00AE
:103E600053776974636820706F776572206F6E0096
:103E700053776974636820706F776572206F6E0086
:103E80005679706E6F7574207A64726F6A0053771A
:103E90006974636820706F776572206F6E00577960
:103EA00063686C6F647A696300456E6672696172FB
:103EB00000526166667265646461005A63686C6191
:103EC00064697400436F6F6C646F776E0050726545
:103ED0006465687265762041425320636F6E6600A8
:103EE000507265686561742041425320636F6E664D
:103EF00000507265686561742041425320636F6EA3
:103F00006600507265646568726576204142532090
:103F1000636F6E660050726568656174204142533C
:103F200020636F6E66005072656465687265762006
:103F30004142532042656400507265686561742097
:103F40004142532042656400507265686561742087
:103F50004142532042656400507265646568726531
:103F60007620414253204265640050726568656165
:103F70007420414253204265640050726564656854
:103F80007265762041425320416C6C005072656826
:103F90006561742041425320416C6C005072656829
:103FA0006561742041425320416C6C00507265641D
:103FB00065687265762041425320416C6C005072F6
:103FC00065686561742041425320416C6C005072F9
:103FD00065646568726576204142532033005072F3
:103FE00065686561742041425320330050726568F2
:103FF00065617420414253203300507265646568E6
:1040000072657620414253203300507265686561C5
:1040100074204142532033005072656465687265B4
:1040200076204142532032005072656865617420E9
:1040300041425320320050726568656174204142EC
:104040005320320050726564656872657620414283
:1040500053203200507265686561742041425320DC
:104060003200507265646568726576204142532063
:1040700031005072656865617420414253203100FF
:10408000507265686561742041425320310050725E
:104090006564656872657620414253203100507234
:1040A0006568656174204142532031005072656437
:1040B000656872657620414253005072656865619B
:1040C000742041425300507265686561742041421A
:1040D00053005072656465687265762041425300F2
:1040E0005072656865617420414253005072656486
:1040F000656872657620504C4120636F6E66005093
:1041000072656865617420504C4120636F6E660073
:104110005072656865617420504C4120636F6E6613
:104120000050726564656872657620504C4120636A
:104130006F6E66005072656865617420504C412056
:10414000636F6E66005072656465687265762050B4
:104150004C4120426564005072656865617420506E
:104160004C4120426564005072656865617420505E
:104170004C412042656400507265646568726576E2
:1041800020504C412042656400507265686561743E
:1041900020504C412042656400507265646568722D
:1041A000657620504C4120416C6C0050726568650A
:1041B000617420504C4120416C6C00507265686500
:1041C000617420504C4120416C6C005072656465F4
:1041D0006872657620504C4120416C6C00507265CD
:1041E0006865617420504C4120416C6C00507265D0
:1041F00064656872657620504C41203300507265CA
:104200006865617420504C412033005072656865C8
:10421000617420504C4120330050726564656872AF
:10422000657620504C41203300507265686561749A
:1042300020504C4120330050726564656872657689
:1042400020504C41203200507265686561742050E6
:104250004C412032005072656865617420504C41B9
:1042600020320050726564656872657620504C415A
:104270002032005072656865617420504C412032D4
:104280000050726564656872657620504C4120313B
:10429000005072656865617420504C4120310050B7
:1042A00072656865617420504C4120310050726520
:1042B00064656872657620504C412031005072650B
:1042C0006865617420504C4120310050726564650E
:1042D0006872657620504C41005072656865617463
:1042E00020504C41005072656865617420504C410B
:1042F0000050726564656872657620504C410050CC
:1043000072656865617420504C41004E6173746140
:104310007620706F636174656B00536574206F72F3
:104320006967696E00536574206F726967696E0012
:104330004E617374617620706F636174656B0053B6
:104340006574206F726967696E004E61737461767F
:1043500020706F636174656B20686F6D65005365D5
:104360007420686F6D65206F6666736574730053A3
:10437000657420686F6D65206F6666736574730081
:104380004E617374617620706F636174656B206831
:104390006F6D650053657420686F6D65206F66668C
:1043A00073657473004175746F20686F6D65004CA0
:1043B0006C6576617220616C206F726967656E0052
:1043C0004175746F20486F6D65004175746F20688A
:1043D0006F6D65004175746F20686F6D650057796A
:1043E0006C61637A79632073696C6E696B690041F3
:1043F0007061676172206D6F746F726573004469DC
:10440000736162696C697461204D6F746F726900C9
:104410005679706E6F7574206D6F746F7279004489
:10442000697361626C652073746570706572730086
:104430004175746F7374617274004175746F737435
:10444000617274004175746F7374617274004175A8
:10445000746F7374617274004175746F73746172F8
:1044600074004D656E7520676C6F776E65004D65E5
:104470006E75207072696E636970616C004D656E57
:1044800075207072696E636970616C6500486C615B
:10449000766E69206E616269646B61004D61696E60
:1044A000004B617274612077796A657461005461B0
:1044B000726A657461207265746972616461005327
:1044C0004420436172642072696D6F737361004BA5
:1044D000617274612076796A6D75746100436172EE
:1044E000642072656D6F766564004B617274612043
:1044F000776C6F7A6F6E61005461726A65746120C7
:10450000636F6C6F63616461005344204361726444
:1045100020696E736572697461004B617274612009
:10452000766C6F7A656E61004361726420696E73A8
:104530006572746564005072757361206933206719
:104540006F746F7761005072757361206933206CEE
:1045500069737461005072757361206933207072E1
:104560006F6E746F2E005072757361206933207006
:10457000726970726176656E610050727573612048
:1045800069332072656164792E004D3834205820DB
:1045900059205A2045004D3234004D3233202573C6
:1045A000006175746F25692E67000A002F000A00EC
:1045B0002E0044656C6574696F6E206661696C6578
:1045C000642C2046696C653A200046696C6520645D
:1045D000656C657465643A002E002E002E002E0076
:1045E0004E6F772066726573682066696C653A2045
:1045F000004E6F7720646F696E672066696C653A5C
:1046000020002220706F73002220706172656E742A
:104610003A2200535542524F5554494E452043418A
:104620004C4C207461726765743A22007472796927
:104630006E6720746F2063616C6C207375622D67E8
:10464000636F64652066696C6573207769746820A0
:10465000746F6F206D616E79206C6576656C732E5A
:10466000204D4158206C6576656C2069733A0000D6
:10467000002110422063308440A550C660E77008D6
:104680008129914AA16BB18CC1ADD1CEE1EFF1315D
:1046900012100273325222B5529442F772D6623926
:1046A0009318837BB35AA3BDD39CC3FFF3DEE362AD
:1046B00024433420040114E664C774A44485546A76
:1046C000A54BB528850995EEE5CFF5ACC58DD5533D
:1046D00036722611163006D776F6669556B4465BC6
:1046E000B77AA719973887DFF7FEE79DD7BCC7C40D
:1046F00048E5588668A7784008611802282338CC16
:10470000C9EDD98EE9AFF9488969990AA92BB9F59C
:104710005AD44AB77A966A711A500A333A122AFD65
:10472000DBDCCBBFFB9EEB799B588B3BBB1AABA66C
:104730006C877CE44CC55C222C033C600C411CAEB5
:10474000ED8FFDECCDCDDD2AAD0BBD688D499D977C
:104750007EB66ED55EF44E133E322E511E700E9F05
:10476000FFBEEFDDDFFCCF1BBF3AAF599F788F88CC
:1047700091A981CAB1EBA10CD12DC14EF16FE1809D
:1047800010A100C230E3200450254046706760B994
:10479000839893FBA3DAB33DC31CD37FE35EF3B1ED
:1047A000029012F322D2323542145277625672EAE4
:1047B000B5CBA5A89589856EF54FE52CD50DC5E23D
:1047C00034C324A01481046674476424540544DB74
:1047D000A7FAB79987B8975FE77EF71DC73CD7D38D
:1047E00026F2369106B01657667676154634564C44
:1047F000D96DC90EF92FE9C899E9898AB9ABA944DD
:1048000058654806782768C018E1088238A3287DD3
:10481000CB5CDB3FEB1EFBF98BD89BBBAB9ABB752C
:104820004A545A376A167AF10AD01AB32A923A2EA3
:10483000FD0FED6CDD4DCDAABD8BADE89DC98D267C
:104840007C076C645C454CA23C832CE01CC10C1FB3
:10485000EF3EFF5DCF7CDF9BAFBABFD98FF89F17CC
:104860006E367E554E745E932EB23ED10EF01E22F1
:10487000004D3232302053256900203A2000004C90
:10488000414E472053454C20464F52434544002259
:1048900000205A3A0020593A0020453A00205A3A5E
:1048A0000020593A00583A0020002E0020423A00D9
:1048B00020453A00543A0020573A0020453A005427
:1048C0003A002042403A0020403A00202F003A00AF
:1048D000205400202F0020423A00202F006F6B2030
:1048E000543A002569206D696E2C20256920736576
:1048F0006300256920686F757273202569206D69D2
:104900006E75746573004D313130004D3239004D94
:104910006172203135203230313600436F6D70695D
:104920006C65643A2000286E6F6E652C20646566A5
:1049300061756C7420636F6E66696729004D6172E2
:1049400020313520323031362031313A34303A3569
:10495000300073746172740022002200FFFFFF00B8
:1049600000A0400000A040000000400000564300AE
:104970000046431FC5484300000000000000001F20
:10498000856B3E000056430000464300004943004B
:10499000000000000000001F856B3E6563686F3AF1
:1049A000004572726F723A0047312045343020461C
:1049B0003130300047312045373020463430300028
:1049C0004D383300473120452D38302046343030C3
:1049D000004D3833002D2D3A2D2D002D2D2D005357
:1049E00044000120000120004D36303000464C4587
:1049F00058202D20203233302F35300050502020C9
:104A0000202D20203235342F31303000484950538A
:104A1000202D20203232302F3130300050455420AC
:104A2000202D20203234302F393000504C412020AE
:104A30002D20203231302F35300041425320202D9F
:104A400020203235352F313030004D3834004D388C
:104A50003420582059205A2045004D3234004D3220
:104A60003320257300580059005A00457874727538
:104A700064657200473238004D38340047323820C0
:104A80005A00453344763666756C6C0052414D428F
:104A90006F31306100315F37356D6D002D2D2D2D5B
:104AA0002D2D2D2D2D2D2D2D004669726D776172C6
:104AB00065202D20322E322E340048617264636FDF
:104AC0006465642044656661756C74205365747414
:104AD000696E6773204C6F616465640046696C6140
:104AE0006D656E742073657474696E67733A2044E3
:104AF000697361626C6564002020204D3230302083
:104B0000440046696C616D656E74207365747469E8
:104B10006E67733A002020204D3230392053004117
:104B200075746F2D526574726163743A20533D3011
:104B300020746F2064697361626C652C203120746D
:104B40006F20696E74657270726574206578747216
:104B50007564652D6F6E6C79206D6F76657320615D
:104B600073207265747261637473206F7220726552
:104B7000636F766572696573002046002020204DC2
:104B80003230382053005265636F7665723A205395
:104B90003D4578747261206C656E67746820286D7D
:104BA0006D2920463A537065656420286D6D2F6D20
:104BB0002900205A002046002020204D3230372086
:104BC0005300526574726163743A20533D4C656EB4
:104BD00067746820286D6D2920463A5370656564B6
:104BE00020286D6D2F6D29205A3A205A4C69667421
:104BF00020286D6D29002044002049002020204DF0
:104C00003330312050005049442073657474696E0C
:104C100067733A00205A0020590020204D32303668
:104C2000205800486F6D65206F6666736574202894
:104C30006D6D293A00204500205A0020580020427E
:104C40000020540020204D3230352053004164763E
:104C5000616E636564207661726961626C65733A46
:104C600020533D4D696E20666565647261746520F0
:104C7000286D6D2F73292C20543D4D696E20747260
:104C80006176656C20666565647261746520286D67
:104C90006D2F73292C20423D6D696E696D756D20F5
:104CA0007365676D656E742074696D6520286D731A
:104CB000292C20583D6D6178696D756D20585920FB
:104CC0006A65726B20286D6D2F73292C20205A3D48
:104CD0006D6178696D756D205A206A65726B202848
:104CE0006D6D2F73292C2020453D6D6178696D75A0
:104CF0006D2045206A65726B20286D6D2F73290029
:104D000020540020204D323034205300416363652D
:104D10006C65726174696F6E3A20533D61636365BF
:104D20006C65726174696F6E2C20543D726574728B
:104D300061637420616363656C65726174696F6E31
:104D400000204500205A0020590020204D323031EB
:104D50002058004D6178696D756D20416363656C05
:104D600065726174696F6E20286D6D2F7332293AF8
:104D700000204500205A0020590020204D323033B9
:104D80002058004D6178696D756D206665656472A7
:104D90006174657320286D6D2F73293A00204500DA
:104DA000205A0020590020204D39322058005374D9
:104DB0006570732070657220756E69743A004530B5
:104DC0003A20005A3A2000593A2000583A20004D23
:104DD00053312C4D53322050696E730A005A002013
:104DE0005A3A00590020593A00580020583A0024F5
:104DF000F4D43050C38E20C2A24017828B7011129F
:104E00007A910D816CD90AA861E108C758660761DB
:104E10005143061E4B5D05C145A7041A4111040903
:104E20003D9803713931034036DB0265339102D47A
:104E3000305402802E1D02632CEE01752AC501B08C
:104E400028A001102781018F2564012B244B01E04C
:104E5000223401AC211F018D200D01801FFC008434
:104E60001EED00971DDF00B81CD200E61BC6002017
:104E70001BBC00641AB200B219A8000A19A0006A8B
:104E8000189900D117910040178B00B51684003196
:104E9000167E00B31579003A157300C7146F0058D9
:104EA000146A00EE1366008813630025135E00C7C2
:104EB000125B006C12570015125400C111510070A2
:104EC000114F0021114B00D61049008D10470046AC
:104ED00010440002104200C00F4000800F3E00420C
:104EE0000F3C00060F3B00CB0E3800930E37005CE2
:104EF0000E3500270E3400F30D3200C10D31009045
:104F00000D3000600D2E00320D2D00050D2C00D946
:104F10000C2B00AE0C2900850C29005C0C270035F9
:104F20000C27000E0C2600E80B2400C40B2400A064
:104F30000B23007D0B23005A0B2100390B21001895
:104F40000B2000F80A1F00D90A1E00BB0A1E009D94
:104F50000A1D00800A1D00630A1C00470A1B002C62
:104F60000A1B00110A1A00F7091A00DD091900C40A
:104F7000091900AB091900920917007B0918006391
:104F80000917004C09160036091600200916000AF8
:104F9000091500F5081500E0081400CC081400B845
:104FA000081400A4081400900813007D0812006B78
:104FB0000813005808120046081200340811002394
:104FC0000811001208110001081100F0071000E09C
:104FD000071000D0071000C0071000B0070F00A195
:104FE00007100091070E0083070F0074070F00657C
:104FF000070E0057070E0049070E003B070D002E55
:10500000070E0020070D0013070D0006070D00F91D
:10501000060C00ED060D00E0060C00D4060C00C8DE
:10502000060C00BC060C00B0060C00A4060B009990
:10503000060C008D060B0082060B0077060B006C39
:10504000060B0061060A0057060B004C060A0042D8
:10505000060A0038060A002E060A0024060A001A6C
:10506000060A001006090007060A00FD050900F4FB
:10507000050900EB050900E2050900D9050900D082
:10508000050900C7050900BE050900B5050800AD02
:10509000050800A50509009C050800940508008C7A
:1050A000050800840508007C050800740508006CEC
:1050B000050700650508005D050700560508004E58
:1050C00005070047050700400508003805070031BF
:1050D0000507002A050700230507001C0506001622
:1050E0000507000F0507000805060002050700FB7D
:1050F000040600F5040700EE040600E8040600E2DA
:10510000040700DB040600D5040600CF040600C92E
:10511000040600C3040600BD040600B7040600B17F
:10512000040500AC040600A6040600A00405009BCC
:1051300004060095040500900406008A0405008515
:10514000040500800406007A04050075040500705B
:105150000405006B04050066040500610405005C9D
:1051600004050057040500520405004D04050048DD
:10517000040500430405003E0404003A040500351C
:10518000040500300404002C040500270404002357
:105190000405001E0404001A04040016040500118E
:1051A0000404000D040400090405000404040000C4
:1051B000040400FC030400F8030400F4030400F0FA
:1051C000030400EC030400E8030400E4030400E02B
:1051D000030400DC030400D8030400D4030400D05B
:1051E000030400CC030400C8030300C50303002428
:1051F000F404D9201BC40C5C0E9804C4095F02653A
:10520000077101F405F900FB04B30048048700C1ED
:105210000369005803550003034500BE023A0084A9
:1052200002310053022A002902250004022000E472
:10523000011C00C8011900AF011700980114008477
:10524000011300710110006101100051010E0043B3
:10525000010D0036010B002B010B0020010B001586
:105260000109000C01090003010800FB000800F31C
:10527000000800EB000700E4000600DE000600D88E
:10528000000600D2000600CC000500C7000500C2E1
:10529000000500BD000400B9000400B5000400B121
:1052A000000400AD000400A9000400A5000300A252
:1052B0000003009F0004009B00030098000300957A
:1052C00000020093000300900003008D0002008B99
:1052D00000030088000200860002008400030081B1
:1052E0000002007F0002007D0002007B00020079C6
:1052F00000020077000100760002007400020072D4
:10530000000100710002006F0002006D0001006CDE
:105310000002006A000100690002006700010066E7
:1053200000010065000100640002006200010061EC
:10533000000100600001005F0002005D0001005CF0
:105340000001005B0001005A0001005900010058F3
:1053500000010057000100560001005500010054F3
:1053600000010053000000530001005200010051F1
:10537000000100500001004F0001004E0000004EEF
:105380000001004D0001004C0001004B0000004BEB
:105390000001004A000100490001004800000048E7
:1053A00000010047000100460000004600010045E2
:1053B00000000045000100440001004300000043DC
:1053C00000010042000000420001004100000041D5
:1053D000000100400001003F0000003F0001003ECE
:1053E0000000003E0001003D0000003D0001003CC7
:1053F0000000003C0000003C0001003B0000003BBE
:105400000001003A0000003A0001003900000039B4
:1054100000010038000000380000003800010037AB
:1054200000000037000100360000003600000036A2
:105430000001003500000035000000350001003497
:10544000000000340000003400010033000000338D
:105450000000003300010032000000320000003282
:105460000001003100000031000000310001003077
:1054700000000030000000300001002F0000002F6D
:105480000000002F0000002F0001002E0000002E61
:105490000000002E0001002D0000002D0000002D56
:1054A0000000002D0001002C0000002C0000002C4A
:1054B0000000002C0001002B0000002B0000002B3E
:1054C0000000002B0001002A0000002A0000002A32
:1054D0000000002A00010029000000290000002926
:1054E0000000002900000029000100280000002819
:1054F000000000280000002800000028000100270C
:1055000000000027000000270000002700000027FF
:1055100000010026000000260000002600000026F2
:1055200000000026000100250000002500000025E5
:1055300000000025000000250000002500010024D7
:1055400000000024000000240000002400000024CB
:1055500000010023000000230000002300000023BE
:1055600000000023000000230000002300010022AF
:1055700000000022000000220000002200000022A3
:105580000000002200010021000000210000002195
:105590000000002100000021000000210000002187
:1055A000000100200000002000000020000000207A
:1055B000000000200000002000000020000000206B
:1055C0000001001F0000001F0000001F0000001F5E
:1055D0000000001F0000001F0000001F0001001E4F
:1055E0000000001E0000001E0000001E0000000061
:1055F00000090A02080B0C0D070603040100000055
:10560000000000000000000000000000000000009A
:10561000000000000000000000000011100F00005A
:10562000000000000000000000000000000000007A
:10563000000000000000000000000000000000006A
:105640000000000000010210202008081020401077
:105650002040800201020108040201010204081036
:105660002040808040201008040201800402018054
:10567000402010080402010804020101020408107D
:105680002040800102040810204080100804088097
:1056900010204004408010204004800505050507C7
:1056A0000508080808020202020A0A08080404049D
:1056B00004010101010101010103030303030303C9
:1056C00003040707070C0C0C0C0C0C0C0C02020258
:1056D0000206060606060606060B0B0B0B0B0B0B4B
:1056E0000B07070A0A0A0A0A0A0505050404040842
:1056F00008000020002300260029002C002F003283
:10570000000001000003010601090100002200253C
:105710000028002B002E003100340002010000059B
:105720000108010B0100002100240027002A002DA0
:10573000003000330001010000040107010A0102EA
:105740004E414E494E495459494E46CDCCCC3D0A66
:10575000D7233C17B7D13877CC2B329595E6241F49
:10576000B14F0A000020410000C84200401C462002
:10577000BCBE4CCA1B0E5AAEC59D74005186C4A057
:10578000FFD3558611241FBECFEFD1E2DEBFCDBFC0
:1057900000E00CBF1DE0A0E0B2E0E4ECFEEC01E0B4
:1057A0000BBF02C007900D92A833B107D9F72CE1C7
:1057B000A8E3BDE001C01D92AD34B207E1F717E5E3
:1057C000C2E8D7E500E006C022970109FE010BBF41
:1057D0000E94EAE0CC37D10780E00807A9F70E94D1
:1057E00003D80C9451E70C940000CF93DF93EC01A5
:1057F0009C012C5F3F4F41E050E060E070E0898DFC
:105800009A8D0E949736882399F04D895E896F8919
:10581000788D452B462B472B59F44C815D816E8149
:105820007F814D8B5E8B6F8B788F99819068998388
:10583000DF91CF910895CF92DF92EF92FF920F9375
:105840001F93CF93DF93EC0189899A89AB89BC8937
:10585000803E9F4FAF41B10510F080E06BC0CE019C
:10586000C4DF8823D1F30E94AB34182F8823A9F317
:10587000E98DFA8DCC80DD80EE80FF8032E0C31AA6
:10588000D108E108F108058404C0CC0CDD1CEE1C35
:10589000FF1C0A94D2F786859785A089B189C80E26
:1058A000D91EEA1EFB1E81E080933E0DC092410F7F
:1058B000D092420FE092430FF092440F80E092E0CA
:1058C000E1E4FDE0DF019C011D9221503040E1F751
:1058D00001E0E98DFA8D8481081790F421E43DE020
:1058E000B701A601400F511D611D711D80913F0D33
:1058F0009091400D0E94665A8823E1F00F5FE9CF36
:10590000C12C82E0D82EE12CF12C058404C0CC0CF3
:10591000DD1CEE1CFF1C0A94D2F749895A896B8959
:105920007C894C0D5D1D6E1D7F1D498B5A8B6B8BC9
:105930007C8B812FDF91CF911F910F91FF90EF9082
:10594000DF90CF900895CF93DF93EC0141E0611198
:1059500001C040E06C857D858E859F850E94EB347B
:10596000882341F0888920E2829FC00111248F5B47
:10597000924F02C080E090E0DF91CF91089530E037
:1059800020E04EE2DC015C91503271F0383029F4B5
:10599000FB01E20FF11D40832F5FFB01E20FF11DC0
:1059A000DC015C9150832F5F3F5F01963B3051F7E4
:1059B000FB01E20FF11D10820895CF93DF93EB01FD
:1059C000FC012381211102C080E00EC02250223050
:1059D00020F48FE28883198206C060E0B4DF00976C
:1059E00099F3BE01CCDF81E0DF91CF910895FB01F7
:1059F0002BE030E231932150E9F7DC0190E027E021
:105A00003A2FEB2F8D9181110AC0DA013C93119648
:105A1000EC9381E0FB019081903239F525C08F3203
:105A2000A1F38E3219F0EAE8F1E008C02A30E1F083
:105A300098E02AE0E5CF31963817B1F03491311172
:105A4000FACF291788F03FED380F3E3568F431E082
:105A5000390FFB01E90FF11D9FE9980F9A3108F406
:105A600080528083932FCCCF80E008950F931F93B3
:105A7000CF93DF93EC018B018B81882311F080E0C1
:105A800042C0FB018789803139F18032C1F783E060
:105A90008B83F801428D538D648D758D4D8B5E8B9C
:105AA0006F8B788F9E012F5E3F4FC8010E94A235F9
:105AB000882329F31A8F098F81E089831C821D8234
:105AC0001E821F82188619861A861B861C861D86D2
:105AD0001E861F86188A17C082E08B831D8A1E8A45
:105AE0001F8A188EFB01408D518D60E070E095E0BB
:105AF000440F551F661F771F9A95D1F7498B5A8B14
:105B00006B8B7C8BD7CFDF91CF911F910F91089535
:105B10002F923F924F925F926F927F928F929F92BD
:105B2000AF92BF92CF92DF92EF92FF920F931F93AB
:105B3000CF93DF93EC015B016A018B81811103C07C
:105B40008FEF9FEFC7C0898180FFFACF49895A89BB
:105B50006B897C8988859985AA85BB852601612CFE
:105B6000712C8A019B01081B190B2A0B3B0B401659
:105B700051066206730618F06A01C81AD90A76013E
:105B80003E0124E0620E711CE114F10409F476C0B8
:105B9000488559856A857B854A0181E098222B8159
:105BA0001A012B01E9E05694479437942794EA951B
:105BB000D1F7898D9A8DFC01223049F4628D738D65
:105BC000848D958D620D731D841D951D3CC01481BF
:105BD0001150122181149104C1F4111116C0452BEA
:105BE000462B472B49F48D899E89AF89B88D8C83CC
:105BF0009D83AE83BF8309C04C815D816E817F81AF
:105C0000930121D7882309F49BCFE98DFA8D6C810C
:105C10007D818E819F81625071098109910905847E
:105C200004C0660F771F881F991F0A94D2F7268534
:105C3000378540895189620F731F841F951F610F3B
:105C4000711D811D911D20E032E02819390987015D
:105C50002E153F0508F489010115F2E01F0769F5CB
:105C60002091410F3091420F4091430F5091440FCA
:105C7000621773078407950719F41FC0C6012AC06D
:105C80009501AB01BC0180913F0D9091400D0E94A8
:105C9000F159882309F454CFA00EB11E8885998547
:105CA000AA85BB85800F911FA11DB11D888799878B
:105CB000AA87BB87E01AF10A67CF40E08CD6882319
:105CC00009F43ECFB4016F5B724FA801C5010E9479
:105CD00010E4E2CFDF91CF911F910F91FF90EF90F1
:105CE000DF90CF90BF90AF909F908F907F906F90FC
:105CF0005F904F903F902F900895CF93DF931F9226
:105D0000CDB7DEB741E050E0BE016F5F7F4F00DFEF
:105D1000019719F4898190E002C08FEF9FEF0F90F7
:105D2000DF91CF910895CF92DF92EF92FF920F9380
:105D30001F93CF93DF936C01EB017A01FC01838108
:105D4000823060F000851185228533850F7111271F
:105D500022273327012B022B032B11F08FEF5CC07E
:105D60004115510511F0F70110821DE040E250E0AD
:105D7000BE01C601CDDE8032910539F021E0892BCC
:105D800009F420E0822F819547C028812223C1F0A9
:105D9000253E61F32E3251F33B853F733F3061F472
:105DA000E114F10449F04A8D5B8D452B29F42F71E4
:105DB0003FEF320F343030F02B8523FDD7CF2CC08E
:105DC00080E02AC030E021503109129FC001139FAA
:105DD000900D1124F701E80FF91F298120832B81F1
:105DE00021832D8122832F812383298524832E855E
:105DF0002583288926832A8927832C8920872E8931
:105E00002187288D22872C8D23872E8D248728811A
:105E100026FFD2CF1586D0CFDF91CF911F910F9162
:105E2000FF90EF90DF90CF9008951F93CF93DF9373
:105E3000EC018B81823018F480E090E023C048852B
:105E400059856A857B85A5E0769567955795479531
:105E5000AA95D1F7142F1F70CE014FDF97FDECCF1D
:105E6000488559856A857B85415E5F4F6F4F7F4FBF
:105E7000488759876A877B8720E2129FC0011124D7
:105E80008F5B924FDF91CF911F9108954F925F9258
:105E90006F927F92AF92BF92CF92DF92EF92FF927A
:105EA0000F931F93CF93DF93EC016A017B012B814A
:105EB000222349F089899A89AB89BC89841795077F
:105EC000A607B70710F480E06BC0223009F463C066
:105ED000C114D104E104F10449F41C821D821E8224
:105EE0001F82188619861A861B8659C0888599854F
:105EF000AA85BB85E98DFA8DE585F0E03996AC0180
:105F0000BD0141505109610971090E2E04C07695F9
:105F10006795579547950A94D2F7970186010150E6
:105F200011092109310904C0369527951795079560
:105F3000EA95D2F7041715072607370720F0892BB3
:105F40008A2B8B2B49F48D899E89AF89B88D8C83E0
:105F50009D83AE83BF8304C0041B150B260B370B38
:105F6000280139015E0184E0A80EB11C41145104DE
:105F70006104710481F04C815D816E817F819501A6
:105F8000898D9A8D60D591E0491A51086108710890
:105F90008111ECCF05C0C886D986EA86FB8681E0F0
:105FA000DF91CF911F910F91FF90EF90DF90CF90F5
:105FB000BF90AF907F906F905F904F9008950F9338
:105FC0001F93CF93DF93EC018B818823D1F18981DB
:105FD00087FF32C061E0CE01B6DC8C01009789F109
:105FE000FC018081853E69F18B81823040F44989D2
:105FF0005A896B897C89448F558F668F778F4D893D
:106000005E896F89788DF801538F428F758B648B11
:10601000E091380DF091390D309759F0B8016A5E72
:106020007F4FC80148961995F801808D918D938B0B
:10603000828B89818F778983DF91CF911F910F9117
:106040008AC481E0888380E0DF91CF911F910F9116
:106050000895CF93DF93EC01B2DF1B82DF91CF91E4
:106060000895FC0123812111F4CF08954F925F928E
:106070006F927F92AF92BF92CF92DF92EF92FF9298
:106080000F931F93CF93DF9300D01F92CDB7DEB74E
:106090005C016A017B01FC0183818130E9F481812B
:1060A00081FF1AC0F50181899289A389B489841777
:1060B0009507A607B70780F0892B8A2B8B2B09F44D
:1060C00072C0F5014084518462847384B701A601D3
:1060D000C501DCDE811102C080E066C0F501818D62
:1060E000928DC114D104E104F10469F44589568903
:1060F0006789708D25D7882379F3F501158A168A6B
:10610000178A108E37C0F5014481558166817781E9
:106110009E012F5F3F4F97D48823F1F249815A8126
:106120006B817C81F501818D928DFC012789203165
:1061300039F4483FFFEF5F0761057105D8F407C0E8
:10614000483F2FEF520762072FE0720798F4F8D606
:10615000882309F4C1CFF501448155816681778197
:106160000FEF1FEF2FEF3FE0818D928D51D58823E8
:1061700009F4B2CFF501C18AD28AE38AF48A818117
:1061800080688183C5011BDF882309F4A5CFB7018F
:10619000A6014C145D046E047F0410F4B301A20147
:1061A000C50174DE01C081E00F900F900F900F9039
:1061B000DF91CF911F910F91FF90EF90DF90CF90E3
:1061C000BF90AF907F906F905F904F900895FF9237
:1061D0000F931F93CF93DF93EC01F42E80E2689F1F
:1061E000F0011124EF5BF24F8385817121F0842F40
:1061F000827109F04EC08091410F9091420FA091A1
:10620000430FB091440F8C879D87AE87BF87688B03
:106210004489558960E070E0BA0155274427028D12
:10622000138D20E030E0402B512B622B732B4D8BD4
:106230005E8B6F8B788F8385887151F4048D158DFB
:10624000268D378D098B1A8B2B8B3C8B81E00BC0F5
:106250008031F9F49E012F5E3F4F898D9A8D72D463
:106260008823B9F084E08B838F2D8F7089831C8203
:106270001D821E821F82188619861A861B86F4FECE
:106280000BC040E050E0BA01CE01F0DE811104C045
:1062900011C01B8280E00EC0F5FE0BC049895A89EF
:1062A0006B897C89CE01DF91CF911F910F91FF9077
:1062B000EDCD81E0DF91CF911F910F91FF90089577
:1062C000AF92BF92CF92DF92EF92FF920F931F9304
:1062D000CF93DF937C01EB016A01B22E898D9A8DF9
:1062E000F701928F818F40E050E0BA01CE01CEDD00
:1062F000A12C088519852A853B8589899A89AB89CE
:10630000BC89081719072A073B07A0F585E03695D1
:106310002795179507958A95D1F70F70CE0185DDE2
:10632000009709F481C0FC012081222311F0253E51
:10633000B9F4A1100EC04091410F5091420F6091ED
:10634000430F7091440FF70144875587668777871D
:10635000008BFC018081AA24A3948111CACF0AC0BA
:106360004BE050E0BC01C6010E9403E4892B09F018
:10637000C0CF58C08B2D8274823409F055C0AA203A
:1063800049F0F701008961E0C701DDDAEC0100970F
:1063900069F44AC08B81823009F446C0CE014BDAE1
:1063A000882309F441C0C1E4DDE000E080E2FE01A1
:1063B00011928A95E9F78BE0F601DE0101900D92CA
:1063C0008A95E1F7E091380DF091390D309739F069
:1063D000BE01625F7F4FCE014096199508C081E2F1
:1063E00098E2998B888B80E098E09F878E878889D8
:1063F00099899B8B8A8B998F888F8E859F859F8BA0
:106400008E8BA9D2882381F04B2D602FC701DF919D
:10641000CF911F910F91FF90EF90DF90CF90BF90A1
:10642000AF90D5CEB7FEF0CF80E0DF91CF911F9136
:106430000F91FF90EF90DF90CF90BF90AF900895B5
:106440003F924F925F926F927F928F929F92AF9204
:10645000BF92CF92DF92EF92FF920F931F93CF9351
:10646000DF93CDB7DEB7C354D1090FB6F894DEBFC2
:106470000FBECDBF5C016B0124965FAF4EAF24977A
:10648000522E1C8E1F8E19821C826115710511F40B
:1064900010E073C0FC0183818111FACF2496EEAD28
:1064A000FFAD249780818F3211F076011DC02496B4
:1064B000EEADFFAD249780818F3231F43196249672
:1064C000FFAFEEAF2497F3CFF60183818250823085
:1064D00060F3F601618D728DCE010196C7DA8823D3
:1064E000B9F2CE0101967C018E01045E1F4F380186
:1064F000FE0131964F01402E312E19C08823A9F19B
:1065000021E0AE01495C5F4FB701C801D9DE8823A5
:1065100009F4BECFEC14FD0411F0C7019ADD061595
:10652000170501F1942D832D7801092F182FAE0145
:106530004E5B5F4FBE01695C7F4F24968EAD9FAD71
:10654000249755DA882309F4A3CF2496EEADFFAD46
:10655000249780818F3291F631962496FFAFEEAF6B
:106560002497F3CF982D892DDFCF252DAE01495CDF
:106570005F4FB701C501A4DE182FCE01019671DD72
:10658000CE014C966EDD812FCD5BDF4F0FB6F894B8
:10659000DEBF0FBECDBFDF91CF911F910F91FF9056
:1065A000EF90DF90CF90BF90AF909F908F907F90B3
:1065B0006F905F904F903F900895CF93DF93EC01E1
:1065C00040E050E0BA0152DD882361F061E0CE0185
:1065D000BAD9009739F025EEFC0120831B82DF91A8
:1065E000CF91B9C180E0DF91CF9108951F93CF93F0
:1065F000DF93CDB7DEB76B970FB6F894DEBF0FBE53
:10660000CDBFAB0119821C8222E0BC01CE010196F4
:1066100017DF182F882321F0CE010196CEDF182F27
:10662000CE0101961EDD812F6B960FB6F894DEBF6A
:106630000FBECDBFDF91CF911F9108952F923F9252
:106640004F925F926F927F928F929F92AF92BF9282
:10665000CF92DF92EF92FF920F931F93CF93DF932E
:1066600000D01F921F92CDB7DEB78C015B013A01BB
:10667000DC0113968C9113978130C1F411968C91A3
:1066800081FF14C082FF18C0F801418952896389D3
:10669000748980859185A285B38584179507A6079F
:1066A000B70751F0C801F2DB811106C081E0F801A3
:1066B00080838FEF9FEF37C1630183C0D801599664
:1066C0008D919C915A97FC01F481F1501A012B0194
:1066D00069E056944794379427946A95D1F7F2214C
:1066E000FD834A0121E09222FF2309F476C080E075
:1066F00092E08819990976018C159D0508F47C01B2
:10670000D8015996ED91FC915A9714962D903D9091
:106710004D905C901797B2E02B1A31084108510850
:10672000058404C0220C331C441C551C0A94D2F767
:1067300086859785A089B189280E391E4A1E5B1E61
:10674000ED812E0E311C411C511CE114F2E0FF06BC
:1067500009F089C08091410F9091420FA091430FA1
:10676000B091440F82159305A405B50569F4109204
:106770003E0D8FEF9FEFDC018093410F9093420F0E
:10678000A093430FB093440F9501B201A1018091F2
:106790003F0D9091400D0E94665A882309F486CFE0
:1067A000F80180859185A285B3858E0D9F1DA11D61
:1067B000B11D80879187A287B387AE0CBF1CCE180E
:1067C000DF08D80118964D915D916D917C911B97D2
:1067D000C114D10409F072CF7AC08114910409F078
:1067E00086CF14964D915D916D917C9117974115CF
:1067F00051056105710559F455968D919D910D9046
:10680000BC91A02D0097A105B10539F520C09E01CE
:106810002F5F3F4F18D1882309F448CF89819A818F
:10682000AB81BC81F801218D328DF901278920319E
:1068300039F4883FFFEF9F07A105B10540F40DC073
:10684000883F2FEF9207A2072FE0B20730F0C80170
:106850000E94F52B81114BCF29CFF80184839583BA
:10686000A683B78344CF8114910411F5D8011896FB
:106870004D915D916D917C911B9751968D919D915C
:106880000D90BC91A02D481759076A077B0780F02F
:1068900062D0882309F40ACF81E080933E0D2092D4
:1068A000410F3092420F4092430F5092440F07C065
:1068B00041E0C201B1018FD0882309F4F7CEA701CE
:1068C000B501C4018F5B924F0E9410E469CF5196CD
:1068D0008D919D910D90BC91A02DF801218184177F
:1068E0009507A607B70738F4418B528B638B748BDF
:1068F000206821830CC08091380D9091390D892B2F
:1069000031F06114710419F02068F8012183D80175
:1069100011968C9183FD02C0C30105C0C8014FDBF5
:106920008111FACFC3CE0F900F900F900F900F9060
:10693000DF91CF911F910F91FF90EF90DF90CF905B
:10694000BF90AF909F908F907F906F905F904F908F
:106950003F902F900895CF9380913E0D8823B9F1F9
:106960004091410F5091420F6091430F7091440F3D
:1069700021E43DE080913F0D9091400D0E94665AC8
:10698000C82F811102C0C0E023C040913A0D509140
:106990003B0D60913C0D70913D0D41155105610518
:1069A000710591F021E43DE080913F0D9091400D03
:1069B0000E94665A882339F310923A0D10923B0DCB
:1069C00010923C0D10923D0D10923E0D01C0C1E0A1
:1069D0008C2FCF910895CF92DF92EF92FF92CF93B9
:1069E0006B017C01C42F8091410F9091420FA091C7
:1069F000430FB091440F8C159D05AE05BF05C9F03E
:106A0000AADF811102C080E018C021E43DE0B70197
:106A1000A60180913F0D9091400D0E94F15988236D
:106A200091F3C092410FD092420FE092430FF09247
:106A3000440F81E0C11180933E0DCF91FF90EF9004
:106A4000DF90CF9008958F929F92AF92BF92CF9296
:106A5000DF92EF92FF920F931F93CF93DF93EC019E
:106A60006A017B01890189859A85AB85BC85019680
:106A7000A11DB11D84179507A607B70710F480E084
:106A800054C08F89803129F49927872F762F652F5D
:106A90000BC08032A1F7CB01BA0127E0969587950C
:106AA000779567952A95D1F78B889C88AD88BE88A5
:106AB000680D791D8A1D9B1D8090410F9090420F9B
:106AC000A090430FB090440F681579058A059B0587
:106AD00081F48F89803191F4DD24EE24FF24F601C6
:106AE000EE0FFF1FEF5BF24F80819181A0E0B0E0DD
:106AF00016C040E070DF8111ECCFC1CFE894C7F839
:106B0000DD24EE24FF24F601EE0FFF1FEE0FFF1F22
:106B1000EF5BF24F80819181A281B381BF70F80158
:106B200080839183A283B38381E0DF91CF911F9112
:106B30000F91FF90EF90DF90CF90BF90AF909F901C
:106B40008F9008954F925F926F927F92AF92BF9213
:106B5000CF92DF92EF92FF920F931F93CF93DF9329
:106B600000D01F92CDB7DEB78C0149835A836B8367
:106B70007C835901C12CD12C7601412C42E0542E4A
:106B8000612C712C49815A816B817C819E012F5F20
:106B90003F4FC80158DF882341F1D301C201F801FA
:106BA000058404C0880F991FAA1FBB1F0A94D2F73F
:106BB000C80ED91EEA1EFB1E49815A816B817C8159
:106BC0008789803139F481E0483F5F4F6105710565
:106BD00038F4D8CF81E0483F5F4F6F4F7F4090F24D
:106BE000F501C082D182E282F3820F900F900F9064
:106BF0000F90DF91CF911F910F91FF90EF90DF9059
:106C0000CF90BF90AF907F906F905F904F9008951E
:106C10004F925F926F927F928F929F92AF92BF92AC
:106C2000CF92DF92EF92FF920F931F93CF93DF9358
:106C3000EC014A015B01280139014230510561052F
:106C4000710508F462C049855A856B857C854F5F64
:106C50005F4F6F4F7F4F481559056A057B0508F454
:106C600054C08F89803129F4FF24EB2CDA2CC92CF5
:106C70000CC0803209F049C07501640177E0F694D8
:106C8000E794D794C7947A95D1F74B895C896D893D
:106C90007E89C40ED51EE61EF71E41E0C701B6016F
:106CA0009ADE882391F19F89903159F49924AA247E
:106CB000BB24F401EE0FFF1FEF5BF24F51824082C5
:106CC00010C0E89487F89924AA24BB24F401EE0F9D
:106CD000FF1FEE0FFF1FEF5BF24F40825182628277
:106CE00073829A89923090F04D815E816F817885B0
:106CF0004C0D5D1D6E1D7F1D40933A0D50933B0D55
:106D000060933C0D70933D0D01C080E0DF91CF9109
:106D10001F910F91FF90EF90DF90CF90BF90AF90B9
:106D20009F908F907F906F905F904F9008952F92DB
:106D30003F924F925F926F927F928F929F92AF920B
:106D4000BF92CF92DF92EF92FF920F931F93CF9358
:106D5000DF93CDB7DEB72F970FB6F894DEBF0FBE27
:106D6000CDBF1C014C875D876E877F873B872A8755
:106D7000DC0119960D911D912D913C911C970F5F8F
:106D80001F4F2F4F3F4F0D831E832F833887EA8578
:106D9000FB8580809180A280B38081149104A1043E
:106DA000B10431F0FFEF8F1A9F0AAF0ABF0A10C07B
:106DB000DC018D909D90AD90BC90B1E0B9870C85C1
:106DC0001D852E853F85013011052105310509F00E
:106DD000198675016401412C512C3201F101818524
:106DE0009285A385B485481659066A067B0608F085
:106DF0004EC00D811E812F8138850C151D052E0575
:106E00003F0550F4F2E0CF2ED12CE12CF12CA2E082
:106E10008A2E912CA12CB12C9E012F5F3F4FB701E0
:106E2000A601C10110DE882391F149815A816B814D
:106E30007C81D701C6010196A11DB11D452B462BB2
:106E4000472B19F04C015D010FC0AC01BD01481981
:106E500059096A097B090C851D852E853F854017D8
:106E600051076207730741F01FEF411A510A610A87
:106E7000710A6C017D01B2CF0FEF1FEF2FEF3FE0E2
:106E8000B701A601C101C4DE8D83811113C01D822B
:106E90003DC02601370121E0421A510861087108FE
:106EA00097018601B301A201C101B2DE882379F303
:106EB000730162018C149D04AE04BF0450F3AA85D3
:106EC000BB854D915D916D917C9141155105610599
:106ED0007105A9F4EA85FB8580829182A282B38242
:106EE000F985FF2399F00FEF801A900AA00AB00AE3
:106EF000D1018D929D92AD92BC92139707C09501DE
:106F00008401C10185DE8111E5CFC1CF8D812F962E
:106F10000FB6F894DEBF0FBECDBFDF91CF911F91AA
:106F20000F91FF90EF90DF90CF90BF90AF909F9028
:106F30008F907F906F905F904F903F902F9008952B
:106F4000AF92BF92CF92DF92EF92FF920F931F9377
:106F5000CF93DF9300D01F92CDB7DEB75C016A01FB
:106F60007B0182E090E0A0E0B0E0F50180839183B6
:106F7000A283B3839E012F5F3F4FB701A601C501D6
:106F800062DD811102C080E023C000E010E09801C2
:106F9000B701A601C5013CDE8823A9F3C980DA80C8
:106FA000EB80FC80F5018789803149F481E0F8EFBE
:106FB000CF16FFEFDF06E104F10450F4DBCF81E0F0
:106FC00098EFC9169FEFD906E9069FE0F90690F2FF
:106FD0000F900F900F900F90DF91CF911F910F9115
:106FE000FF90EF90DF90CF90BF90AF9008957F9289
:106FF0008F929F92AF92BF92CF92DF92EF92FF92C9
:107000000F931F93CF93DF93EC01142F7093400DD8
:1070100060933F0D1F8A82E090E0A0E0B0E088839B
:107020009983AA83BB8310923E0D10923A0D109261
:107030003B0D10923C0D10923D0D8FEF9FEFDC0148
:107040008093410F9093420FA093430FB093440F4E
:10705000442349F1453008F0DEC040E060E070E0D4
:10706000CB01B9DC882309F4D6C020E1129FF001DE
:107070001124E151F14F80818F7709F0CCC08485D4
:107080009585A685B78584369105A105B10508F4D7
:10709000C2C0C084D184E284F384C114D104E10469
:1070A000F10421F4B8C0C12CD12C760140E0C70115
:1070B000B60191DC782E882309F4ADC080914C0D87
:1070C00090914D0D8115924009F0A5C03091510D60
:1070D000332309F4A0C080914F0D9091500D892B5E
:1070E00009F499C020914E0D222309F494C03A8BE3
:1070F0002C831D8630E041E050E06D85062FCA01EB
:10710000062E02C0880F991F0A94E2F72817390744
:1071100031F081E0860F8D87683078F37CC0209154
:10712000570D3091580D2115310519F040E050E010
:1071300008C02091650D3091660D4091670D50910A
:10714000680D2D833E834F83588780914F0D90911A
:10715000500D46015701880E991EA11CB11C8B8A47
:107160009C8AAD8ABE8AE091520DF091530DF98F41
:10717000E88FA091510DB0E00E94DAE0680D791D12
:107180008A1D9B1D6A8F7B8F8C8F9D8FB5E0EE0FC4
:10719000FF1FBA95E1F7E150FE4FEF2FFF27E6956D
:1071A000DC01CB018E0F9F1FA11DB11D8E879F8714
:1071B000A88BB98B8090540D9090550D811491043B
:1071C00019F0A12CB12C08C08090610D9090620D37
:1071D000A090630DB090640DA7019601281B390B98
:1071E0004A0B5B0BDA01C901880D991DAA1DBB1D55
:1071F00004C0B695A795979587950A95D2F7898784
:107200009A87AB87BC87853F3FE09307A105B1050F
:1072100020F48CE08F8B712C15C0853F9F4FA1050A
:10722000B10510F480E10DC080916D0D90916E0D4F
:10723000A0916F0DB091700D8A8F9B8FAC8FBD8F19
:1072400080E28F8B872DDF91CF911F910F91FF905F
:10725000EF90DF90CF90BF90AF909F908F907F90F6
:1072600008954F925F926F927F928F929F92AF920A
:10727000BF92CF92DF92EF92FF920F931F93CF9323
:10728000DF932C0124EF33E081E090E0F901459198
:107290005491441655060CF062C0AC01415051099E
:1072A000DA01AA0FBB1FAA0FBB1FAE50BC4FFD01D6
:1072B00065917491440F551F440F551F40515C4F09
:1072C000FA0165907490FC01EE0FFF1FEE0FFF1F97
:1072D000EE50FC4FA590B490FD0105911491F90179
:1072E000C591D491FA0185909490882777FD809577
:1072F000982F0E9454DD6B017C01B2016619770959
:10730000882777FD8095982F0E9454DD2B013C0142
:10731000B501601B710B882777FD8095982F0E941F
:1073200054DD9B01AC01C301B2010E9487DF2B0138
:107330003C01BE0168197909882777FD8095982F4F
:107340000E9454DD9B01AC01C301B2010E94B9DC73
:107350009B01AC01C701B6010E94D9DB11C00196A7
:107360002C5F3F4F8D33910509F090CFE2EEF4E0B2
:1073700065917491882777FD8095982F0E9454DD40
:10738000DF91CF911F910F91FF90EF90DF90CF9001
:10739000BF90AF909F908F907F906F905F904F9035
:1073A00008954F925F926F927F928F929F92AF92C9
:1073B000BF92CF92DF92EF92FF920F931F93CF93E2
:1073C000DF932C01662371F1E1EAF9E484918823CB
:1073D00041F09091C00095FFFCCF8093C60031969C
:1073E000F5CF70E04AE050E08BE295E10E9487B76C
:1073F000E9E5F2E08491882341F09091C00095FF87
:10740000FCCF8093C6003196F5CF8091C00085FFF8
:10741000FCCF8AE08093C6000E94586460E070E070
:10742000CB017EC024E733E081E090E0F901459193
:107430005491441655060CF062C0AC0141505109FC
:10744000DA01AA0FBB1FAA0FBB1FAE58BC4FFD012C
:1074500065917491440F551F440F551F40595C4F5F
:10746000FA0165907490FC01EE0FFF1FEE0FFF1FF5
:10747000EE58FC4FA590B490FD0105911491F901CF
:10748000C591D491FA0185909490882777FD8095D5
:10749000982F0E9454DD6B017C01B20166197709B7
:1074A000882777FD8095982F0E9454DD2B013C01A1
:1074B000B501601B710B882777FD8095982F0E947E
:1074C00054DD9B01AC01C301B2010E9487DF2B0197
:1074D0003C01BE0168197909882777FD8095982FAE
:1074E0000E9454DD9B01AC01C301B2010E94B9DCD2
:1074F0009B01AC01C701B6010E94D9DB11C0019606
:107500002C5F3F4F8032910509F090CFEEEEF3E013
:1075100065917491882777FD8095982F0E9454DD9E
:10752000DF91CF911F910F91FF90EF90DF90CF905F
:10753000BF90AF909F908F907F906F905F904F9093
:10754000089560E080919A0F90919B0F2ADF6093DD
:10755000960F7093970F8093980F9093990F809147
:10756000940F9091950F7DDE6093900F7093910F23
:107570008093920F9093930F8FB7F8941092880F87
:107580008FBF089520911402309115024091160288
:107590005091170260E070E08FE793E40E94B9DC3D
:1075A0006093680F7093690F80936A0F90936B0FCD
:1075B000089597FF03C080918F0F04C0FC01EE591E
:1075C000F04F808190E00895CF93DF93D82FC62F9E
:1075D000C19561E00E9463D66C2F8D2F0E949CD6CE
:1075E0006C2F70E08D2FDF91CF910C9459D5CF93F4
:1075F000C1E020E030E048E452E46091960F7091E1
:10760000970F8091980F9091990F0E94B5DE1816F0
:107610000CF0C0E06C2F88E090E0CF91D5CF2F9296
:107620003F924F925F926F927F928F929F92AF9212
:10763000BF92CF92DF92EF92FF920F931F93CF935F
:10764000DF93CDB7DEB728970FB6F894DEBF0FBE35
:10765000CDBF8091880F882309F4F8C172DF809034
:10766000960F9090970FA090980FB090990F00915F
:107670009E0F10919F0FB801882777FD8095982F56
:107680000E9454DDA50194010E94D8DB6B017C01AE
:107690006093700F7093710F8093720F9093730FBC
:1076A00020E030E040E251E40E94B5DE181624F4F8
:1076B00081E08093670FF7C020E030E040E251ECBA
:1076C000C701B6010E94B2DC87FD02C0012B21F484
:1076D00081E08093670F0CC18091670F882351F080
:1076E0001092840F1092850F1092860F1092870FC0
:1076F0001092670F209118023091190240911A02DE
:1077000050911B02C701B6010E9487DF69837A830B
:107710008B839C8360937C0F70937D0F80937E0F8F
:1077200090937F0F2091840F3091850F4091860FA9
:107730005091870FC701B6010E94D9DB2B013C0194
:1077400020906C0F30906D0F10916E0F00916F0FA5
:107750009101412F502F0E94B2DC87FD14C0209070
:10776000680F3090690F10916A0F00916B0F9101B3
:10777000412F502FB201C3010E94B5DE18161CF034
:107780001201162D072DC101A12FB02F8093840F58
:107790009093850FA093860FB093870F20911402CA
:1077A000309115024091160250911702B101812FBC
:1077B000902F0E9487DF6D837E838F8398876093ED
:1077C000780F7093790F80937A0F90937B0F2091AD
:1077D000800F3091810F4091820F5091830FC5012E
:1077E000B4010E94D8DB2091100230911102409127
:1077F0001202509113020E9487DF20ED3CEC4CE412
:107800005DE30E9487DF2B013C0123E333E343E781
:107810005FE36091740F7091750F8091760F909176
:10782000770F0E9487DF9B01AC01C301B2010E9468
:10783000D9DB2B013C016093740F7093750F80931B
:10784000760F9093770F2D813E814F815885698106
:107850007A818B819C810E94D9DBA30192010E94D5
:10786000D8DB2B013C0120E030E04FE753E40E94DD
:10787000B5DE20E030E0A9011816E4F4C701B60136
:107880000E94B5DE18167CF4A7019601B101812F84
:10789000902F0E94D8DB6093840F7093850F8093A4
:1078A000860F9093870F412C512C9FE7692E93E40C
:1078B000792E21C0C301B2010E94B2DC87FF1BC038
:1078C00020E030E0A901C701B6010E94B2DC87FFC9
:1078D0000FC0A7019601B101812F902F0E94D8DB24
:1078E0006093840F7093850F8093860F9093870F1A
:1078F000412C512C32018092800F9092810FA092E6
:10790000820FB092830F60915A0F70915B0F88279E
:1079100077FD8095982F0E9454DD9B01AC01C50135
:10792000B4010E94B5DE1816DCF460910802709173
:107930000902882777FD8095982F0E9454DD9B01CE
:10794000AC01C501B4010E94B2DC87FF09C0C301CC
:10795000B2010E9421DD759567956093620F02C0A8
:107960001092620F0E9443D700915E0F10915F0F3B
:107970002091600F3091610F601B710B820B930B94
:10798000653C79408105910558F031DE0E9443D76E
:1079900060935E0F70935F0F8093600F9093610F01
:1079A0000E9443D70091630F1091640F2091650FDF
:1079B0003091660F601B710B820B930B683873411B
:1079C0008105910508F442C00E9443D76093630F7C
:1079D0007093640F8093650F9093660FC090900F23
:1079E000D090910FE090920FF090930F20E030E054
:1079F00040E751E4C701B6010E94B5DE18161CF538
:107A000020E030E046E153E4C701B6010E94B2DC59
:107A100087FF19C060919C0F70919D0F882777FD9B
:107A20008095982F0E9454DD9B01AC01C701B601DF
:107A30000E94B5DE87FD03C010928F0F07C08FE74D
:107A400080938F0F03C010928F0FA59828960FB6C2
:107A5000F894DEBF0FBECDBFDF91CF911F910F9184
:107A6000FF90EF90DF90CF90BF90AF909F908F905E
:107A70007F906F905F904F903F902F900895CF939D
:107A8000DF9310926C0F10926D0F10926E0F109288
:107A90006F0F2091140230911502409116025091FF
:107AA000170260E070E08FE793E40E94B9DC609316
:107AB000680F7093690F80936A0F90936B0F6D9AA4
:107AC000809101018061809301019D9A8091010163
:107AD00088608093010187ED80937A0010927E0088
:107AE00010927D0080917E00816080937E00809165
:107AF0007E00826080937E0080917E00846080930F
:107B00007E0080E888BD80916E00846080936E0066
:107B10006AEF70E080E090E00E9472D78FE090E022
:107B200090935B0F80935A0F60E080910A029091CE
:107B30000B0237DC20E030E040E751E40E94B2DC89
:107B400087FF0AC080910A0290910B0240979093A0
:107B50000B0280930A02E8CF86E391E0909309023A
:107B60008093080260E080915C0F90915D0F19DCBA
:107B700020E030E04BE953E40E94B5DE181654F4DF
:107B800080915C0F90915D0F409690935D0F809374
:107B90005C0FE8CFC091580FD091590FCE0161DB37
:107BA00020E030E046E153E40E94B5DE181634F4DC
:107BB0006096D093590FC093580FECCFDF91CF91BF
:107BC0000895089510929F0F10929E0F10929D0F8E
:107BD00010929C0F1092620F759810929D0F109248
:107BE0009C0F10928F0FA59808952F923F924F925D
:107BF0005F926F927F928F929F92AF92BF92CF923D
:107C0000DF92EF92FF920F931F93CF93DF93CDB745
:107C1000DEB7AE970FB6F894DEBF0FBECDBF6B8F49
:107C20007C8F8D8F292E5A8749873CA72BA70E94CE
:107C300043D76F8F78A389A39AA30E9443D76FA3DA
:107C400078A789A79AA729853A85121613061CF0EA
:107C5000E4EEFBE017C0E7EFFBE08191882339F009
:107C60009091C00095FFFCCF8093C600F6CF809125
:107C7000C00085FFFCCF1BC29091C00095FFFCCFD8
:107C80008093C60081918111F7CF8091C00085FF5C
:107C9000FCCF8AE08093C60095DF49855A858FE73F
:107CA000452B99F180938F0F8F8D98A1A9A1BAA12F
:107CB000898B9A8BAB8BBC8B8D879E87AF87B88B5C
:107CC0001D8290E4988FACE1A98FB6E4BA8F1DA60F
:107CD0001D8A1E8A1F8A2FE730E040E050E029838A
:107CE0003A834B835C83EFE74E2E512C612C712C31
:107CF0001BA21CA21DA21EA231E03E8F1C861B8669
:107D0000312C00E010E01EA605C08093620FCCCF9E
:107D10000E945A988091880F882309F4F6C011DCDC
:107D200049855A85452B51F03090900F0091910F65
:107D30001091920F5091930F5EA709C03090960F4B
:107D40000091970F1091980F8091990F8EA7232D76
:107D5000302F412F5EA56DA57D898E899F890E9458
:107D6000B5DE18162CF03DA60D8B1E8B9EA59F8BA5
:107D7000232D302F412F5EA56D81788D898D9A8DB1
:107D80000E94B2DC87FD05C03D82088F198FAEA529
:107D9000AA8F0E9443D72FA138A549A55AA5621BD7
:107DA000730B840B950B653C79408105910538F088
:107DB0001EDC0E9443D76FA378A789A79AA74E8D90
:107DC000442309F44FC02B8D3C8D4D8D522D632DD6
:107DD000702F812F9EA50E94B5DE18160CF095C05D
:107DE0000E9443D729893A894B895C89621B730BAE
:107DF000840B950B693873418105910508F485C0A2
:107E0000D301C20129813A814B815C81821B930B92
:107E1000A40BB50B49855A85B595A7959795879578
:107E2000452B19F080938F0F02C08093620F0E9440
:107E300043D76D877E878F87988BDC01CB0129899B
:107E40003A894B895C89821B930BA40BB50B8BA3DE
:107E50009CA3ADA3BEA33B8D3DA74C8D4D8B5D8DEB
:107E60005E8B2F8A2B8D3C8D4D8D522D632D702F67
:107E7000812F9EA50E94B2DC87FFEEC20E9443D7ED
:107E80002D853E854F855889621B730B840B950B9E
:107E9000693873418105910508F4DEC20E9443D719
:107EA000698B7A8B8B8B9C8BDC01CB012D853E857E
:107EB0004F855889821B930BA40BB50B4B855C85B2
:107EC000452B09F010C189819A81AB81BC81840D59
:107ED000951DA61DB71D29853A85B595A79597953A
:107EE0008795232B09F4B5C280938F0F4B855C8552
:107EF0004F5F5F4F5C874B875B8D5D838C8D888F79
:107F00009D8D998F2A8EA1E0AE8F20E030E040EA6F
:107F100051E46B8D7C8D8D8D922D0E94D9DB9B0160
:107F2000AC01632D702F812F9EA50E94B5DE18161F
:107F300094F4EFEFF2E08491882341F09091C00037
:107F400095FFFCCF8093C6003196F5CF8091C0009D
:107F500085FFFCCFACC00E9443D72F8D38A149A12B
:107F60005AA1621B730B840B950B613D7740810511
:107F7000910508F44FC049855A85452B81F0E09062
:107F80008F0FF12CE9EFF2E084918823C1F09091FA
:107F9000C00095FFFCCF8093C6003196F5CFE090EE
:107FA000620FF12CE3EFF2E08491882341F090918D
:107FB000C00095FFFCCF8093C6003196F5CF22E03C
:107FC00030E0432D502F612F7EA58BE295E10E947A
:107FD0005DB8EFEEF2E08491882341F09091C0000B
:107FE00095FFFCCF8093C6003196F5CF4AE050E074
:107FF000B7018BE295E10E9487B78091C00085FFB1
:10800000FCCF8AE08093C6000E9443D76F8F78A38D
:1080100089A39AA30E9443D76B017C010E9443D796
:1080200089889A88AB88BC882D853E854F8558897C
:10803000820E931EA41EB51EC818D908EA08FB08B4
:10804000C60ED71EE81EF91E31E8C3163FE4D3065C
:1080500032E1E306F10490F0E2EDF2E0849188234E
:1080600041F09091C00095FFFCCF8093C6003196FF
:10807000F5CF8091C00085FFFCCF19C04B855C8592
:108080008BA59CA5841795070CF042CEE6E7F2E09D
:108090008491882341F09091C00095FFFCCF80939C
:1080A000C6003196F5CF8091C00085FFFCCF8AE0F5
:1080B0008093C600AE960FB6F894DEBF0FBECDBF5C
:1080C000DF91CF911F910F91FF90EF90DF90CF90B4
:1080D000BF90AF909F908F907F906F905F904F90E8
:1080E0003F902F9008958BA09CA0ADA0BEA0880EBD
:1080F000991EAA1EBB1E2BA13CA14DA15EA1281B4F
:10810000390B4A0B5B0BCA01B90129813A814B81BA
:108110005C810E944DE0A50194010E94B2E0240D13
:10812000351D461D571D243131054105510504F10A
:1081300029013A013CEE43165104610471042CF00C
:108140006BEE462E512C612C712C40E844165104E4
:1081500061047104DCF08EEF90E0A0E0B0E08419DF
:108160009509A609B70989839A83AB83BC8312C09A
:1081700054E1452E512C612C712C24E130E040E07B
:1081800050E029833A834B835C8304C049825A823E
:108190006B827C82E8E6F3E08491882341F0909141
:1081A000C00095FFFCCF8093C6003196F5CF2AE042
:1081B00030E0B301A2018BE295E10E945CB7E3E6F7
:1081C000F3E08491882341F09091C00095FFFCCFAB
:1081D0008093C6003196F5CF2AE030E049815A817C
:1081E0006B817C818BE295E10E945CB7ECE5F3E06A
:1081F0008491882341F09091C00095FFFCCF80933B
:10820000C6003196F5CF22E030E04D81588D698D62
:108210007A8D8BE295E10E945DB8E5E5F3E084910B
:10822000882341F09091C00095FFFCCF8093C60059
:108230003196F5CF22E030E04DA55D896E897F89CA
:108240008BE295E10E945DB88091C00085FFFCCF74
:108250008AE08093C6002B853C85233031050CF4E1
:1082600032CE69817A818B819C810E9454DD20E02D
:1082700030E040E850E40E9487DF6B017C012D81F3
:10828000388D498D5A8D6DA57D898E899F890E9473
:10829000D8DB20ED3FE049E450E40E9487DF20E096
:1082A00030E040E05FE30E9487DF9B01AC01C70143
:1082B000B6010E94B9DC6B017C01C501B4010E94CA
:1082C00054DD20E030E04AE754E40E94B9DC4B0181
:1082D0005C01EFE4F3E08491882341F09091C000C9
:1082E00095FFFCCF8093C6003196F5CF22E030E0B9
:1082F000B701A6018BE295E10E945DB8E9E4F3E0E5
:108300008491882341F09091C00095FFFCCF809329
:10831000C6003196F5CF22E030E0B501A4018BE232
:1083200095E10E945DB88091C00085FFFCCF8AE096
:108330008093C6002AE939E949E15FE3C701B60144
:108340000E9487DF6B017C019B01AC010E94D9DB9D
:10835000A50194010E94B9DC6D837E838F83988789
:10836000A5019401C701B6010E9487DF20E030E03B
:1083700040E05EE30E9487DF4B015C01EBE3F3E04A
:108380008491882341F09091C00095FFFCCF8093A9
:10839000C6003196F5CF8091C00085FFFCCF8AE002
:1083A0008093C600E5E3F3E08491882341F0909147
:1083B000C00095FFFCCF8093C6003196F5CF22E038
:1083C00030E0B701A6018BE295E10E945DB8809193
:1083D000C00085FFFCCF8AE08093C600EFE2F3E0A7
:1083E0008491882341F09091C00095FFFCCF809349
:1083F000C6003196F5CF22E030E04D815E816F817D
:1084000078858BE295E10E945DB88091C00085FF80
:10841000FCCF8AE08093C600E9E2F3E084918823F0
:1084200041F09091C00095FFFCCF8093C60031963B
:10843000F5CF22E030E0B501A4018BE295E10E9486
:108440005DB88091C00085FFFCCF8AE08093C600B4
:108450003ACD8093620F4ACD1E8E57CDCF93C82F51
:10846000B1DB0E94A769811134C0E1EAF9E494917B
:10847000992341F08091C00085FFFCCF9093C60006
:108480003196F5CF6C2F70E04AE050E08BE295E139
:108490000E9487B78091C00085FFFCCF8AE080935F
:1084A000C600ECE2F2E08491882341F09091C00094
:1084B00095FFFCCF8093C6003196F5CF8091C00028
:1084C00085FFFCCF8AE08093C6008FE192E00E9496
:1084D000CB97CF910C944F69CF93C82F73DB0E9439
:1084E000A769811134C0E1EAF9E49491992341F03C
:1084F0008091C00085FFFCCF9093C6003196F5CFE8
:108500006C2F70E04AE050E08BE295E10E9487B763
:108510008091C00085FFFCCF8AE08093C600E2EF27
:10852000F1E08491882341F09091C00095FFFCCF49
:108530008093C6003196F5CF8091C00085FFFCCFB7
:108540008AE08093C60085EE91E00E94CB97CF91A0
:108550000C944F69A5980E94A769811125C0E1EA92
:10856000F9E48491882341F09091C00095FFFCCFFD
:108570008093C6003196F5CFEBEAF1E08491882331
:1085800041F09091C00095FFFCCF8093C6003196DA
:10859000F5CF8091C00085FFFCCF8AE08093C600B4
:1085A0008AE991E00E94CB970C944F691F920F9239
:1085B0000FB60F9211240BB60F920F931F932F93A8
:1085C0003F934F935F936F937F938F939F93AF935B
:1085D000BF93CF93DF93EF93FF93809107028111B5
:1085E00012C08091620F8093570F882311F0759A03
:1085F00001C0759880918F0F8093560F882311F0DA
:10860000A59A01C0A5989091570F809107029817DD
:1086100008F475989091560F80910702981708F406
:10862000A598809107028F5F8F77809307028091D2
:10863000060290E08B30910508F093C0FC01EE58E3
:10864000FF4F0C94CEE010927B0080E480937C007E
:1086500080917A00806480937A000E94D49781E0B0
:1086600019C020917800309179008091520F90913B
:10867000530FA091540FB091550F820F931FA11D5E
:10868000B11D8093520F9093530FA093540FB0934A
:10869000550F82E08093060264C010927B0082E452
:1086A00080937C0080917A00806480937A000E949D
:1086B000D49783E0EFCF20917800309179008091BA
:1086C0004E0F90914F0FA091500FB091510F820F0C
:1086D000931FA11DB11D80934E0F90934F0FA09338
:1086E000500FB093510F84E0D5CF10927B0081E4FE
:1086F00080937C0080917A00806480937A000E944D
:10870000D49785E0C7CF209178003091790080918F
:108710004A0F90914B0FA0914C0FB0914D0F820FCB
:10872000931FA11DB11D80934A0F90934B0FA093EF
:108730004C0FB0934D0F86E0ADCF0E94D49787E0E9
:10874000A9CF88E0A7CF0E94D49789E0A3CF109249
:1087500006028091490F8F5F8093490F02C01092EB
:1087600006028091490F803108F463C08091880F20
:10877000811110C08091520F9091530F90939B0FD5
:1087800080939A0F80914E0F90914F0F9093950F79
:108790008093940F81E08093880F1092490F10927C
:1087A000520F1092530F1092540F1092550F1092B7
:1087B0004A0F10924B0F10924C0F10924D0F1092C7
:1087C000450F1092460F1092470F1092480F1092CB
:1087D0004E0F10924F0F1092500F1092510F209188
:1087E0009A0F30919B0F80915C0F90915D0F8217D3
:1087F000930714F080E032DE20919A0F30919B0FA6
:1088000080910A0290910B022817390714F080E03A
:1088100063DE2091940F3091950F8091580F9091C5
:10882000590F821793072CF010929D0F10929C0FF6
:1088300091DE00E010E0E801CC0FDD1FC757D04FFC
:10884000888199811816190644F461E0802F0E94EE
:1088500073C188819981019709C0892B49F060E033
:10886000802F0E9473C188819981019699838883A2
:108870000F5F1F4F03301105F1F6FF91EF91DF916C
:10888000CF91BF91AF919F918F917F916F915F91A8
:108890004F913F912F911F910F910F900BBE0F9011
:1088A0000FBE0F901F9018952CEA35EC47E25EE35F
:1088B0000C9487DF2CEA35EC47E25EE30C94B9DCDC
:1088C0002CEA35EC47E25EE30C94B9DC2CEA35EC9B
:1088D00047E25EE30C9487DFCF93DF93EC0160E027
:1088E0008E810E949CD681E090E00E9496D761E044
:1088F0008E810E949CD681E090E00E9496D760E035
:108900008E810E949CD684E690E0DF91CF910C94FA
:1089100096D7CF92DF92EF92FF920F931F93CF9350
:10892000DF937C01C0E0D0E0C62ED12C87010C0F74
:108930001D1F61E0F80187810E9463D6B6010C2EED
:1089400002C0759567950A94E2F76170F801878116
:108950000E949CD62196C430D10541F7C701DF9112
:10896000CF911F910F91FF90EF90DF90CF90B4CFF8
:10897000CF92DF92EF92FF920F931F93CF93DF93EB
:108980007C01C0E0D0E0C62ED12C87010C0F1D1F4A
:1089900061E0F80187810E9463D6B6010C2E02C007
:1089A000759567950A94E2F76170F80187810E94D6
:1089B0009CD62196C830D10541F7C701DF91CF91F0
:1089C0001F910F91FF90EF90DF90CF9085CF1F9375
:1089D000CF93DF93EC01162F642F8C810E949CD6DD
:1089E0008D818F3F19F060E00E949CD68F85612FAA
:1089F00084FF05C0CE01DF91CF911F91B9CF70E008
:108A000084E0759567958A95E1F7CE0182DF612F45
:108A1000CE01DF91CF911F917CCF40E0D8CF61E0B4
:108A2000FCDF80E496E00C9496D762E0F6DF80E409
:108A300096E00C9496D7CF93DF93CDB7DEB7289707
:108A40000FB6F894DEBF0FBECDBF28E0EFE5FBE028
:108A5000DE01119601900D922A95E1F7FC01238920
:108A6000421710F04FEF420FFE013196E40FF11D57
:108A7000E40FF11D2081260F2068622F28960FB683
:108A8000F894DEBF0FBECDBFDF91CF91C6CFFC0102
:108A90006089262F2460208B6C60BFCFCF93DF933B
:108AA000EC01423018F08F8588608F874B8B1C8AD1
:108AB000222329F0413019F48F8584608F8780E567
:108AC00093EC0E9496D760E08C810E949CD660E077
:108AD0008E810E949CD68D818F3F19F060E00E94AC
:108AE0009CD66F8564FD19C063E0CE0112DF84E976
:108AF00091E10E9496D763E0CE010BDF84E991E11A
:108B00000E9496D763E0CE0104DF86E990E00E94E0
:108B100096D762E0CE01FDDE13C06062CE017DDF3C
:108B200084E991E10E9496D76F856062CE0175DF7E
:108B300086E990E00E9496D76F856062CE016DDF76
:108B40006F856062CE0169DF8CE390E00E9496D76A
:108B500084E0888BCE019BDF8CE390E00E9496D767
:108B6000CE015DDF88EB9BE00E9496D782E0898B87
:108B700066E0CE0152DF8CE390E0DF91CF910C9460
:108B800096D76F927F928F92AF92CF92EF920F9380
:108B90001F93CF93DF93CDB7DEB73C01162F842F01
:108BA0005E854F8538899989F301848325830683FF
:108BB000E782C086A1868286538744873587968759
:108BC00061E00E9463D6F30185818F3F19F061E077
:108BD0000E9463D661E0F30186810E9463D611236F
:108BE00019F0F301178603C080E1F301878720E0C5
:108BF00041E060E1C301DF91CF911F910F91EF90B0
:108C0000CF90AF908F907F906F9048CF8F92AF9220
:108C1000CF92EF920F93DC0113961C921E92129743
:108C2000E5E2FCE0ED93FC931F921F921F921F92CE
:108C30008C2CAE2CC02EE22E042F2FEF462F61E09D
:108C4000A0DF0F900F900F900F900F91EF90CF90AB
:108C5000AF908F900895CF93DF93EC01423018F0DE
:108C60008F8588608F874B8B1C8A222329F04130A7
:108C700019F48F8584608F8780E593EC0E9496D7E6
:108C800060E08C810E949CD660E08E810E949CD620
:108C90008D818F3F19F060E00E949CD66F8564FD46
:108CA00019C063E0CE0135DE84E991E10E9496D7D8
:108CB00063E0CE012EDE84E991E10E9496D763E065
:108CC000CE0127DE86E990E00E9496D762E0CE01D1
:108CD00020DE13C06062CE01A0DE84E991E10E9433
:108CE00096D76F856062CE0198DE86E990E00E949B
:108CF00096D76F856062CE0190DE6F856062CE018F
:108D00008CDE8CE390E00E9496D784E0888BCE01C5
:108D1000BEDE8CE390E00E9496D7CE0186DE80E432
:108D200096E00E9496D782E0898B66E0CE0175DEE0
:108D30008CE390E00E9496D740E068E0CE017BDEB5
:108D400062E07DE0CE010E94D0DB41E068E0CE0130
:108D500072DE62E07DE0CE010E94D0DB42E066E0A0
:108D6000CE0169DE60E07DE0CE01DF91CF910C9411
:108D7000D0DBCF92DF92EF92FF920F931F93CF93AE
:108D8000DF931F921F92CDB7DEB78C01677088E02A
:108D9000689FB00111246064C80149835A833DDE95
:108DA0004981C42E5A81D52EE12CF12CD6016D912A
:108DB0006D01D801ED91FC910190F081E02DC80189
:108DC0001995BFEFEB1AFB0AE8E0EE16F10471F714
:108DD0000F900F90DF91CF911F910F91FF90EF9027
:108DE000DF90CF90089541E0F2DD81E090E00895BA
:108DF0000F931F93CF93DF93EC018B0144E150E07D
:108E0000BC0180EA9FE00E94DAE3CE010E94B9E350
:108E1000992744E150E0481B590BB8018056904F08
:108E20000E94DAE380EA9FE0DF91CF911F910F91DA
:108E30000895AF92BF92CF92DF92EF92FF920F937D
:108E40001F93CF93DF93EC015B017A01690144E149
:108E500050E0BC0180EA9FE00E94DAE3CE010E946C
:108E6000B9E3EC01DD2704E110E0A8014C1B5D0B28
:108E7000B501CE018056904F0E94DAE3C5010E94F1
:108E8000B9E3C80FD91FDD27A8014C1B5D0BB70143
:108E9000CE018056904F0E94DAE3C7010E94B9E3E9
:108EA0008C0F9D1F9927A801481B590BB6018056AE
:108EB000904F0E94DAE380EA9FE0DF91CF911F910B
:108EC0000F91FF90EF90DF90CF90BF90AF900895FB
:108ED0002F923F924F925F926F927F928F929F92CA
:108EE000AF92BF92CF92DF92EF92FF920F931F93B8
:108EF000CF93DF93CDB7DEB7CF54D1090FB6F89437
:108F0000DEBF0FBECDBF1C017E8F6D8F4A012FAB20
:108F100009AF2896EFAE28972C96ACAEBDAECEAE7C
:108F2000DFAE2C9734E0239F50011124FC01EA0DA1
:108F3000FB1D80819181A281B381898F9A8FAB8F34
:108F4000BC8FDA01AA0DBB1DBCAFABAF4D905D90DD
:108F50006D907C90A3019201698D7A8D8B8D9C8D93
:108F60000E94D9DB21966CAF7DAF8EAF9FAF21976A
:108F7000B4E00B9F80011124F101E00FF11F20816B
:108F80003181428153812F8F38A349A35AA3A40171
:108F9000400F511F23965FAF4EAF2397DA01CD905C
:108FA000DD90ED90FC90A70196016F8D78A189A1CD
:108FB0009AA10E94D9DB27966CAF7DAF8EAF9FAF91
:108FC00027972896EFAD2897B4E0EB9FC0011124B6
:108FD000F101E80FF91F20813181428153812BA3D8
:108FE0003CA34DA35EA3ED8DFE8DE80FF91F6081BC
:108FF0007181828193810E94D8DB6FA378A789A7B2
:109000009AA7AD8DBE8D1C968D919D910D90BC91B2
:10901000A02D60968CAF9DAFAEAFBFAF6097D10172
:109020001C962D913D914D915C911F972BA73CA7CC
:109030004DA75EA7A301920150582D8B3E8B4F8BFD
:10904000588FD701C601B058898B9A8BAB8BBC8BDC
:10905000ED8DFE8DEA0DFB1D208131814281538112
:109060002FA738AB49AB5AAB21962CAD3DAD4EADD9
:109070005FAD21976FA578A989A99AA90E94D8DB2D
:109080006B017C01ED8DFE8DE00FF11F80819181E0
:10909000A281B3818BAB9CABADABBEAB27962CADA5
:1090A0003DAD4EAD5FAD2797BC01CD010E94D8DB31
:1090B0004B015C01A70196016D897E898F89988D8E
:1090C0000E9487DF2B013C01A501940169897A89FF
:1090D0008B899C890E9487DF9B01AC01C301B2018F
:1090E0000E94D9DB2B013C01A50194016D897E8989
:1090F0008F89988D0E9487DF4B015C01A701960143
:1091000069897A898B899C890E9487DF9B01AC01E0
:10911000C501B4010E94D8DBA30192010E944CDC7E
:109120006B017C0120E030E0A9010E94B2DC87FFE6
:109130000AC02BED3FE049EC50E4C701B6010E94A4
:10914000D9DB6B017C01AA968FADAA97882351F0D9
:109150002BED3FE049EC50E4C701B6010E94D8DB9B
:109160006B017C012FA538A949A95AA9698D7A8D6F
:109170008B8D9C8D0E94B2DC81111FC02BA93CA954
:109180004DA95EA96F8D78A189A19AA10E94B2DC38
:10919000811113C020E030E0A901C701B6010E948F
:1091A000B2DC81110AC02BED3FE049EC50E4C7016D
:1091B000B6010E94D9DB6B017C01A9962CAD3DADB7
:1091C0004EAD5FADA997C701B6010E9487DF2FA101
:1091D00038A549A55AA55F770E94C2DE4B015C0104
:1091E0002FE632E143E85AE30E94B2DC87FDC8C1B2
:1091F000C501B4010E948FDD0E9426DD7A8F698F40
:10920000DB01AB2B21F4E1E0F0E0FA8FE98F298D4F
:109210003A8DB90180E090E00E9452DD4B015C0183
:109220009B01AC01C701B6010E94B9DC2B013C01D6
:10923000A50194016FA178A589A59AA50E94B9DC22
:109240006FA778AB89AB9AAB2BA53CA54DA55EA5C6
:1092500060966CAD7DAD8EAD9FAD60970E94D8DB02
:10926000A50194010E94B9DC6BAB7CAB8DAB9EABCE
:1092700020E030E040E05FE3C301B2010E9487DFFD
:10928000A30192010E9487DF9B01AC0160E070E0C6
:1092900080E89FE30E94D8DB6FA378A789A79AA7ED
:1092A000CE010196FC0128964FAD289734E0439FEC
:1092B000E00DF11D11242BA13CA14DA15EA1208345
:1092C0003183428353832BA53CA54DA55EA52D87F5
:1092D0003E874F87588BB12C41E050E058A34F8F09
:1092E0001C01BFA9A4E0BA9F800D911D112498AF65
:1092F0008FAB910159AD44E0549F200D311D1124D5
:109300003AAF29AFFCA7EBA74F8D58A1898D9A8D55
:109310004817590708F01AC188E18B150CF444C0AE
:109320002FA138A549A55AA569897A898B899C8975
:109330000E9487DF6B017C01A30192016D897E8908
:109340008F89988D0E9487DFA70196010E94D9DB43
:10935000A62E172F982E892E2FA138A549A55AA5DC
:109360006D897E898F89988D0E9487DF6B017C01D2
:10937000A301920169897A898B899C890E9487DF80
:109380009B01AC01C701B6010E94D8DB6D8B7E8BBF
:109390008F8B988FB3948A2D912FA92DB82D898BFF
:1093A0009A8BAB8BBC8B6CC0AF8DB8A1BD0180E03C
:1093B00090E00E9452DDA30192010E9487DF6B01C1
:1093C0007C010E94B6DC698B7A8B8B8B9C8BC701EE
:1093D000B6010E94EADF4B015C01EBADFCADC08041
:1093E000D180E280F380F7FAF094F7F8F0942396B6
:1093F000AEADBFAD23972D913D914D915C912BA3C7
:109400003CA34DA35EA329893A894B895C89C70196
:10941000B6010E9487DF6D8B7E8B8F8B988FA501A5
:1094200094016BA17CA18DA19EA10E9487DF9B016D
:10943000AC016D897E898F89988D0E94D9DB6D8BF7
:109440007E8B8F8B988FA5019401C701B6010E9476
:1094500087DF6B017C0129893A894B895C896BA183
:109460007CA18DA19EA10E9487DF9B01AC01C70159
:10947000B6010E94D8DB698B7A8B8B8B9C8BB12CCD
:109480002D893E894F89588D21966CAD7DAD8EAD6D
:109490009FAD21970E94D9DBEFA9F8AD608371835E
:1094A0008283938329893A894B895C8927966CAD9D
:1094B0007DAD8EAD9FAD27970E94D9DBA9ADBAAD2A
:1094C0006D937D938D939C9313972FA538A949A9EC
:1094D0005AA9EBA5FCA560817181828193810E94CC
:1094E000D9DBABA5BCA56D937D938D939C9313970E
:1094F0002BA93CA94DA95EA96D857E858F8598898C
:109500000E94D9DB6D877E878F87988BC1010E946F
:10951000A060FE01E659FF4F6F012C96ECACFDAC4C
:109520000EAD1FAD2C979E01235F3F4FAE01475FED
:109530005F4FBE016B5F7F4FC1010E946EC82F8DD0
:1095400038A12F5F3F4F38A32F8FDECE2D8D3E8D5C
:10955000245F3F4F4D8D5E8D485F5F4F6D8D7E8DDB
:109560006C5F7F4FDE01A659BF4F6D012C96ECACAE
:10957000FDAC0EAD1FAD2C978D8D9E8D0E946EC8DB
:10958000C15BDF4F0FB6F894DEBF0FBECDBFDF91DA
:10959000CF911F910F91FF90EF90DF90CF90BF90F0
:1095A000AF909F908F907F906F905F904F903F9083
:1095B0002F900895FC01148217821382128283E295
:1095C0009DE091838083089523E23DE0FC01318397
:1095D00020832781222319F004960C9429300895C2
:1095E000CF92DF92EF92FF920F931F93CF93DF936F
:1095F000EC01875B9F4FDEDFCE0186599F4FDADF9C
:109600007E0129E8E20EF11C87016E0131E4C31AE4
:109610003EEFD30AC801CEDF015E1F4F0C151D05BA
:10962000C9F7FE01EF53FE4F89E18183148235961D
:10963000178ACE018C519E4FBDDFFE01EB56FD4FC8
:109640001082118212821382389610821182128245
:1096500013821A821B82188219826E0187E6C81A49
:109660008DEFD80AF6011082118212821382F8015E
:1096700011821082FE01ED5FFD4F108286E391E0C2
:10968000F7019C01119221503040E1F7FE01EF55A6
:10969000FD4F81E08083C95BDF4F198218820E94F1
:1096A00043D768577C4E8F4F9F4FF601608371837D
:1096B00082839383DF91CF911F910F91FF90EF9061
:1096C000DF90CF900895FC0120E03EE2DB014C9159
:1096D000403241F0283011F430833196DB014C9157
:1096E000408331962F5F6F5F7F4F2B3079F7108269
:1096F00008952F923F924F925F926F927F928F9236
:109700009F92AF92BF92CF92DF92EF92FF920F9310
:109710001F93CF93DF93CDB7DEB7CA58D1090FB6E9
:10972000F894DEBF0FBECDBF8C016B017A014901F9
:10973000CA57DF4F1882C658D04084E0E80EF11CAB
:10974000180191E1290E311CF801EA5BFF4FC9575E
:10975000DF4FF983E883C758D0403801FEE56F1A20
:10976000FDEF7F0A58018CE5A81A8DEFB80A90E446
:10977000492E512C4C0E5D1E94E0490E511CA10146
:10978000BE016F5F7F4FC7010E94932E18160CF029
:109790004AC12C85322F3871303109F0ACC0F30149
:1097A000808191810197029708F4A5C0BE016F5F87
:1097B0007F4FCE0187589F4F86DFA0961FAEA097A0
:1097C000F6018081811107C069E27CE0CE01815AF7
:1097D0009F4F0E9433E4B601CE01815A9F4F0E94F1
:1097E00033E4BE0167587F4FCE01815A9F4F0E94DC
:1097F00033E469E27CE0CE01815A9F4F0E9433E45A
:10980000CE01805C9F4FD6DE21E0AE0147585F4F0E
:10981000B701C2010E942032811147C0F30180814B
:109820009181892B09F041C0EBE9F9E48491882307
:1098300041F09091C00095FFFCCF8093C600319617
:10984000F5CFE091C011F0E0EE0FFF1FE45EFD4F99
:109850000190F081E02DEA57FE4F0190F081E02D5C
:109860008191882339F09091C00095FFFCCF8093BF
:10987000C600F6CF8091C00085FFFCCF8AE08093C0
:10988000C600FE01E758FF4F8191882339F090917F
:10989000C00095FFFCCF8093C600F6CF8091C0003A
:1098A00085FFFCCF8AE08093C6008BE1FE01EC5B74
:1098B000FF4FDE01959601900D928A95E1F724966F
:1098C0008EAD9FAD24979CA38BA383E29DE09AA3CA
:1098D00089A320E030E0AE014F5D5F4FBE01615AC9
:1098E0007F4FC80106DFCE0181966EDECE01805C1F
:1098F0009F4F6ADE44CF8981882309F494C08E3259
:1099000009F43DCF8F3509F43ACFF80181898E32C1
:1099100009F435CF8F3509F432CF23FD30CF81E004
:10992000303109F080E0C957DF4FE881F981C7582D
:10993000D0408083811108C08985873409F01FCF0A
:109940008A858E3709F41BCF98012C5F3F4FBE01EB
:109950006F5F7F4FC901C757DF4F2883C958D04079
:10996000C657DF4F3883CA58D040ADDEF30180813F
:109970009181C757DF4F2881C958D040C657DF4F64
:109980003881CA58D0400097F1F4F60181918823BC
:1099900039F09091C00095FFFCCF8093C600F6CFC0
:1099A000F9018191882339F09091C00095FFFCCF97
:1099B0008093C600F6CF8091C00085FFFCCF8AE07F
:1099C0008093C600DCCE8130910539F4F5018081A9
:1099D0009181019691838083D2CE029709F0CFCEF8
:1099E0008114910439F0B901C4010E9420E4892B4B
:1099F00071F419C0CA57DF4FF881C658D0402F2FD5
:109A000030E0F501808191812817390761F0CA574C
:109A1000DF4FF881C658D040FF5FCA57DF4FF88349
:109A2000C658D040ACCEC657DF4F0FB6F894DEBF55
:109A30000FBECDBFDF91CF911F910F91FF90EF909F
:109A4000DF90CF90BF90AF909F908F907F906F905E
:109A50005F904F903F902F9008950F931F93CF9357
:109A6000DF93CDB7DEB76F970FB6F894DEBF0FBEAA
:109A7000CDBF8C01FC01EE55FD4F1182108240E0FC
:109A800050E0BA01835B9F4F0E94462FC801875B5D
:109A90009F4F2BE1FC013496DE01159601900D924B
:109AA0002A95E1F7FC01828193819C838B8383E279
:109AB0009DE09A83898320E030E0AE014F5F5F4FE5
:109AC00068E07DE0C80115DECE0101967DDD6F9670
:109AD0000FB6F894DEBF0FBECDBFDF91CF911F91BF
:109AE0000F9108952BE1FB013496DC01149601904F
:109AF0000D922A95E1F7FB0122813381FC0133832A
:109B000022830895EF92FF920F931F93CF93DF93D9
:109B1000EC011B82FC01E05BFF4F8081882329F070
:109B2000CE01835B9F4F0E9429307E018FE3E81AAC
:109B30008EEFF80A45E360E0C7010E943E598111AB
:109B40002CC0EBE9F9E48491882341F09091C000A6
:109B500095FFFCCF8093C6003196F5CFE091C01100
:109B6000F0E0EE0FFF1FE45EFD4F0190F081E02D6D
:109B7000E857FE4F0190F081E02D8491882341F059
:109B80009091C00095FFFCCF8093C6003196F5CF31
:109B90008091C00085FFFCCF9EC08E010A531E4FEE
:109BA00041E0B701C8010E94F737811133C040E09E
:109BB000B701C8010E94F73781112CC0E1EAF9E42E
:109BC0008491882341F09091C00095FFFCCF809351
:109BD000C6003196F5CFE091C011F0E0EE0FFF1F07
:109BE000E45EFD4F0190F081E02DE657FE4F0190BD
:109BF000F081E02D8491882341F09091C00095FF81
:109C0000FCCF8093C6003196F5CF8091C00085FFD0
:109C1000FCCF61C0B801CE01835B9F4F0E94362DFF
:109C200081112CC0E1EAF9E48491882341F09091FC
:109C3000C00095FFFCCF8093C6003196F5CFE09130
:109C4000C011F0E0EE0FFF1FE45EFD4F0190F081C8
:109C5000E02DE457FE4F0190F081E02D84918823A0
:109C600041F09091C00095FFFCCF8093C6003196E3
:109C7000F5CF8091C00085FFFCCF2DC081E08B83A4
:109C8000EBE9F9E48491882341F09091C00095FFBD
:109C9000FCCF8093C6003196F5CFE091C011F0E083
:109CA000EE0FFF1FE45EFD4F0190F081E02DE257C3
:109CB000FE4F0190F081E02D8491882341F0909136
:109CC000C00095FFFCCF8093C6003196F5CF809100
:109CD000C00085FFFCCF8AE08093C6008E01075B41
:109CE0001F4FB801CE0186599F4FFCDEC859DF4F88
:109CF00019830883DF91CF911F910F91FF90EF900F
:109D00000895FC01128213820895FC01238122230D
:109D100011F021E022830895FC0122812111128299
:109D20000895AF92BF92CF92DF92EF92FF920F937E
:109D30001F93CF93DF931F92CDB7DEB78C018FE2D5
:109D4000FB0181935F01D12C41E07801F1E4EF1A2E
:109D5000FEEFFF0A6FE1C62E2D2D30E0F701808166
:109D6000918128173907D8F4C29EC001C39E900D77
:109D7000112483579F4FB501800F911F49830E9483
:109D8000DD2CC50149815C010196F501208122236A
:109D900021F04D3810F44F5FF6CFD394DDCF47FD5F
:109DA00011C0B501C80188519E4F0F90DF91CF912E
:109DB0001F910F91FF90EF90DF90CF90BF90AF90E9
:109DC0000C94DD2CF50110820F90DF91CF911F9143
:109DD0000F91FF90EF90DF90CF90BF90AF900895DC
:109DE0003F924F925F926F927F928F929F92AF922B
:109DF000BF92CF92DF92EF92FF920F931F93CF9378
:109E0000DF93CDB7DEB7AC970FB6F894DEBF0FBEC9
:109E1000CDBF7C015B01FC018381882309F408C16B
:109E2000C70188519E4F0E942930F7011282CE014E
:109E300001966C01BFDB270198E6490E511CC70152
:109E4000875B9F4FF20191838083F50180818F3280
:109E500009F084C06FE270E0C5010E943EE48C010D
:109E60000F5F1F4F7AE0372E0115110509F47CC0F2
:109E70006FE270E0C8010E943EE44C01009709F4D3
:109E800074C00817190708F070C03C01601A710A05
:109E9000A301B801CE0180960E9467E4E0E2F0E001
:109EA000EC0FFD1FE60DF71D1082FE01B0968191AB
:109EB000882339F09091C00095FFFCCF8093C600B5
:109EC000F6CF8091C00085FFFCCF3092C600F20132
:109ED000608171816115710519F06C5F7F4F02C05F
:109EE00060E070E021E0AE01405E5F4FCE0105967C
:109EF0000E94203281112BC0EBE2FCE08491882388
:109F000041F09091C00095FFFCCF8093C600319640
:109F1000F5CFFE01B0968191882339F09091C00071
:109F200095FFFCCF8093C600F6CFE8EDF5E4849171
:109F3000882341F09091C00095FFFCCF8093C6002C
:109F40003196F5CF8091C00085FFFCCF6CC0F20147
:109F5000D182C08284010F5F1F4F86CFC70186590F
:109F60009F4FF201918380838501F201808191816D
:109F7000009711F0049602C080E090E0B8010E94C2
:109F8000F632882339F1EAECF5E48491882341F034
:109F90009091C00095FFFCCF8093C6003196F5CF1D
:109FA000F8018191882339F09091C00095FFFCCF92
:109FB0008093C600F6CF8091C00085FFFCCF8AE079
:109FC0008093C600F701E356FD4F10821182128282
:109FD00013822CC0E2EBF5E48491882341F0909148
:109FE000C00095FFFCCF8093C6003196F5CFF801F5
:109FF0008191882339F09091C00095FFFCCF809328
:10A00000C600F6CFE0EBF5E48491882341F090910F
:10A01000C00095FFFCCF8093C6003196F5CF8091AC
:10A02000C00085FFFCCF8AE08093C600C601CCDA71
:10A03000AC960FB6F894DEBF0FBECDBFDF91CF91C7
:10A040001F910F91FF90EF90DF90CF90BF90AF9056
:10A050009F908F907F906F905F904F903F9008956A
:10A060008F929F92AF92BF92CF92DF92EF92FF9228
:10A07000CF93DF931F92CDB7DEB77C01FC018281C5
:10A08000882309F4BCC071968191882339F090919E
:10A09000C00095FFFCCF8093C600F6CFEEEAF5E452
:10A0A0008491882341F09091C00095FFFCCF80936C
:10A0B000C6003196F5CFE091C011F0E0EE0FFF1F22
:10A0C000E45EFD4F0190F081E02DE456FE4F0190DB
:10A0D000F081E02D8491882341F09091C00095FF9C
:10A0E000FCCF8093C6003196F5CFF701E356FD4FC4
:10A0F00040815181628173812AE030E08BE295E1F9
:10A100000E94B3B7ECEAF5E48491882341F0909182
:10A11000C00095FFFCCF8093C6003196F5CFF701C4
:10A12000EB56FD4F40815181628173812AE030E01E
:10A130008BE295E10E94B3B78091C00085FFFCCF10
:10A140008AE08093C6000E9443D7E0E6CE2EEAEE76
:10A15000DE2EE12CF12CA70196010E9490E049012E
:10A160005A016091BD0F7091BE0F8091BF0F909109
:10A17000C00FA70196010E9490E0821A930AC401C1
:10A180006CE370E00E9469E06983CE0101960E9451
:10A190004899FC012191CF01222339F03091C00070
:10A1A00035FFFCCF2093C600F4CF40E050E06AE3D7
:10A1B0008BE295E10E946BB7C4016CE370E00E94F2
:10A1C00069E08983CE0101960E944899FC012191A2
:10A1D000CF01222339F03091C00035FFFCCF20930E
:10A1E000C600F4CFEAEAF5E484918823E1F0909187
:10A1F000C00095FFFCCF8093C6003196F5CFEFE30A
:10A20000FCE08491882341F09091C00095FFFCCF41
:10A210008093C6003196F5CF8091C00085FFFCCFBA
:10A220008AE08093C6000F90DF91CF91FF90EF906E
:10A23000DF90CF90BF90AF909F908F900895AF9296
:10A24000BF92CF92DF92EF92FF920F931F93CF9323
:10A25000DF935C01EB01FB0101900020E9F78F0126
:10A2600001501109061B170B6C01F8E1CF1AFEEF24
:10A27000DF0AF60110826EE470E0CE010E943EE437
:10A280007C01009729F4F8013197EC0FFD1F0DC0F8
:10A2900060E270E00E943EE4EC0121966AE270E028
:10A2A000C7010E943EE4FC0131978DE081838AE082
:10A2B00082831382BE01C5018C519E4F0E9470B8EB
:10A2C000F6018081882371F1E1EAF9E48491882321
:10A2D00041F09091C00095FFFCCF8093C60031966D
:10A2E000F5CFE091C011F0E0EE0FFF1FE45EFD4FEF
:10A2F0000190F081E02DE056FE4F0190F081E02DBD
:10A300008491882341F09091C00095FFFCCF809309
:10A31000C6003196F5CF8091C00085FFFCCF8AE062
:10A320008093C600DF91CF911F910F91FF90EF9026
:10A33000DF90CF90BF90AF9008952F923F924F92B1
:10A340005F926F927F928F929F92AF92BF92CF92C5
:10A35000DF92EF92FF920F931F93CF93DF93CDB7CE
:10A36000DEB7CC55D1090FB6F894DEBF0FBECDBF16
:10A370004C018C010F551D4F662339F0F8011082F6
:10A38000F401838181111DC015C0F80180818823EB
:10A3900009F4AFC0F401E756FD4FC080D180E280E0
:10A3A000F3800E9443D7C616D706E806F90608F4DC
:10A3B000A0C0E4CFC401A6DBF4018381882309F4A3
:10A3C00098C07401F7E4EF0EF11CF70181818F93BF
:10A3D00080818F9381EA95E49F938F938E01015C36
:10A3E0001F4F1F930F930E9476E40F900F900F90D2
:10A3F0000F900F900F90B12CF80101900020E9F719
:10A400003197E01BF10BBE1684F46801CB0CD11C14
:10A41000B7FCDA94F6018081992787FD90950E9418
:10A42000AAE3F6018083B394E7CFFDE48F0E911C7D
:10A4300040E050E0BA01C4010E94462F512CCE01E9
:10A4400001966C018AE9682E85E4782E5E0191E21E
:10A45000A90EB11C40E050E0B601C4010E94932E49
:10A460001816DCF5412CF60101900020E9F7319730
:10A47000EC19FD094E1674F41601240C311C47FC2E
:10A480003A94F101808190E00E94AAE3F101808377
:10A490004394E9CF8A858E37E9F245E050E0B80170
:10A4A000C6010E9459E4892BA9F61F930F937F924E
:10A4B0006F92BF92AF920E9476E4C5010E943F5C0A
:10A4C00086E995E40E94BF5C0F900F900F900F906B
:10A4D0000F900F9055245394BDCF511004C08FEFAF
:10A4E0009FEFF70104C0F70180819181019691836C
:10A4F0008083C45ADF4F0FB6F894DEBF0FBECDBFC6
:10A50000DF91CF911F910F91FF90EF90DF90CF904F
:10A51000BF90AF909F908F907F906F905F904F9083
:10A520003F902F9008950F931F93CF93DF93EC01EB
:10A530008C0108511E4FC8010E94DF2FC8010E94E4
:10A54000293018821982DF91CF911F910F910895C0
:10A55000CF92DF92EF92FF920F931F93CF93DF93EF
:10A56000CDB7DEB76F970FB6F894DEBF0FBECDBF85
:10A570008C016A017C0188E6E80EF11CC80186594D
:10A580009F4FF70191838083E65CFD4F22E030E02E
:10A590003183208332967183608340E050E0BA01BA
:10A5A00004960E94462FF701808191812BE1FC01E6
:10A5B0003496DE01159601900D922A95E1F7FC0183
:10A5C000828193819C838B8383E29DE09A8389833C
:10A5D0009601AE014F5F5F4F68E07DE0C80189D80A
:10A5E000CE0101960E94E44A6F960FB6F894DEBF42
:10A5F0000FBECDBFDF91CF911F910F91FF90EF90D4
:10A60000DF90CF9008952F923F924F925F926F927A
:10A610007F928F929F92AF92BF92CF92DF92EF92F2
:10A62000FF920F931F93CF93DF93CDB7DEB7AC9715
:10A630000FB6F894DEBF0FBECDBF8C016B01342E78
:10A64000DC0113968C91882309F449C3F801E55184
:10A65000FE4F8081882309F4F5C02111C1C0780123
:10A66000BDEFEB1AFB0AF7018081882361F1E1EA73
:10A67000F9E48491882341F09091C00095FFFCCFCC
:10A680008093C6003196F5CFECE2F6E484918823FE
:10A6900041F09091C00095FFFCCF8093C6003196A9
:10A6A000F5CF4AE050E061E070E08BE295E10E9476
:10A6B00087B78091C00085FFFCCF8AE08093C600F9
:10A6C0000E9458640CC3EBE9F9E48491882341F0BB
:10A6D0009091C00095FFFCCF8093C6003196F5CFD6
:10A6E000E3E1F6E48491882341F09091C00095FF66
:10A6F000FCCF8093C6003196F5CFF6018191882377
:10A7000039F09091C00095FFFCCF8093C600F6CF42
:10A71000E8E0F6E48491882341F09091C00095FF31
:10A72000FCCF8093C6003196F5CFD7018C91FDE820
:10A73000BF2EB801B89E600D711D1124685F7D4F5A
:10A74000C801EFDAF7018081F801B89EE00DF11D34
:10A750001124E85FFD4F8191882339F09091C0006A
:10A7600095FFFCCF8093C600F6CFE2E0F6E484913B
:10A77000882341F09091C00095FFFCCF8093C600E4
:10A780003196F5CF5801F3E6AF1AFDEFBF0AD501B8
:10A790004D915D916D917C912AE030E08BE295E1E5
:10A7A0000E94B3B78091C00085FFFCCF8AE0809300
:10A7B000C600F7012081F80184E0289FE00DF11D1B
:10A7C0001124EC5FFD4FD5014D915D916D917C9110
:10A7D00040835183628373832F5FF70120832CC0F2
:10A7E000EBE9F9E48491882341F09091C00095FF52
:10A7F000FCCF8093C6003196F5CFE1EFF5E484916C
:10A80000882341F09091C00095FFFCCF8093C60053
:10A810003196F5CFF6018191882339F09091C000EF
:10A8200095FFFCCF8093C600F6CF8091C00085FFD6
:10A83000FCCF8AE08093C600C80188519E4F0E94D9
:10A84000293030C0F801ED5FFD4F1082EBE9F9E4EB
:10A850008491882341F09091C00095FFFCCF8093B4
:10A86000C6003196F5CFE0EEF5E48491882341F0FF
:10A870009091C00095FFFCCF8093C6003196F5CF34
:10A88000F6018191882339F09091C00095FFFCCFAB
:10A890008093C600F6CF8091C00085FFFCCF8AE090
:10A8A0008093C600D80112961C92FE0131965F017A
:10A8B000CF010E94DA4A2801F8E64F0E511CC80168
:10A8C000875B9F4FD2018D939C93F60180818F32DD
:10A8D00009F091C06FE270E0C6010E943EE401966B
:10A8E0007C01EAE02E2EE114F10409F48AC06FE243
:10A8F00070E0C7010E943EE44C01009709F482C059
:10A90000E816F90608F07EC03C016E187F08A30126
:10A91000B701CE0180960E9467E4E0E2F0E0EC0F20
:10A92000FD1FE60DF71D1082FE01B0968191882370
:10A9300039F09091C00095FFFCCF8093C600F6CF10
:10A940008091C00085FFFCCF2092C600D2016D919E
:10A950007C916115710519F06C5F7F4F02C060E05A
:10A9600070E021E0AE01405E5F4FCE0105960E948F
:10A970002032811138C0E091C011F0E0EE0FFF1FCE
:10A98000E45EFD4F0190F081E02DEE56FE4F019008
:10A99000F081E02D8491882341F09091C00095FFD3
:10A9A000FCCF8093C6003196F5CFFE01B096819121
:10A9B000882339F09091C00095FFFCCF8093C600AA
:10A9C000F6CFEEEDF5E48491882341F09091C0003C
:10A9D00095FFFCCF8093C6003196F5CF8091C000E3
:10A9E00085FFFCCF43C1F201B182A0827401FFEF69
:10A9F000EF1AFF0A78CFC80186599F4FD2018D9375
:10AA00009C937601F801E851FE4F4F01332009F481
:10AA1000E5C0D2016D917C916115710519F06C5FF3
:10AA20007F4F02C060E070E021E0A701C4010E94F6
:10AA300020322091C011882309F49AC0F401818941
:10AA40009289A389B489F801EB56FD4F80839183E5
:10AA5000A283B383E22FF0E0EE0FFF1FE45EFD4F11
:10AA60000190F081E02DEC56FE4F0190F081E02D39
:10AA70008491D801AB56BD4F882349F09091C00016
:10AA800095FFFCCF8093C60031968491F5CFF701F6
:10AA90008191882339F09091C00095FFFCCF80937D
:10AAA000C600F6CFE091C011F0E0EE0FFF1FE45EAC
:10AAB000FD4F0190F081E02DEA56FE4F0190F081AC
:10AAC000E02D8491882341F09091C00095FFFCCF48
:10AAD0008093C6003196F5CF4D915D916D917C913B
:10AAE0002AE030E08BE295E10E94B3B78091C0008C
:10AAF00085FFFCCF8AE08093C600F801E356FD4F46
:10AB00001082118212821382E091C011F0E0EE0FE8
:10AB1000FF1FE45EFD4F0190F081E02DE856FE4FEF
:10AB20000190F081E02D8491882341F09091C00044
:10AB300095FFFCCF8093C6003196F5CF8091C00081
:10AB400085FFFCCF8AE08093C600A70160E070E03B
:10AB5000C801FEDCD80151968C91882319F0C801F8
:10AB6000419601C0C7010E948E978CE49CE0B2C060
:10AB7000E22FF0E0EE0FFF1FE45EFD4F0190F08149
:10AB8000E02DEE56FE4F0190F081E02D8491882358
:10AB900041F09091C00095FFFCCF8093C6003196A4
:10ABA000F5CFF7018191882339F09091C00095FF8E
:10ABB000FCCF8093C600F6CFECEDF5E484918823BA
:10ABC00041F09091C00095FFFCCF8093C600319674
:10ABD000F5CF8091C00085FFFCCF48C0F2016081B5
:10ABE00071816115710519F06C5F7F4F02C060E0E3
:10ABF00070E026E5A701C4010E94203281113AC00D
:10AC0000E091C011F0E0EE0FFF1FE45EFD4F0190F8
:10AC1000F081E02DEE56FE4F0190F081E02D849101
:10AC2000882341F09091C00095FFFCCF8093C6002F
:10AC30003196F5CFF7018191882339F09091C000CA
:10AC400095FFFCCF8093C600F6CFEAEDF5E4849142
:10AC5000882341F09091C00095FFFCCF8093C600FF
:10AC60003196F5CF8091C00085FFFCCF8AE08093BC
:10AC7000C60032C081E0D8018C93E091C011F0E0B1
:10AC8000EE0FFF1FE45EFD4F0190F081E02DE656D0
:10AC9000FE4F0190F081E02D8491882341F0909146
:10ACA000C00095FFFCCF8093C6003196F5CFF6012A
:10ACB0008191882339F09091C00095FFFCCF80935B
:10ACC000C600F6CF8091C00085FFFCCF8AE080935C
:10ACD000C600C7010E948E97C5010E94E44AAC9647
:10ACE0000FB6F894DEBF0FBECDBFDF91CF911F919D
:10ACF0000F91FF90EF90DF90CF90BF90AF909F901B
:10AD00008F907F906F905F904F903F902F9008951D
:10AD100021E0FC01218340E076CCCF92DF92EF92DC
:10AD2000FF920F931F93CF93DF93CDB7DEB76F974B
:10AD30000FB6F894DEBF0FBECDBF8C016C0128E6C4
:10AD4000C20ED11C86599F4FF60191838083E65C29
:10AD5000FD4F21E030E0318320837801FCE5EF1ADC
:10AD6000FDEFFF0AF7011182108240E050E0BA01C6
:10AD700004960E94462FF601808191812BE1FC010F
:10AD80003496DE01159601900D922A95E1F7FC01AB
:10AD9000828193819C838B8383E29DE09A83898364
:10ADA00020E030E0AE014F5F5F4F68E07DE0C8011A
:10ADB0000E94794BCE0101960E94E44AF7018081FE
:10ADC00091816F960FB6F894DEBF0FBECDBFDF91B5
:10ADD000CF911F910F91FF90EF90DF90CF9008954A
:10ADE000AF92BF92CF92DF92EF92FF920F931F9399
:10ADF000CF93DF93CDB7DEB76F970FB6F894DEBF72
:10AE00000FBECDBF8C017B01CE0101960E94DA4AB4
:10AE1000F801EF58FF4F80816801811104C029E4D7
:10AE2000C20ED11C03C08AE6C80ED11C21E0A701C6
:10AE3000B6016C5F7F4FCE0105960E9420328111D2
:10AE40003AC0EBE9F9E48491882341F09091C00085
:10AE500095FFFCCF8093C6003196F5CFE091C011ED
:10AE6000F0E0EE0FFF1FE45EFD4F0190F081E02D5A
:10AE7000EE55FE4F0190F081E02D8491882341F042
:10AE80009091C00095FFFCCF8093C6003196F5CF1E
:10AE9000F7018191882339F09091C00095FFFCCF94
:10AEA0008093C600F6CF8091C00085FFFCCF8AE07A
:10AEB0008093C60036C0F801E154FE4F8081918135
:10AEC0008A30910530F59C012F5F3F4F31832083FD
:10AED0002FE1289F7001299FF00C112429E8E20E30
:10AEE000F11CE00EF11E5C01B701C7014F960E94F4
:10AEF000724D81E0A81AB1082FE1E21AF1088FEF34
:10AF0000A816B80689F7B601C80187579F4F0E9457
:10AF1000724DBE016F5F7F4FC80186599F4F0E94DF
:10AF2000724DCE0101960E94E44A6F960FB6F894D6
:10AF3000DEBF0FBECDBFDF91CF911F910F91FF906C
:10AF4000EF90DF90CF90BF90AF900895EF92FF9277
:10AF50000F931F93CF93DF93EC01C154DE4F2881F1
:10AF6000398121153105F9F02150310939832883C0
:10AF70008C0107571F4FB80186599F4F0E94724D91
:10AF8000C80100E010E07C012FE1E20EF11C2881F5
:10AF900039810217130738F40F5F1F4FB7010E9462
:10AFA000724DC701F0CFDF91CF911F910F91FF90AC
:10AFB000EF900895EF92FF920F931F93CF93DF933B
:10AFC000EC010E94DBC08E010D5F1D4FF8018081F6
:10AFD0009E0128513E4F79018823A1F1C9010E94A9
:10AFE0002930F801808181508083BE01FDE88F9F68
:10AFF000600D711D1124685F7D4F21E041E0CE019D
:10B0000002DBF8018081FE0124E0829FE00DF11D4A
:10B010001124EC5FFD4F4081518162817381FE01FB
:10B02000E356FD4F4083518362837383C7010E94BF
:10B03000462FCE01DF91CF911F910F91FF90EF909E
:10B040000C94854E0E9451C1C7010E9429301A827A
:10B050008AE895E4DF91CF911F910F91FF90EF90D7
:10B060008EC48FEF8EBD0DB407FEFDCF8EB5089553
:10B070008EBD0DB407FEFDCF089561E0FC01808117
:10B080000C949CD6FC012281322F306A36953CBD4F
:10B0900020FD06C031E0263009F430E0232F01C046
:10B0A00020E02DBD60E0FC0180810C949CD6CF9205
:10B0B000DF92EF92FF920F931F93CF93DF93EC01F8
:10B0C0008B017A010E9443D76B01CBDF8B838F3FCB
:10B0D00049F40E9443D76C197D096D327140A8F381
:10B0E00081E144C08E3F11F08FE040C0E114F104D3
:10B0F000D9F0C70101972FEF2EBDF8014FEF9F0147
:10B10000201B310B2817390738F40DB407FEFDCF8B
:10B110002EB521934EBDF3CF0DB407FEFDCF2EB556
:10B12000F801E80FF91F2083D801E00EF11EC12CB1
:10B13000D12CAE15BF0579F08D91ED2DFF27E827B5
:10B14000EE0FFF1FE159F94B85919491DC2CCC2433
:10B15000C826D926EECF85DF082F10E0102F002754
:10B1600080DF082BC016D10631F080E28983CE0142
:10B1700084DF80E003C0CE0180DF81E0DF91CF91EA
:10B180001F910F91FF90EF90DF90CF9008950F9354
:10B190001F93CF93DF93EB010E9443D78B0161DFB5
:10B1A0008F3F49F00E9443D7601B710B6C177D07DE
:10B1B000B0F380E001C081E0DF91CF911F910F914A
:10B1C0000895CF92DF92FF920F931F93CF93DF9357
:10B1D00000D01F92CDB7DEB76C01F62E29833A83DB
:10B1E0004B835C834FDF6CE271E0C601D0DF8F2DB3
:10B1F00080643EDF08E110E05C814B813A81298167
:10B20000DA01C901002E04C0B695A79597958795D8
:10B210000A94D2F729833A834B835C8329DF085051
:10B22000110929813A814B815C81083F8FEF180712
:10B2300039F7FF2029F0E8E0FE1621F08FEF03C078
:10B2400085E901C087E814DFFCE0FF1201C009DFD7
:10B2500010E007DFF601838387FF04C01F3F11F072
:10B260001F5FF7CF0F900F900F900F90DF91CF914E
:10B270001F910F91FF90DF90CF900895BF92CF92D2
:10B28000DF92EF92FF920F931F93CF93DF93EC0126
:10B29000B62E1C82198248830E9443D78B0161E03D
:10B2A00088810E9463D6CE01E8DE60E082E30E94DE
:10B2B00063D661E083E30E9463D661E084E30E9489
:10B2C00063D661E085E30E9463D661E085E30E9476
:10B2D0009CD685E08A8382E58CBD1DBC6AE0F62E93
:10B2E0008FEFC6DEFA94E1F720E030E0A90160E0DC
:10B2F000CE0167DFF82E8B8381E0F81649F00E94BB
:10B3000043D7601B710B613D774070F381E046C00D
:10B310002AEA31E040E050E068E0CE0152DF82FFEF
:10B3200002C0FC820CC054E0F52E9BDE8B83FA94A5
:10B33000E1F78A3A11F082E031C082E08C838C819F
:10B34000823031F4C12CD12CE12C40E4F42E03C026
:10B35000C12CD12C760120E030E0A90167E3CE01B9
:10B3600030DFA701960169E2CE012BDF8B838823B2
:10B3700049F00E9443D7601B710B613D774058F341
:10B380008AE00CC08C818230B1F420E030E0A90169
:10B390006AE3CE0116DF882329F088E08983CE0195
:10B3A0006CDE14C05EDE807C803C11F483E08C8314
:10B3B00058DE57DE56DECE0160DE86E08B1518F4CF
:10B3C00088E1898303C0BA8281E001C080E0DF9117
:10B3D000CF911F910F91FF90EF90DF90CF90BF9092
:10B3E0000895AF92BF92CF92DF92EF92FF920F93A8
:10B3F0001F93CF93DF93EC016A017B0189018C815C
:10B40000833039F0F9E0CC0CDD1CEE1CFF1CFA9502
:10B41000D1F773E0B72EE4E0AE2EBA94A7019601FF
:10B4200061E1CE01CEDE882311F0A98207C040E0A1
:10B4300052E0B801CE013BDE81110EC0CE01BB202F
:10B4400049F01BDE20E030E0A9016CE0CE01B9DE5E
:10B450001982E3CF12DE80E0DF91CF911F910F912F
:10B46000FF90EF90DF90CF90BF90AF900895CF9373
:10B47000DF93EC016EBD20E030E00DB407FEFDCFA0
:10B48000FA01E20FF31F80818EBD0DB407FEFDCFE0
:10B4900081818EBD2E5F3F4F211582E0380769F70D
:10B4A0000DB407FEFDCF8FEFE3DD8FEFE1DDD9DDDA
:10B4B0008B838F71853031F083E18983CE01DDDDAF
:10B4C00080E001C081E0DF91CF9108950F931F9339
:10B4D000CF93DF93EC0189018C81833039F0B9E09F
:10B4E000440F551F661F771FBA95D1F79A01AB011C
:10B4F00068E1CE0166DE882311F086E01EC0A80157
:10B500006EEFCE01B4DF8823C9F068E572E0CE01AA
:10B510003EDE182F811102C087E10FC020E030E02D
:10B52000A9016DE0CE014DDE811106C09ADD8111C9
:10B5300003C0CE01A2DD05C086E18983CE019DDD79
:10B5400010E0812FDF91CF911F910F910895FC01A1
:10B55000659175918591949108952F923F924F92A4
:10B560005F926F927F928F929F92AF92BF92CF9293
:10B57000DF92EF92FF920F931F93CF93DF9300D050
:10B5800000D0CDB7DEB71C01FC01E45AF64B149194
:10B590009C01220F331F220F331F3E832D83215521
:10B5A0003E4E4901F90110821182128213822BEB67
:10B5B00031E147EB51E163EB71E18FEA91E10E94E8
:10B5C00050D28D819E818559964BC1DF6B017C01E4
:10B5D000612F772767FD7095872F972F0E9454DD85
:10B5E0002B013C012D813E8126583E4E590120E021
:10B5F00030E040EC5FE3C701B6010E9487DFA301A2
:10B6000092010E9487DFF5016083718382839383B7
:10B610002D813E81215E344F3C832B83F901608173
:10B620007181828193816093E10A7093E20A809331
:10B63000E30A9093E40A20E030E040E752E40E94FD
:10B64000B9DC2BE9C22E21E1D22E7B018C0126E848
:10B6500031E142E851E16EE771E18AE791E10E9450
:10B660006EC80E94DBC0F401108211821282138224
:10B670002BEB31E147EB51E163EB71E18FEA91E1B3
:10B680000E9450D22D813E81215A364B3A83298324
:10B69000C9015DDF9058A30192010E9487DFF50187
:10B6A000608371838283938320E030E040E752E43B
:10B6B0006091E10A7091E20A8091E30A9091E40AB4
:10B6C0000E94B9DC7B018C0126E831E142E851E1BE
:10B6D0006EE771E18AE791E10E946EC80E94DBC0CB
:10B6E00089819A8134DF9B01AC010E94D9DBA301DF
:10B6F00092010E9487DFF5016083718382839383C7
:10B7000020E030E040E05FE3EB81FC81608171810B
:10B71000828193810E9487DF6093E10A7093E20A3D
:10B720008093E30A9093E40A20E030E040E752E49B
:10B730000E94B9DC7B018C0126E831E142E851E14D
:10B740006EE771E18AE791E10E946EC80E94DBC05A
:10B750008D819E818958964BFADE0D811E810D5593
:10B760001E4EF80120813181428153810E94D9DB34
:10B77000F40160837183828393838D819E818157DD
:10B78000964BE5DE2D813E812D5F344F7901F80126
:10B7900020813181428153810E94D9DBF70160838E
:10B7A0007183828393838D819E818D57964BCFDEEB
:10B7B0002D813E812950354F7901F8012081318159
:10B7C000428153810E94D9DBF701608371838283B8
:10B7D0009383F40180819181A281B381F5018083FB
:10B7E0009183A283B3831092E10A1092E20A10922D
:10B7F000E30A1092E40A0E9454B9F101E056FE4EA9
:10B8000081E0808326960FB6F894DEBF0FBECDBFD1
:10B81000DF91CF911F910F91FF90EF90DF90CF902C
:10B82000BF90AF909F908F907F906F905F904F9060
:10B830003F902F900895FC012491222341F03091F4
:10B84000C00035FFFCCF2093C6000196F4CF22E064
:10B8500030E08BE295E10C945DB8FC012491222349
:10B8600041F03091C00035FFFCCF2093C600019617
:10B87000F4CF2AE030E08BE295E10C94B3B720914D
:10B88000CF0F3091D00F243031050CF077C04091AC
:10B89000D10F5091D20F60E6649F9001659F300DEB
:10B8A0001124BC01C9018752904F0E9452E4EBE978
:10B8B000F9E48491882341F09091C00095FFFCCF7A
:10B8C0008093C6003196F5CFE091C011F0E0EE0F05
:10B8D000FF1FE45EFD4F0190F081E02DEA5DFE4F19
:10B8E0000190F081E02D8491882341F09091C00077
:10B8F00095FFFCCF8093C6003196F5CF8091D10F94
:10B900009091D20F20E6289FF001299FF00D11247D
:10B91000E752F04F8191882339F09091C00095FF54
:10B92000FCCF8093C600F6CFEAE5F9E48491882342
:10B9300041F09091C00095FFFCCF8093C6003196F6
:10B94000F5CF8091C00085FFFCCF8AE08093C600D0
:10B950008091D10F9091D20F019664E070E00E9427
:10B960007DE09093D20F8093D10F8091CF0F909173
:10B97000D00F01969093D00F8093CF0F0895209110
:10B98000CF0F3091D00F243031050CF077C04091AB
:10B99000D10F5091D20F60E6649F9001659F300DEA
:10B9A0001124BC01C9018752904F0E94B2E3EBE918
:10B9B000F9E48491882341F09091C00095FFFCCF79
:10B9C0008093C6003196F5CFE091C011F0E0EE0F04
:10B9D000FF1FE45EFD4F0190F081E02DEA5DFE4F18
:10B9E0000190F081E02D8491882341F09091C00076
:10B9F00095FFFCCF8093C6003196F5CF8091D10F93
:10BA00009091D20F20E6289FF001299FF00D11247C
:10BA1000E752F04F8191882339F09091C00095FF53
:10BA2000FCCF8093C600F6CFE8E5F9E48491882343
:10BA300041F09091C00095FFFCCF8093C6003196F5
:10BA4000F5CF8091C00085FFFCCF8AE08093C600CF
:10BA50008091D10F9091D20F019664E070E00E9426
:10BA60007DE09093D20F8093D10F8091CF0F909172
:10BA7000D00F01969093D00F8093CF0F08959B9A8B
:10BA8000A3980895FCDF40E052EC61E070E08BE2A7
:10BA900095E10E946BB6E2E5F9E48491882341F0D8
:10BAA0009091C00095FFFCCF8093C6003196F5CFF2
:10BAB0008091C00085FFFCCF8AE08093C6002BE90F
:10BAC00039E4F9018491882341F09091C00095FFF9
:10BAD000FCCF8093C6003196F5CF84B780FF20C09D
:10BAE000A091C011B0E0AA0FBB1FA45EBD4FED91A5
:10BAF000FC91E85DFE4F0190F081E02D9491992337
:10BB000041F04091C00045FFFCCF9093C6003196B4
:10BB1000F5CF9091C00095FFFCCF9AE09093C600BE
:10BB200081FF20C0A091C011B0E0AA0FBB1FA45E8E
:10BB3000BD4FED91FC91E65DFE4F0190F081E02D4F
:10BB40009491992341F04091C00045FFFCCF909320
:10BB5000C6003196F5CF9091C00095FFFCCF9AE0DA
:10BB60009093C60082FF20C0A091C011B0E0AA0F40
:10BB7000BB1FA45EBD4FED91FC91E45DFE4F0190B3
:10BB8000F081E02D9491992341F04091C00045FF50
:10BB9000FCCF9093C6003196F5CF9091C00095FFF1
:10BBA000FCCF9AE09093C60083FF20C0A091C01103
:10BBB000B0E0AA0FBB1FA45EBD4FED91FC91E25D0A
:10BBC000FE4F0190F081E02D9491992341F0409136
:10BBD000C00045FFFCCF9093C6003196F5CF909101
:10BBE000C00095FFFCCF9AE09093C60085FF20C06F
:10BBF000A091C011B0E0AA0FBB1FA45EBD4FED9194
:10BC0000FC91E05DFE4F0190F081E02D849188234E
:10BC100041F09091C00095FFFCCF8093C600319613
:10BC2000F5CF8091C00085FFFCCF8AE08093C600ED
:10BC300014BEE1E6FCE08491882341F09091C000BD
:10BC400095FFFCCF8093C6003196F5CFE8E6FCE087
:10BC50008491882341F09091C00095FFFCCF8093A0
:10BC6000C6003196F5CF8091C00085FFFCCF8AE0F9
:10BC70008093C600F9018491EBE9F9E4882349F047
:10BC80009091C00095FFFCCF8093C60031968491BF
:10BC9000F5CFA091C011B0E0AA0FBB1FA45EBD4FAD
:10BCA000ED91FC91EC5CFE4F0190F081E02D8491D0
:10BCB000882341F09091C00095FFFCCF8093C6008F
:10BCC0003196F5CFEDE3F9E48491882341F090912A
:10BCD000C00095FFFCCF8093C6003196F5CFA091B0
:10BCE000C011B0E0AA0FBB1FA45EBD4FED91FC9147
:10BCF000EE5CFE4F0190F081E02D4491442341F031
:10BD00005091C00055FFFCCF4093C6003196F5CF4F
:10BD1000E6E2F9E48491882341F09091C00095FF18
:10BD2000FCCF8093C6003196F5CF8091C00085FF8F
:10BD3000FCCF8AE08093C600EBE1F9E4849188238C
:10BD400041F09091C00095FFFCCF8093C6003196E2
:10BD5000F5CFEFE0F9E48491882341F09091C000A1
:10BD600095FFFCCF8093C6003196F5CF8091C0003F
:10BD700085FFFCCF8AE08093C600F9012491EBE9AE
:10BD8000F9E4222349F08091C00085FFFCCF209385
:10BD9000C60031962491F5CFE091C011F0E0EE0F8E
:10BDA000FF1FE45EFD4F0190F081E02DEA5CFE4F45
:10BDB0000190F081E02D8491882341F09091C000A2
:10BDC00095FFFCCF8093C6003196F5CF0E944FC4FB
:10BDD0004AE050E0BC018BE295E10E9487B7E09118
:10BDE000C011F0E0EE0FFF1FE45EFD4F0190F08107
:10BDF000E02DE85CFE4F0190F081E02D84918823D6
:10BE000041F09091C00095FFFCCF8093C600319621
:10BE1000F5CF4AE050E060ED74E08BE295E10E94DE
:10BE200087B78091C00085FFFCCF8AE08093C60071
:10BE30001092D50F1092D60F1092D70F1092D80FE4
:10BE40000E948EB40E9460B00E943F3D0E941EC8B6
:10BE50000E943DC30E942E98489913C0FFEF23ED26
:10BE600080E3F15020408040E1F700C00000489995
:10BE700011C06A9A729A0E946997489BFECF729885
:10BE800008959FEFE3EDF0E39150E040F040E1F7DB
:10BE900000C0000008958091C90F9091CA0F60E022
:10BEA00070E001960C9409E18091C90F9091CA0F3E
:10BEB0004AE050E060E070E001960C9471E2682F77
:10BEC000772767FD70952091D30F3091D40F40E60E
:10BED000429FC001439F900D11248752904F0E94B2
:10BEE0003EE49093CA0F8093C90F21E0892B09F497
:10BEF00020E0822F08950E9443D76093C50F70936E
:10BF0000C60F8093C70F9093C80F08950E9443D720
:10BF10006093C50F7093C60F8093C70F9093C80F9F
:10BF2000E091D30FF091D40FEB52F04F808181114B
:10BF300021C0E091C011F0E0EE0FFF1FE45EFD4F65
:10BF40000190F081E02DE65CFE4F0190F081E02D44
:10BF50008491882341F09091C00095FFFCCF80939D
:10BF6000C6003196F5CF8091C00085FFFCCF8AE0F6
:10BF70008093C60008958BE295E10E94BDB6E091E2
:10BF8000C011F0E0EE0FFF1FE45EFD4F0190F08165
:10BF9000E02DE659FE4F0190F081E02D8491882339
:10BFA00041F09091C00095FFFCCF8093C600319680
:10BFB000F5CF40915E1150915F11609160117091C9
:10BFC00061114F5F5F4F6F4F7F4F2AE030E08BE290
:10BFD00095E10E945CB78091C00085FFFCCF8AE0AC
:10BFE0008093C60093CF8F929F92AF92BF92CF92D1
:10BFF000DF92EF92FF920F931F93CF93DF93B8EEF0
:10C00000EB2EBCE0FB2E0FEA11E1CAE7D1E185EC93
:10C01000C82E81E1D82EF70181917F0150DF88235E
:10C0200011F139DF4B015C01F6018081811103C000
:10C030006091591101C061E070E080E090E00E94E1
:10C0400054DDF80120813181428153810E9487DFD4
:10C050009B01AC01C501B4010E94D9DB68837983DF
:10C060008A839B8309C0F80180819181A281B38179
:10C0700088839983AA83BB830C5F1F4F2496FFEFAD
:10C08000CF1ADF0A8CEEE8168CE0F80621F686E47B
:10C0900016DF8823D1F0FFDE6B017C0160936A110B
:10C0A00070936B1180936C1190936D1120E030E0D0
:10C0B000A9010E94B5DE181644F4C092E10AD0929C
:10C0C000E20AE092E30AF092E40ADF91CF911F9135
:10C0D0000F91FF90EF90DF90CF90BF90AF909F9027
:10C0E0008F90089580DF89E4EADE882351F0D3DE63
:10C0F00060936E1170936F11809370119093711112
:10C1000008C010926E1110926F111092701110925F
:10C1100071118AE4D4DE882351F0BDDE6093721180
:10C120007093731180937411909375110895109208
:10C13000721110927311109274111092751108956A
:10C14000CF92DF92EF92FF92CF93DF93EC01C090FA
:10C15000030BD090040BE090050BF090060BA701A9
:10C160009601688179818A819B810E94B2DC87FF78
:10C1700004C0C882D982EA82FB82C090070BD090AB
:10C18000080BE090090BF0900A0BA70196016C8157
:10C190007D818E819F810E94B2DC87FF04C0CC82AA
:10C1A000DD82EE82FF8220E030E0A90160910B0B7E
:10C1B00070910C0B80910D0B90910E0B0E94D9DBAE
:10C1C0006B017C019B01AC01688579858A859B8523
:10C1D0000E94B2DC87FF04C0C886D986EA86FB8647
:10C1E000C090F70AD090F80AE090F90AF090FA0AA5
:10C1F000A7019601688179818A819B810E94B5DEC1
:10C20000181624F4C882D982EA82FB82C090FB0A05
:10C21000D090FC0AE090FD0AF090FE0AA70196017A
:10C220006C817D818E819F810E94B5DE181624F479
:10C23000CC82DD82EE82FF82C090FF0AD090000B9C
:10C24000E090010BF090020BA701960168857985BB
:10C250008A859B850E94B5DE181624F4C886D98687
:10C26000EA86FB86DF91CF91FF90EF90DF90CF9031
:10C270000895CF92DF92EF92FF920F931F938AE778
:10C2800091E15EDF0E9443D76093C50F7093C60FA4
:10C290008093C70F9093C80F20917A1130917B1132
:10C2A00040917C1150917D116091AF117091B0114E
:10C2B0008091B1119091B2110E94B2DC811179C0CC
:10C2C00020917E1130917F11409180115091811108
:10C2D0006091B3117091B4118091B5119091B61124
:10C2E0000E94B2DC811165C020E030E040E752E4FA
:10C2F0006091E10A7091E20A8091E30A9091E40A68
:10C300000E94B9DC2BE9C22E21E1D22E7B018C01E7
:10C3100026E831E142E851E16EE771E18AE791E117
:10C320000E946EC880917A1190917B11A0917C112E
:10C33000B0917D118093AF119093B011A093B11182
:10C34000B093B21180917E1190917F11A0918011D4
:10C35000B09181118093B3119093B411A093B51152
:10C36000B093B6118091821190918311A0918411A4
:10C37000B09185118093B7119093B811A093B91122
:10C38000B093BA118091861190918711A091881174
:10C39000B09189118093BB119093BC11A093BD11F2
:10C3A000B093BE111F910F91FF90EF90DF90CF904F
:10C3B000089560911D0B70911E0B882777FD809565
:10C3C000982F0E9454DD2091E10A3091E20A4091B9
:10C3D000E30A5091E40A0E9487DF20E030E040E762
:10C3E00052E40E94B9DC20E030E048EC52E488CF0F
:10C3F000CF92DF92EF92FF92CF93C62FE0919B11E5
:10C40000F0E0882309F4C2C0DF01A956BE4E8C912A
:10C41000811196C18091AF119091B011A091B1118D
:10C42000B091B21180937A1190937B11A0937C11FB
:10C43000B0937D118091B3119091B411A091B51179
:10C44000B091B61180937E1190937F11A0938011CB
:10C45000B09381118091B7119091B811A091B91149
:10C46000B091BA118093821190938311A09384119B
:10C47000B0938511C090BB11D090BC11E090BD115C
:10C48000F090BE11C0928611D0928711E09288116F
:10C49000F0928911EE0FFF1FEE0FFF1FE15FF44FC7
:10C4A0002081318142815381662349F06091EF0AF6
:10C4B0007091F00A8091F10A9091F20A08C060919F
:10C4C000F30A7091F40A8091F50A9091F60A0E949D
:10C4D000B9DC9B01AC01C701B6010E94D9DB6093B6
:10C4E000BB117093BC118093BD119093BE118BEB67
:10C4F00091E10E94F5D2C090E10AD090E20AE0906A
:10C50000E30AF090E40A20E030E040E752E4609172
:10C51000EB0A7091EC0A8091ED0A9091EE0A0E946C
:10C5200087DF6093E10A7093E20A8093E30A9093B5
:10C53000E40AE0919B11F0E0E956FE4E81E0808331
:10C5400098DE209193113091941140919511509162
:10C5500096116091B7117091B8118091B9119091B5
:10C56000BA110E94D8DB6093B7117093B811809311
:10C57000B9119093BA112BEB31E147EB51E163EB29
:10C5800071E18FEA91E10E9450D2D1C0E956FE4E8E
:10C590008081882309F4D4C08091AF119091B011AB
:10C5A000A091B111B091B21180937A1190937B1147
:10C5B000A0937C11B0937D118091B3119091B4112F
:10C5C000A091B511B091B61180937E1190937F1117
:10C5D000A0938011B09381116091B7117091B8113F
:10C5E0008091B9119091BA11609382117093831167
:10C5F0008093841190938511C090BB11D090BC1191
:10C60000E090BD11F090BE11C0928611D0928711BA
:10C61000E0928811F0928911209193113091941138
:10C6200040919511509196110E94D9DB6093B711FA
:10C630007093B8118093B9119093BA112BEB31E13B
:10C6400047EB51E163EB71E18FEA91E10E9450D237
:10C65000F0909B11CC2389F020918B1130918C119B
:10C6600040918D1150918E116091EF0A7091F00AF6
:10C670008091F10A9091F20A10C020918F113091AF
:10C68000901140919111509192116091F30A709123
:10C69000F40A8091F50A9091F60A0E94D9DB24E011
:10C6A000F29EF0011124E15FF44F2081318142813B
:10C6B00053810E94B9DC9B01AC016091BB11709168
:10C6C000BC118091BD119091BE110E94D8DB609386
:10C6D000BB117093BC118093BD119093BE118BEB75
:10C6E00091E10E94F5D2C090E10AD090E20AE09078
:10C6F000E30AF090E40A20E030E040E752E4609181
:10C70000E70A7091E80A8091E90A9091EA0A0E948A
:10C7100087DF6093E10A7093E20A8093E30A9093C3
:10C72000E40AE0919B11F0E0E956FE4E1082A1DD93
:10C73000C092E10AD092E20AE092E30AF092E40A9F
:10C74000CF91FF90EF90DF90CF900895AF92BF927E
:10C75000CF92DF92EF92FF920F931F93CF93DF93CD
:10C76000D82F209172113091731140917411509112
:10C77000751160916E1170916F118091701190918F
:10C7800071110E94C2DEC62F172F082FF92E60915B
:10C790001D0B70911E0B882777FD8095982F0E94A6
:10C7A00054DD2091E10A3091E20A4091E30A509170
:10C7B000E40A0E9487DF20E030E040E752E40E9474
:10C7C000B9DC20E030E048EC52E40E94B9DC209172
:10C7D0009B112F93DF93FF920F931F93CF935B01D6
:10C7E0006C0142E0E42E01E020E04EE651E16AE710
:10C7F00071E18FEA91E10E94684780917A119091EE
:10C800007B11A0917C11B0917D118093AF11909319
:10C81000B011A093B111B093B21180917E1190919B
:10C820007F11A0918011B09181118093B3119093E9
:10C83000B411A093B511B093B6118091821190916B
:10C840008311A0918411B09185118093B7119093B9
:10C85000B811A093B911B093BA118091861190913B
:10C860008711A0918811B09189118093BB11909389
:10C87000BC11A093BD11B093BE110E9443D7609329
:10C88000C50F7093C60F8093C70F9093C80F0F907A
:10C890000F900F900F900F900F90DF91CF911F91FD
:10C8A0000F91FF90EF90DF90CF90BF90AF900895E1
:10C8B000F8940E94E23D179A1092A011169A1092D5
:10C8C000A111159A1092A211149A60E087E40E94B7
:10C8D00063D6E1EAF9E48491882341F09091C000A5
:10C8E00095FFFCCF8093C6003196F5CFE091C01143
:10C8F000F0E0EE0FFF1FE45EFD4F0190F081E02DB0
:10C90000EA59FE4F0190F081E02D8491882341F097
:10C910009091C00095FFFCCF8093C6003196F5CF73
:10C920008091C00085FFFCCF8AE08093C600E09133
:10C93000C011F0E0EE0FFF1FE45EFD4F0190F081AB
:10C94000E02DE653FF4F808191810E94CB97789430
:10C95000C6E0D0E02197209749F068EC70E080E0D5
:10C9600090E00E9472D70E945A98F4CFF894FFCFBB
:10C970002F923F924F925F926F927F928F929F92EF
:10C98000AF92BF92CF92DF92EF92FF920F931F93DD
:10C99000CF93DF93CDB7DEB76E970FB6F894DEBFB7
:10C9A0000FBECDBF30E6D32E44E0E42EF12C5AE08A
:10C9B000C52EBB24B3948091AC159091AD152091F8
:10C9C000AE153091AF15821B930B8F779927892B6A
:10C9D00009F467C28091CF0F9091D00F04970CF0AB
:10C9E00060C28BE295E10E94A1B68093CE0F2091A8
:10C9F000CC0F3091CD0F8A3061F08D3051F08A33F9
:10CA000021F49091CB0F992321F02F3531050CF4AF
:10CA100042C12115310509F45CC18091D10F90917B
:10CA2000D20FD89E4001D99E900C1124F401E20F40
:10CA3000F31FE752F04F10822091CB0F211126C136
:10CA40001092CB0FFC01EB52F04F10828401075281
:10CA5000104F6EE470E0C8010E943EE40097F1F1CF
:10CA60009093CA0F8093C90F801B910B880D991D5D
:10CA70004AE050E060E070E08652904F0E9471E220
:10CA800060936211709363118093641190936511A8
:10CA900040905E1150905F11609060117090611134
:10CAA0002FEF421A520A620A720A0091D10F1091B6
:10CAB000D20F641575058605970509F40DC1D09E42
:10CAC000C001D19E900D112466E079E48752904F09
:10CAD0000E94E9E3892B09F0FFC0A9C16AE270E076
:10CAE000C8010E943EE4892B09F451C0E1EAF9E44F
:10CAF0008491882341F09091C00095FFFCCF8093F2
:10CB0000C6003196F5CFE091C011F0E0EE0FFF1FA7
:10CB1000E45EFD4F0190F081E02DEC5BFE4F019053
:10CB2000F081E02D8491882341F09091C00095FF21
:10CB3000FCCF8093C6003196F5CF40915E115091A5
:10CB40005F1160916011709161112AE030E08BE219
:10CB500095E10E945CB78091C00085FFFCCF8AE020
:10CB60008093C6001092CD0F1092CC0F0DC3809110
:10CB7000621190916311A0916411B091651180933D
:10CB80005E1190935F11A0936011B0936111809139
:10CB9000D10F9091D20FD89E8001D99E100D1124F3
:10CBA000C8018752904F4C0167E470E00E943EE458
:10CBB000009709F447C09093CA0F8093C90F881952
:10CBC0009909800F911F60E070E08652904F0E949B
:10CBD00009E10E9421DD64307105A0F58091B70F55
:10CBE000882381F1E091C011F0E0EE0FFF1FE45EB9
:10CBF000FD4F0190F081E02DE859FE4F0190F0814A
:10CC0000E02D8491882341F09091C00095FFFCCFE6
:10CC10008093C6003196F5CF8091C00085FFFCCF90
:10CC2000C092C600E091C011F0E0EE0FFF1FE45E7D
:10CC3000FD4F0190F081E02DE453FF4F8081918101
:10CC40000E94BE970091D10F1091D20FD09EC001CB
:10CC5000D19E900D11246EE67CE08752904F0E9489
:10CC600049E4892B09F424DEC8010196B7010E942A
:10CC70007DE09093D20F8093D10F8091CF0F909150
:10CC8000D00F01969093D00F8093CF0F1092CD0FBD
:10CC90001092CC0F90CE8B3311F4B092CB0F9091B9
:10CCA000CB0F911188CE4091D10F5091D20FB90185
:10CCB0006F5F7F4F7093CD0F6093CC0FD49EF001C8
:10CCC000D59EF00D1124E20FF31FE752F04F808341
:10CCD00072CE1092CB0F58C2D09E4001D19E900CC4
:10CCE0001124C4018752904F3C016AE270E00E9417
:10CCF0003EE4009709F03EC0E1EAF9E4849188231C
:10CD000041F09091C00095FFFCCF8093C600319612
:10CD1000F5CFE091C011F0E0EE0FFF1FE45EFD4F94
:10CD20000190F081E02DEE5BFE4F0190F081E02D4F
:10CD30008491882341F09091C00095FFFCCF8093AF
:10CD4000C6003196F5CF40915E1150915F11609110
:10CD50006011709161112AE030E08BE295E10E9450
:10CD60005CB78091C00085FFFCCF8AE08093C6004D
:10CD700002D9F8CE20E010E0F401E20FF11DE752F5
:10CD8000F04F30813A3219F02F5F1327F5CF90938F
:10CD9000CA0F8093C90F86199709880D991D60E005
:10CDA00070E08652904F0E9409E10E9421DD212F00
:10CDB00030E02617370709F4DACEE1EAF9E4849186
:10CDC000882341F09091C00095FFFCCF8093C6006E
:10CDD0003196F5CFE091C011F0E0EE0FFF1FE45E59
:10CDE000FD4F0190F081E02DE05CFE4F0190F0815D
:10CDF000E02D8491882341F09091C00095FFFCCFF5
:10CE00008093C6003196F5CF40915E1150915F112D
:10CE100060916011709161112AE030E08BE295E140
:10CE20000E945CB78091C00085FFFCCF9ECFE1EAF5
:10CE3000F9E48491882341F09091C00095FFFCCFE4
:10CE40008093C6003196F5CFE091C011F0E0EE0F6F
:10CE5000FF1FE45EFD4F0190F081E02DE25CFE4F8C
:10CE60000190F081E02D8491882341F09091C000E1
:10CE700095FFFCCF8093C6003196F5CF40915E11AF
:10CE800050915F1160916011709161112AE030E062
:10CE90008BE295E10E945CB78091C00085FFFCCFDA
:10CEA00064CF8091D111882309F46EC18091CC0F99
:10CEB0009091CD0F892B09F067C18091CF0F909190
:10CEC000D00F892B11F41092B50FF8EE2F2EF3E04E
:10CED0003F2E412C512CACE3CA2ED12CE12CF12C4D
:10CEE0008E010F5F1F4FE0E66E2E77247394409102
:10CEF0006C1450916D1460916E1470916F14809148
:10CF0000641490916514A0916614B0916714481749
:10CF100059076A077B0708F037C18091CF0F9091BE
:10CF2000D00F04970CF030C18091B50F81112CC146
:10CF30008091BF139091C013A091C113B091C213FF
:10CF400080936C1490936D14A0936E14B0936F142F
:10CF500087EB93E10E947D2E482F8093CE0F8A307D
:10CF6000B9F04D30A9F0433229F42091CB0F2223A0
:10CF700079F002C04A33C9F32091CC0F3091CD0F24
:10CF80002F3531052CF48F3FAFEF9A0709F0DEC043
:10CF900040916C1450916D1460916E1470916F14E7
:10CFA0008091641490916514A0916614B0916714F7
:10CFB000481759076A077B0708F48EC0E091C01133
:10CFC000F0E0EE0FFF1FE45EFD4F0190F081E02DD9
:10CFD000EA5BFE4F0190F081E02D8491882341F0BF
:10CFE0009091C00095FFFCCF8093C6003196F5CF9D
:10CFF0008091C00085FFFCCFBAE0B093C6000E94CC
:10D0000043D76093B90F7093BA0F8093BB0F90937F
:10D01000BC0F8090BD0F9090BE0FA090BF0FB0903E
:10D02000C00F681979098A099B09A20191010E9420
:10D0300090E049015A01CA01B901A70196010E9475
:10D0400090E0CA01B901A70196010E9490E07F9388
:10D050006F93C501B40120E13EE040E050E00E9442
:10D0600090E03F932F93A2EFB8E4BF93AF931F9349
:10D070000F930E9476E4EBE9F9E484910FB6F894FB
:10D08000DEBF0FBECDBF882349F09091C00095FF51
:10D09000FCCF8093C60031968491F5CFF801819141
:10D0A000882339F09091C00095FFFCCF8093C60093
:10D0B000F6CF8091C00085FFFCCF3AE03093C600E8
:10D0C000C8010E948E978FEC91E10E94DA5761E0CF
:10D0D0008FEC91E10E949D518091CE0F833211F42B
:10D0E0007092B50F2091CC0F3091CD0F21153105E5
:10D0F00009F4EFCD8091D10F9091D20F689EF0018D
:10D10000699EF00D1124E20FF31FE752F04F1082D9
:10D11000FC01EB52F04F70822091CF0F3091D00F75
:10D120002F5F3F4F3093D00F2093CF0F019664E0D5
:10D1300070E00E947DE09093D20F8093D10F109207
:10D14000CB0F1092CD0F1092CC0FD1CE4B3311F4E8
:10D150007092CB0F4091CB0F4111C5CE4091D10FB2
:10D160005091D20FB9016F5F7F4F7093CD0F6093D5
:10D17000CC0F649EF001659EF00D1124E20FF31FA9
:10D18000E752F04F8083B3CE6E960FB6F894DEBFB1
:10D190000FBECDBFDF91CF911F910F91FF90EF9008
:10D1A000DF90CF90BF90AF909F908F907F906F90C7
:10D1B0005F904F903F902F900895CF92DF92EF9223
:10D1C000FF920F931F93CF93C82F8091CF0F909111
:10D1D000D00F03970CF4CCDB0E9443D70091C10F12
:10D1E0001091C20F2091C30F3091C40FC090C50F92
:10D1F000D090C60FE090C70FF090C80F6C197D0952
:10D200008E099F09061717072807390728F4012BED
:10D21000022B032B09F04CDB4091DD0A5091DE0A12
:10D220006091DF0A7091E00A452B462B472B19F1DC
:10D230000E9443D70091C50F1091C60F2091C70FD0
:10D240003091C80F601B710B820B930B0091DD0AAC
:10D250001091DE0A2091DF0A3091E00A06171707C5
:10D260002807390740F49091FD158091FC1598131B
:10D2700002C0CC2349F0CF911F910F91FF90EF9006
:10D28000DF90CF900C9452C8179A1092A011169A62
:10D290001092A111159A1092A211149AECCF0E942B
:10D2A000E23D8091B70F811151C081E08093B70FAB
:10D2B00080915E1190915F11A0916011B091611108
:10D2C00080935A1190935B11A0935C11B0935D1100
:10D2D000E1EAF9E48491882341F09091C00095FF40
:10D2E000FCCF8093C6003196F5CFE091C011F0E0FD
:10D2F000EE0FFF1FE45EFD4F0190F081E02DE85935
:10D30000FE4F0190F081E02D8491882341F09091AF
:10D31000C00095FFFCCF8093C6003196F5CF809179
:10D32000C00085FFFCCF8AE08093C600E091C01169
:10D33000F0E0EE0FFF1FE45EFD4F0190F081E02D65
:10D34000E453FF4F808191810C94BE9708958091A2
:10D35000B70F0895CF93DF93EC0180919B118093D9
:10D36000B80F84E50E945F5F811102C080E0B8C001
:10D370000E944B5F0E9426DD6093B80F6623B1F3D5
:10D38000EBE9F9E48491882341F09091C00095FF86
:10D39000FCCF8093C6003196F5CFCD36D10509F488
:10D3A00054C0BCF4C836D10561F1C936D10509F0C5
:10D3B00087C0E091C011F0E0EE0FFF1FE45EFD4F6B
:10D3C0000190F081E02DE25BFE4F0190F081E02DB5
:10D3D00038C0CA3DD10509F451C0CD3DD10509F091
:10D3E0006FC0E091C011F0E0EE0FFF1FE45EFD4F53
:10D3F0000190F081E02DEC5AFE4F0190F081E02D7C
:10D400005CC0E091C011F0E0EE0FFF1FE45EFD4F45
:10D410000190F081E02DE45BFE4F0190F081E02D62
:10D420008191882309F44CC09091C00095FFFCCFF6
:10D430008093C600F5CF9091C00095FFFCCF8093FC
:10D44000C60081918111F7CF3BC0E091C011F0E09F
:10D45000EE0FFF1FE45EFD4F0190F081E02DE85AD2
:10D46000FE4F0190F081E02D8191882349F1909148
:10D47000C00095FFFCCF8093C600F6CFE091C011AD
:10D48000F0E0EE0FFF1FE45EFD4F0190F081E02D14
:10D49000EE5AFE4F0190F081E02D8191882381F0BA
:10D4A0009091C00095FFFCCF8093C600F6CF90917D
:10D4B000C00095FFFCCF8093C60081918111F7CF0A
:10D4C00040E050E06091B80F8BE295E10E94BEB75A
:10D4D0008091C00085FFFCCF8AE08093C60081E088
:10D4E000DF91CF910895CF92DF92EF92FF9220913A
:10D4F000BF112223F1F020E030E040E05FE30E9422
:10D5000087DF6B017C0120E030E0A9010E94B2DCE2
:10D51000882379F0A7019601C701B6010E9487DF31
:10D520002BED3FE049E450E40E9487DF9B01AC0112
:10D5300004C020E030E040E85FE360E070E080E8B5
:10D540009FE30E94B9DCFF90EF90DF90CF900895A9
:10D550006091130B7091140B8091150B9091160B29
:10D56000C2DF60930F0B7093100B8093110B90939D
:10D57000120B08953F924F925F926F927F928F921B
:10D580009F92AF92BF92CF92DF92EF92FF920F9352
:10D590001F93CF93DF93CDB7DEB7E9970FB6F8941B
:10D5A000DEBF0FBECDBF81E40E945F5F882309F418
:10D5B0004CC082E70E945F5F8823A9F0E3E7FCE0AC
:10D5C0008191882339F09091C00095FFFCCF809322
:10D5D000C600F6CF8091C00085FFFCCF8AE0809323
:10D5E000C6000C947C8386E70E945F5F8823A9F0C5
:10D5F000E9E7FCE08191882339F09091C00095FF24
:10D60000FCCF8093C600F6CF8091C00085FFFCCF91
:10D610008AE08093C6000C947C8387E60E945F5F5B
:10D62000882321F00E9469970C947C838AE70E94EA
:10D630005F5F882311F40C947C8360E070E089EFD5
:10D640009FE00E9421940C947C8387E40E945F5F9A
:10D65000882309F46EC20E944B5F0E9421DD6A306C
:10D66000710509F4BBC09CF46230710509F44CC02B
:10D6700024F477FF25C00C947C836330710509F492
:10D680004EC06430710509F455C00C947C836A3532
:10D69000710509F4FAC154F46B30710509F4A4C0A2
:10D6A0006C31710509F4A6C00C947C836B3571054F
:10D6B00009F4EFC16C35710509F4F0C10C947C8359
:10D6C0008091B70F81110C947C830E94F35F80914D
:10D6D00098118823A9F088E50E945F5F811110C02E
:10D6E00089E50E945F5F81110BC08AE50E945F5F40
:10D6F000811106C085E40E945F5F81110C947F83D5
:10D700000E9439610C947C838091B70F81110C9435
:10D710007C830E94726081E019D80C947C83809194
:10D72000B70F81110C947C830E94726080E00ED848
:10D730000C947C83E091C011F0E0EE0FFF1FE45EDB
:10D74000FD4F0190F081E02DE054FF4F80819181E9
:10D750000E94BE9780E50E945F5F882339F00E9497
:10D760004B5F0E9426DD4B015C0103C0812C912C94
:10D77000540183E50E945F5F882361F00E944B5F44
:10D7800020E030E04AE754E40E9487DF0E9426DD73
:10D790004B015C010E94DBC00E9443D76B017C01FE
:10D7A000C80CD91CEA1CFB1C0E9443D76093C50F10
:10D7B0007093C60F8093C70F9093C80F0E9443D7F2
:10D7C0006C157D058E059F0510F00C947C830E94DE
:10D7D0000F3B80E0F2DC0E945A98F0CF60E081E0DD
:10D7E0000E94F8610C947C8360E080E00E94F86104
:10D7F0000C947C838091E10A9091E20AA091E30A63
:10D80000B091E40A8093661190936711A093681118
:10D81000B093691180911D0B90911E0B9093C411D0
:10D820008093C31184E690E090931E0B80931D0BB0
:10D830000E9443D76093C50F7093C60F8093C70FA4
:10D840009093C80F81E00E945BB98091AF119091D5
:10D85000B011A091B111B091B21180937A1190934F
:10D860007B11A0937C11B0937D118091B3119091A5
:10D87000B411A091B511B091B61180937E1190931F
:10D880007F11A0938011B09381118091B711909175
:10D89000B811A091B911B091BA11809382119093EF
:10D8A0008311A0938411B09385118091BB11909145
:10D8B000BC11A091BD11B091BE11809386119093BF
:10D8C0008711A0938811B09389111092E10A1092E8
:10D8D000E20A1092E30A1092E40A88E50E945F5F70
:10D8E000882311F090E00AC089E50E945F5F8111F2
:10D8F000F9CF8AE50E945F5F91E098279093E50A4F
:10D9000091110C94AE8388E50E945F5F81110C94A5
:10D91000AE838091E50A81110C94B48389E50E945D
:10D920005F5F81110C94B48388E50E945F5F882358
:10D93000D1F00E94545F672B682B692BA1F00E94E5
:10D940004B5F2091A3113091A4114091A5115091EA
:10D95000A6110E94D9DB6093AF117093B011809330
:10D96000B1119093B21189E50E945F5F8823D1F0D5
:10D970000E94545F672B682B692BA1F00E944B5FBC
:10D980002091A7113091A8114091A9115091AA118D
:10D990000E94D9DB6093B3117093B4118093B511D9
:10D9A0009093B6118091E50A81110C94BA838AE5AF
:10D9B0000E945F5F81110C94BA838AE50E945F5FC9
:10D9C0008823D1F00E94545F672B682B692BA1F04C
:10D9D0000E944B5F2091AB113091AC114091AD1181
:10D9E0005091AE110E94D9DB6093B7117093B811BA
:10D9F0008093B9119093BA112BEB31E147EB51E1D0
:10DA000063EB71E18FEA91E10E9450D280E00E94C5
:10DA10005BB98091661190916711A0916811B091E6
:10DA200069118093E10A9093E20AA093E30AB0930C
:10DA3000E40A8091C3119091C41190931E0B8093BE
:10DA40001D0B0E9443D76093C50F7093C60F809340
:10DA5000C70F9093C80F0E9454B98091D1118823A9
:10DA600011F40C947C836DEC71E189EF9FE00E94CE
:10DA700032948091CD119091CE11892B11F40C9498
:10DA80007C830E94CEAA0C947C83109259110C9432
:10DA90007C8381E0809359110C947C8385E40E94FF
:10DAA0005F5F811102C00E94DBC098EEC92E9CE02E
:10DAB000D92E23EAE22E21E1F22E0FEA11E1B12C58
:10DAC000F60181916F010E945F5F882339F1F3E0D5
:10DAD000BF120CC00E944B5FF80160837183828388
:10DAE00093838BEB91E10E94F5D218C00E944B5FAB
:10DAF000F70120813181428153810E94D9DBF801F5
:10DB000060837183828393832BEB31E147EB51E197
:10DB100063EB71E18FEA91E10E9450D2B394F4E09B
:10DB2000EF0EF11C0C5F1F4F24E0B212C9CF0C9412
:10DB30007C838DE40E945F5F882311F40C948382C0
:10DB40000E944B5F0E9421DD6537710511F40C9432
:10DB5000A0760CF0D0C06032710509F44EC30CF011
:10DB600071C06731710509F4A3C20CF044C0623181
:10DB7000710511F40C94C4751CF577FF02C00C9468
:10DB80007C83623071050CF498C16131710511F02C
:10DB90000C947C83E091C011F0E0EE0FFF1FE45E77
:10DBA000FD4F0190F081E02DE853FF4F808191817E
:10DBB0000E94BE9717981698159814980C947C8319
:10DBC0006531710509F468C20CF06CC264317105ED
:10DBD00011F00C947C83E091C011F0E0EE0FFF1F78
:10DBE000E45EFD4F0190F081E02DE85BFE4F019077
:10DBF000F081E02D20C26B31710509F485C2B4F4C7
:10DC00006931710509F46CC20CF070C28FEC91E1BE
:10DC10000E94854E0E9443D76093BD0F7093BE0F44
:10DC20008093BF0F9093C00F0C947C836E3171056D
:10DC300009F4A5C20CF07DC36C31710509F46AC208
:10DC40000C947C836C35710509F4ECC7ECF46235F7
:10DC5000710509F490C764F46035710509F443C790
:10DC60000CF058C76A32710509F4C1C30C947C8367
:10DC70006435710509F488C70CF481C765357105F1
:10DC800009F4B5C70C947C836B36710509F425C77C
:10DC900064F46936710509F422C40CF0EEC66836E6
:10DCA000710509F4EBC30C947C836037710509F4AA
:10DCB00003C434F46D36710509F41EC50C947C83DD
:10DCC0006237710511F40C94B4766337710511F065
:10DCD0000C947C83E091C011F0E0EE0FFF1FE45E36
:10DCE000FD4F0190F081E02DEE59FE4F0190F08143
:10DCF000E02D0C949B76623E710511F40C94027C2D
:10DD00000CF05FC06B3C710511F40C94417AACF5DA
:10DD10006C38710509F4D2C304F56837710511F444
:10DD20000C94A1776937710511F40C94A6776737C5
:10DD3000710511F00C947C83E091C011F0E0EE0FBE
:10DD4000FF1FE45EFD4F0190F081E02DE258FE4F91
:10DD50000190F081E02D0C94B277683C710511F4CC
:10DD60000C949E79693C710511F40C94207A6E3BF9
:10DD7000710511F00C947C8355C56F3C710511F44D
:10DD80000C94FE7A54F46D3C710511F40C94807A75
:10DD900014F40C945E7A0C94E07A613D710511F4F0
:10DDA0000C945D7B14F40C94357B6C3D710511F47F
:10DDB0000C94CD7B6D3D710511F40C94DC7B0C94BF
:10DDC0007C83653F31E0730711F40C94AF7D54F50B
:10DDD0006F3291E0790711F40C94747D84F46D3204
:10DDE000F1E07F0711F40C94937C14F00C94667DA1
:10DDF0006C32714011F40C945D7C0C947C836F3513
:10DE000081E0780711F40C942782603991E079075A
:10DE100011F40C94AC7D6E35714011F00C947C8340
:10DE20000C94F0816835F2E07F0711F40C94F77ED2
:10DE3000A4F4673F31E0730711F40C94B77D14F438
:10DE40000C94B47D6D3F714011F00C947C830E9462
:10DE50006997EBE9F9E40C94C17D6B38E3E07E0748
:10DE600011F40C94CA813CF46335734011F40C94A2
:10DE7000D27D0C947C83603A33E0730709F426C2A8
:10DE8000673E734011F00C947C831092B70F0E9490
:10DE9000D19780915A1190915B11A0915C11B09132
:10DEA0005D1180935E1190935F11A0936011B09308
:10DEB00061110E94BB5F0C947C830091C90F10918B
:10DEC000CA0F0E5F1F4F80E50E945F5F882379F0C5
:10DED0000E944B5F0E9426DD6B017C01BB24B39442
:10DEE000611571058105910531F4B12C04C0B12C87
:10DEF000C12CD12C760183E50E945F5F882399F0C5
:10DF00000E944B5F20E030E04AE754E40E9487DF44
:10DF10000E9426DD6B017C01AA24A3946115710582
:10DF20008105910509F4A12C6AE270E0C8010E9404
:10DF30003EE4009711F0FC011082F801CF0121911D
:10DF40002032E1F3B11007C0A11005C0222319F05F
:10DF50000E948E9710C0E091C011F0E0EE0FFF1FFD
:10DF6000E45EFD4F0190F081E02DEE53FF4F808184
:10DF700091810E94BE9781E00E946E970E94DBC053
:10DF80000E9443D76093C50F7093C60F8093C70F4D
:10DF90009093C80FC114D104E104F104A9F00E94C8
:10DFA00043D74B015C018C0C9D1CAE1CBF1C0E9416
:10DFB00043D7681579058A059B05B8F40E944299F4
:10DFC000811113C00C94C0830E944099882311F4DE
:10DFD0000C947C830E94429981110AC00E940F3BDD
:10DFE00080E0EBD80E945A98F5CF80E00E946E97AF
:10DFF0008091D111E091C011F0E0EE0FFF1FE45EBF
:10E00000FD4F0190F081E02D882341F0EC53FF4F4C
:10E01000808191810E94BE970C947C838081918144
:10E020000E94BE970C947C839091C00095FFFCCF1A
:10E030008093C600319684918111F6CF8091C00003
:10E0400085FFFCCF8AE08093C6008FEC91E10E94AF
:10E050002D4DE091C011F0E0EE0FFF1FE45EFD4F8B
:10E060000190F081E02DE65BFE4F0190F081E02D04
:10E070008491882341F09091C00095FFFCCF80935C
:10E08000C6003196F5CF8091C00085FFFCCF8AE0B5
:10E090008093C6000C947C838FEC91E10E94824DAA
:10E0A0000C947C838FEC91E10E94814E0C947C83D4
:10E0B0000091C90F1091CA0F0C5F1F4F6AE270E008
:10E0C000C8010E943EE4009711F0FC01108221E09B
:10E0D00041E0B8018FEC91E10E9403530C947C83E2
:10E0E0008FEC91E10E948C4E0C947C838091D21134
:10E0F000882311F40C947C8383E50E945F5F811177
:10E100000C94C9830C947C838FEC91E10E94305075
:10E110000C947C838091C90F9091CA0F6AE270E0E1
:10E1200004960E943EE48C010097D9F02091D30F11
:10E130003091D40F40E6429FC001439F900D1124BF
:10E140006EE470E08752904F0E943EE460E270E01F
:10E150000E943EE401969093CA0F8093C90FF80184
:10E1600010826091C90F7091CA0F6C5F7F4F21E0E0
:10E1700040E08FEC91E10E9403530C947C838091EA
:10E18000D211882311F40C947C8360E08FEC91E130
:10E190000E9493528091C90F9091CA0F6AE270E079
:10E1A00004960E943EE48C010097D9F02091D30F91
:10E1B0003091D40F40E6429FC001439F900D11243F
:10E1C0006EE470E08752904F0E943EE460E270E09F
:10E1D0000E943EE401969093CA0F8093C90FF80104
:10E1E00010826091C90F7091CA0F6C5F7F4F8FECE6
:10E1F00091E10E94F04E0C947C838091D1118111A9
:10E200000E94DBC00091C90F1091CA0F0C5F1F4F15
:10E210006AE270E0C8010E943EE47C0161E270E0C5
:10E22000C8010E943EE4009719F08C010F5F1F4F58
:10E23000E114F10411F0F701108280E50E945F5FA4
:10E24000F82E2091C90F3091CA0F0217130708F456
:10E25000F12C8091D211882311F40C947C8321E05D
:10E260002F2541E0B8018FEC91E10E94035383E533
:10E270000E945F5F8823B9F02091C90F3091CA0FC7
:10E280002017310780F40E94545FAB01BC0140931A
:10E290006C1450936D1460936E1470936F1487EB2D
:10E2A00093E10E94462F8FEC91E10E94854EF11080
:10E2B0000C947C830E9443D76093BD0F7093BE0F74
:10E2C0008093BF0F9093C00F0C947C838091C90FF3
:10E2D0009091CA0F6AE270E005960E943EE48C01BC
:10E2E0000097D9F02091D30F3091D40F40E6429F90
:10E2F000C001439F900D11246EE470E08752904F4F
:10E300000E943EE460E270E00E943EE40196909339
:10E31000CA0F8093C90FF80110826091C90F7091E4
:10E32000CA0F6B5F7F4F8FEC91E10E9488560C946F
:10E330007C830E9443D76093B90F7093BA0F809388
:10E34000BB0F9093BC0F0091BD0F1091BE0F209199
:10E35000BF0F3091C00F601B710B820B930B28EE27
:10E3600033E040E050E00E9490E0CA01B9012CE3A4
:10E3700030E040E050E00E9490E07F936F933F9345
:10E380002F9383EE98E49F938F93CE0101969F93F2
:10E390008F930E9476E4EBE9F9E484910FB6F89448
:10E3A000DEBF0FBECDBF882349F09091C00095FF1E
:10E3B000FCCF8093C60031968491F5CFFE01319653
:10E3C0008191882339F09091C00095FFFCCF809314
:10E3D000C600F6CF8091C00085FFFCCF8AE0809315
:10E3E000C600CE0101960E948E970C947C8383E533
:10E3F0000E945F5F882311F40C947C830E944B5F22
:10E400000E9421DDF62EE72E862F9E2D8C0180E5C1
:10E410000E945F5F882331F00F3F110509F010F46F
:10E420000C94DA830DE010E0E0EBFCE08191919137
:10E430008017910711F40C947C833CE0E83EF307CD
:10E44000A9F70630110539F48F2D9E2D90939A115E
:10E450008093991104C017FF02C00C947C8361E083
:10E46000802F0E9463D66F2D802F0E949CD66F2D27
:10E470007E2D802F0E9459D50C947C8388E690E0F5
:10E480000E94AA6981110C947C8383E50E945F5FDE
:10E49000882371F00091B80F0E944B5F10E0000FCD
:10E4A000111F0256104F0E9421DDF8017183608315
:10E4B0000E94E13D0C947C830E94586483E50E9495
:10E4C0005F5F882311F40C947C830E944B5F0E9451
:10E4D00021DD70939D0F60939C0F0C947C8389E6E3
:10E4E00090E00E94AA6981110C947C83EDEDF8E420
:10E4F0008491882341F09091C00095FFFCCF8093D8
:10E50000C6003196F5CFE091B80F24E0E29FF0010C
:10E510001124EA56F04F408151816281738121E0DC
:10E5200030E08BE295E10E945DB8EAEDF8E4849179
:10E53000882341F09091C00095FFFCCF8093C600E6
:10E540003196F5CFE091B80FF0E0EE0FFF1FE256E5
:10E55000F04F60817181882777FD8095982F0E9408
:10E5600054DDAB01BC0121E030E08BE295E10E947B
:10E570005DB8E6EDF8E48491882341F09091C00005
:10E5800095FFFCCF8093C6003196F5CF4091900F58
:10E590005091910F6091920F7091930F21E030E0B4
:10E5A0008BE295E10E945DB8E3EDF8E48491882365
:10E5B00041F09091C00095FFFCCF8093C60031964A
:10E5C000F5CF60919C0F70919D0F882777FD809506
:10E5D000982F0E9454DDAB01BC0121E030E08BE2BA
:10E5E00095E10E945DB8E0EDF8E48491882341F064
:10E5F0009091C00095FFFCCF8093C6003196F5CF77
:10E600004AE050E060E070E08BE295E10E9487B75D
:10E61000EEECF8E48491882341F09091C00095FFDE
:10E62000FCCF8093C6003196F5CF4091960F509164
:10E63000970F6091980F7091990F21E030E08BE275
:10E6400095E10E945DB8EBECF8E48491882341F0F9
:10E650009091C00095FFFCCF8093C6003196F5CF16
:10E6600060919E0F70919F0F882777FD8095982F5E
:10E670000E9454DDAB01BC0121E030E08BE295E16A
:10E680000E945DB8E7ECF8E48491882341F0909112
:10E69000C00095FFFCCF8093C6003196F5CF8091E6
:10E6A000B80F90E00E94D93A4AE050E0BC018BE2FA
:10E6B00095E10E9487B7E2ECF8E48491882341F069
:10E6C0009091C00095FFFCCF8093C6003196F5CFA6
:10E6D0008FEF9FEF0E94D93A4AE050E0BC018BE2F5
:10E6E00095E10E9487B78091C00085FFFCCF8AE04A
:10E6F0008093C6000C944A858DE690E00E94AA693A
:10E7000081110C947C83E091C011F0E0EE0FFF1FAB
:10E71000E45EFD4F0190F081E02DE65AFE4F8081CE
:10E7200091810E94BE9783E50E945F5F882391F0EC
:10E730000091B80F0E944B5F10E0000F111F0256AE
:10E74000104F0E9421DDF8017183608381E0809386
:10E75000DC0A15C082E50E945F5F882381F000918A
:10E76000B80F0E944B5F10E0000F111F0256104FB0
:10E770000E9421DDF801718360831092DC0A0E94FF
:10E78000E13D0E9443D74B015C010091B80F10E0BE
:10E79000F801EE0FFF1FE256F04F6081718188276C
:10E7A00077FD8095982F0E9454DDF801EE0FFF1F32
:10E7B000EE0FFF1FEA56F04F11E0208131814281B8
:10E7C00053810E94B5DE18160CF010E01093B60FBE
:10E7D00010928A11CC24CA94DC2C7601F8EE4F2ECC
:10E7E000F3E05F2E612C712CAAE03A2E80918A1101
:10E7F00081110C94F584FFEFCF16DF06EF06FF06BC
:10E8000011F40C94E183F7FE02C00C94F5840E948D
:10E8100043D76C197D09683B7B4010F40C94E1836D
:10E820000C94F584E091C011F0E0EE0FFF1FE45E60
:10E83000FD4F0190F081E02DE25AFE4F80819181E1
:10E840000E94BE9783E50E945F5F882361F00E946B
:10E850004B5F0E9421DD70939D0F60939C0F81E0C0
:10E860008093DC0A0FC082E50E945F5F882351F02D
:10E870000E944B5F0E9421DD70939D0F60939C0F5F
:10E880001092DC0A0E9443D74B015C0110928A115E
:10E8900060919C0F70919D0F882777FD8095982F30
:10E8A0000E9454DD11E02091900F3091910F409122
:10E8B000920F5091930F0E94B5DE18160CF010E0E5
:10E8C0001093B60F04EB18E480EBE82E88E4F82EE2
:10E8D0009CEAC92E98E4D92E2AE0722E8091B60FB8
:10E8E00060919C0F70919D0F882309F48BC08091DB
:10E8F0008A11811187C0882777FD8095982F0E9403
:10E9000054DD2091900F3091910F4091920F5091D2
:10E91000930F0E94B5DE18160CF08BC00E9443D7EF
:10E92000681979098A099B09693E73408105910537
:10E9300008F460C0E0919B1184E0E89FF00111248D
:10E94000EA56F04F4081518162817381F8018491D0
:10E95000E4EBF8E4882349F09091C00095FFFCCFE8
:10E960008093C60031968491F5CF22E030E08BE2AF
:10E9700095E10E945DB8F7018491E0EBF8E488230B
:10E9800049F09091C00095FFFCCF8093C60031966E
:10E990008491F5CF60919B1170E04AE050E08BE2EA
:10E9A00095E10E9487B7F6018491ECEAF8E48823A8
:10E9B00049F09091C00095FFFCCF8093C60031963E
:10E9C0008491F5CF4091900F5091910F6091920FEB
:10E9D0007091930F21E030E08BE295E10E945DB8E9
:10E9E0008091C00085FFFCCF7092C6000E9443D783
:10E9F0004B015C010E940F3B80E00E94DD680E9499
:10EA00005A986CCF882777FD8095982F0E9454DD07
:10EA10002091900F3091910F4091920F5091930F50
:10EA20000E94B2DC87FF05C08091DC0A882309F4CC
:10EA300075CFE091C011F0E0EE0FFF1FE45EFD4FD7
:10EA40000190F081E02DE05AFE4F808191810E947B
:10EA5000BE978091D111882321F08CE49CE00E9424
:10EA60008E970E9443D76093C50F7093C60F809313
:10EA7000C70F9093C80F0C947C8383E50E945F5F5F
:10EA8000882319F10E944B5F20E030E0A9010E9429
:10EA9000B2DC87FD0FC00E944B5F20E030E04FE703
:10EAA00053E40E94B5DE181644F00E944B5F0E94AA
:10EAB00021DD05C060E070E002C06FEF70E0709390
:10EAC0009A11609399110C947C838FEF90E090934E
:10EAD0009A11809399110C947C8310929A11109240
:10EAE00099110C947C839B9AA39881E08093E60A09
:10EAF000E091C011F0E0EE0FFF1FE45EFD4F0190CA
:10EB0000F081E02D808191810E94BE970E945A98E9
:10EB10000C947C830E94E23D0E94DBC0149A0E9408
:10EB200045C110929A111092991168EE73E080E03D
:10EB300090E00E9472D79B9AA39A1092E60AE09105
:10EB4000C011F0E0EE0FFF1FE45EFD4F0190F08179
:10EB5000E02DE459FF4F408151812AEA38E468EA08
:10EB600078E485E99CE00E9419470E94BE970E94C4
:10EB70005A980C947C831092C8110C947C8381E089
:10EB80008093C8110C947C8383E50E945F5F882387
:10EB9000A1F00E944B5F20E030E04AE754E40E947D
:10EBA00087DF0E9426DD6093DD0A7093DE0A809382
:10EBB000DF0A9093E00A0C947C8388E50E945F5FF3
:10EBC00081110C94228589E50E945F5F81110C946C
:10EBD00022858AE50E945F5F81110C94228585E47D
:10EBE0000E945F5F81110C9422850C94448583E51B
:10EBF0000E945F5F882311F40C947C830E944B5F1A
:10EC000020E030E04AE754E40E9487DF0E9426DDDE
:10EC10006093C10F7093C20F8093C30F9093C40F82
:10EC20000C947C8328EE3CE039AF28AF01E31BE174
:10EC3000E1E48E2EEBE19E2EF5EFAF2EFAE1BF2E32
:10EC4000312CE8ADF9AD8191F9AFE8AF0E945F5F7B
:10EC5000882309F45BC0F3E03F1251C00E944B5F70
:10EC60006B017C0120E030E040EA51E40E94B2DC1C
:10EC700087FF3FC0A7019601F80160817181828101
:10EC800093810E94B9DC2B013C019B01AC01609196
:10EC9000091B70910A1B80910B1B90910C1B0E9409
:10ECA00087DF6093091B70930A1B80930B1B909363
:10ECB0000C1BA3019201F401608171818281938117
:10ECC0000E9487DFF4016083718382839383F5015F
:10ECD00060817181828193810E9452DDA301920142
:10ECE0000E9487DF0E9426DDF501608371838283A5
:10ECF0009383F801C082D182E282F38207C00E942E
:10ED00004B5FF801608371838283938333940C5F3C
:10ED10001F4FF4E08F0E911C24E0A20EB11C34E0D2
:10ED200033128FCF0C947C839091C00095FFFCCF61
:10ED30008093C600319684918111F6CF0C947C8328
:10ED40000091C90F1091CA0F0B5F1F4F6AE270E06C
:10ED5000C8010E943EE4009711F0FC011082C80136
:10ED60000E948E970C947C83E5EAF8E484918823D2
:10ED700041F09091C00095FFFCCF8093C600319682
:10ED8000F5CF4091AF115091B0116091B1117091D8
:10ED9000B21122E030E08BE295E10E945DB8E1EA39
:10EDA000F8E48491882341F09091C00095FFFCCF56
:10EDB0008093C6003196F5CF4091B3115091B411B4
:10EDC0006091B5117091B61122E030E08BE295E1CF
:10EDD0000E945DB8EDE9F8E48491882341F09091B8
:10EDE000C00095FFFCCF8093C6003196F5CF4091CF
:10EDF000B7115091B8116091B9117091BA1122E018
:10EE000030E08BE295E10E945DB8E9E9F8E4849195
:10EE1000882341F09091C00095FFFCCF8093C600FD
:10EE20003196F5CF4091BB115091BC116091BD114D
:10EE30007091BE1122E030E08BE295E10E945DB856
:10EE4000E091C011F0E0EE0FFF1FE45EFD4F019076
:10EE5000F081E02DEC59FE4F0190F081E02D84917E
:10EE6000882341F09091C00095FFFCCF8093C600AD
:10EE70003196F5CF0E9437C10E9454DD2091311B9D
:10EE80003091321B4091331B5091341B0E94B9DCEE
:10EE9000AB01BC0122E030E08BE295E10E945DB85D
:10EEA000E5E9F8E48491882341F09091C00095FF52
:10EEB000FCCF8093C6003196F5CF81E00E9437C128
:10EEC0000E9454DD2091351B3091361B4091371B39
:10EED0005091381B0E94B9DCAB01BC0122E030E04C
:10EEE0008BE295E10E945DB8E1E9F8E48491882322
:10EEF00041F09091C00095FFFCCF8093C600319601
:10EF0000F5CF82E00E9437C10E9454DD2091391B69
:10EF100030913A1B40913B1B50913C1B0E94B9DC45
:10EF2000AB01BC0122E030E08BE295E10E945DB8CC
:10EF30008091C00085FFFCCF8AE08093C6000C94CE
:10EF40007C8380E00E945BB90C947C8381E00E940A
:10EF50005BB90C947C839091C00095FFFCCF8093AB
:10EF6000C600319684918111F6CF8091C00085FF53
:10EF7000FCCF8AE08093C600E091C011F0E0EE0F74
:10EF8000FF1FE45EFD4F0190F081E02DEE58FE4F33
:10EF90000190F081E02D8491882341F09091C00090
:10EFA00095FFFCCF8093C6003196F5CFE091C0115C
:10EFB000F0E0EE0FFF1FE45EFD4F1E9B13C00190BB
:10EFC000F081E02DE058FE4F0190F081E02D84911A
:10EFD0008823D9F09091C00095FFFCCF8093C600A4
:10EFE0003196F5CF0190F081E02DEE57FE4F019064
:10EFF000F081E02D8491882341F09091C00095FF2D
:10F00000FCCF8093C6003196F5CF8091C00085FF7C
:10F01000FCCF8AE08093C600E091C011F0E0EE0FD3
:10F02000FF1FE45EFD4F0190F081E02DEC58FE4F94
:10F030000190F081E02D8491882341F09091C000EF
:10F0400095FFFCCF8093C6003196F5CFE091C011BB
:10F05000F0E0EE0FFF1FE45EFD4F029913C0019038
:10F06000F081E02DE058FE4F0190F081E02D849179
:10F070008823D9F09091C00095FFFCCF8093C60003
:10F080003196F5CF0190F081E02DEE57FE4F0190C3
:10F09000F081E02D8491882341F09091C00095FF8C
:10F0A000FCCF8093C6003196F5CF8091C00085FFDC
:10F0B000FCCF8AE08093C600E091C011F0E0EE0F33
:10F0C000FF1FE45EFD4F0190F081E02DEA58FE4FF6
:10F0D0000190F081E02D8491882341F09091C0004F
:10F0E00095FFFCCF8093C6003196F5CFE091C0111B
:10F0F000F0E0EE0FFF1FE45EFD4F1D9B13C001907B
:10F10000F081E02DE058FE4F0190F081E02D8491D8
:10F110008823D9F09091C00095FFFCCF8093C60062
:10F120003196F5CF0190F081E02DEE57FE4F019022
:10F13000F081E02D8491882341F09091C00095FFEB
:10F14000FCCF8093C6003196F5CF8091C00085FF3B
:10F15000FCCF8AE08093C600E091C011F0E0EE0F92
:10F16000FF1FE45EFD4F0190F081E02DE858FE4F57
:10F170000190F081E02D8491882341F09091C000AE
:10F1800095FFFCCF8093C6003196F5CFE091C0117A
:10F19000F0E0EE0FFF1FE45EFD4F019913C00190F8
:10F1A000F081E02DE058FE4F0190F081E02D849138
:10F1B0008823D9F09091C00095FFFCCF8093C600C2
:10F1C0003196F5CF0190F081E02DEE57FE4F019082
:10F1D000F081E02D8491882341F09091C00095FF4B
:10F1E000FCCF8093C6003196F5CF8091C00085FF9B
:10F1F000FCCF8AE08093C600E091C011F0E0EE0FF2
:10F20000FF1FE45EFD4F0190F081E02DE658FE4FB8
:10F210000190F081E02D8491882341F09091C0000D
:10F2200095FFFCCF8093C6003196F5CFE091C011D9
:10F23000F0E0EE0FFF1FE45EFD4F1C9B13C001903A
:10F24000F081E02DE058FE4F0190F081E02D849197
:10F250008823D9F09091C00095FFFCCF8093C60021
:10F260003196F5CF0190F081E02DEE57FE4F0190E1
:10F27000F081E02D8491882341F09091C00095FFAA
:10F28000FCCF8093C6003196F5CF8091C00085FFFA
:10F29000FCCF8AE08093C600E091C011F0E0EE0F51
:10F2A000FF1FE45EFD4F0190F081E02DE458FE4F1A
:10F2B0000190F081E02D8491882341F09091C0006D
:10F2C00095FFFCCF8093C6003196F5CFE091C01139
:10F2D000F0E0EE0FFF1FE45EFD4F379913C0019081
:10F2E000F081E02DE058FE4F0190F081E02D8491F7
:10F2F0008823D9F09091C00095FFFCCF8093C60081
:10F300003196F5CF0190F081E02DEE57FE4F019040
:10F31000F081E02D8491882341F09091C00095FF09
:10F32000FCCF8093C6003196F5CF8091C00085FF59
:10F33000FCCF8AE08093C6000C947C8380919B1163
:10F340008093B80F84E50E945F5F882381F10E945B
:10F350004B5F0E9426DD6093B80F662341F1EBE915
:10F36000F9E48491882341F09091C00095FFFCCF8F
:10F370008093C6003196F5CFE091C011F0E0EE0F1A
:10F38000FF1FE45EFD4F0190F081E02DE05BFE4F3A
:10F390000190F081E02D8191882311F40C947C83FD
:10F3A0009091C00095FFFCCF8093C600F4CF84E419
:10F3B0000E945F5F882311F40C947C830E944B5F52
:10F3C00020E030E0A9010E94B2DC811103C010925C
:10F3D000BF1132C00091B80F10E00E944B5FF801DE
:10F3E000EE0FFF1FEE0FFF1FED5EF44F6083718382
:10F3F00082839383E090130BF090140B0091150B14
:10F400001091160B20E030E0A901B701C8010E945D
:10F41000B2DC811104C0E12CF12C00E410E4C7013E
:10F42000D8018093130B9093140BA093150BB093FA
:10F43000160B81E08093BF110E94A86A0C947C8314
:10F4400008EE1CE021E2E22E2BE1F22EF801819180
:10F450008F010E945F5F882349F00E944B5F0E94EA
:10F4600026DDF7016083718382839383F4E0EF0EDE
:10F47000F11C2CE00C3E120749F70E9422D30C9499
:10F480007C8308EE1CE091E4E92E9BE1F92EF80163
:10F4900081918F010E945F5F882339F00E944B5F4A
:10F4A000F7016083718382839383F4E0EF0EF11C94
:10F4B0002CE00C3E120759F70C947C8383E50E94E4
:10F4C0005F5F882351F00E944B5F6093191B70931C
:10F4D0001A1B80931B1B90931C1B84E50E945F5F8B
:10F4E000882311F40C947C830E944B5F6093151B5E
:10F4F0007093161B8093171B9093181B0C947C839E
:10F5000083E50E945F5F882351F00E944B5F609308
:10F510001D1B70931E1B80931F1B9093201B84E563
:10F520000E945F5F882351F00E944B5F6093051B30
:10F530007093061B8093071B9093081B82E40E9424
:10F540005F5F882361F00E944B5F0E9426DD60931D
:10F55000511B7093521B8093531B9093541B88E54F
:10F560000E945F5F882351F00E944B5F6093111BE4
:10F570007093121B8093131B9093141B8AE50E94B7
:10F580005F5F882351F00E944B5F60930D1B709367
:10F590000E1B80930F1B9093101B85E40E945F5FEE
:10F5A000882311F40C947C830E944B5F6093091BA9
:10F5B00070930A1B80930B1B90930C1B0C947C8301
:10F5C00008EE1CE083EAE82E81E1F82EF801819133
:10F5D0008F010E945F5F882339F00E944B5FF70123
:10F5E0006083718382839383F4E0EF0EF11C2CE03F
:10F5F0000B3E120711F40C947C83E8CF83E50E9444
:10F600005F5F882351F00E944B5F6093F30A709311
:10F61000F40A8093F50A9093F60A86E40E945F5FED
:10F62000882381F00E944B5F20E030E040E752E405
:10F630000E94B9DC6093EB0A7093EC0A8093ED0AA8
:10F640009093EE0A8AE50E945F5F882311F40C9480
:10F650007C830E944B5F609393117093941180930D
:10F660009511909396110C947C8383E50E945F5FC3
:10F67000882351F00E944B5F60938F11709390111B
:10F68000809391119093921186E40E945F5F88238A
:10F6900011F40C947C830E944B5F20E030E040E743
:10F6A00052E40E94B9DC6093E70A7093E80A809301
:10F6B000E90A9093EA0A0C947C8383E50E945F5FD9
:10F6C000882311F40C947C830E944B5F0E9421DDFF
:10F6D0006115710551F06130710569F481E0809325
:10F6E0009811109297110C947C831092981110929B
:10F6F00097110C947C83EBE9F9E48491882341F021
:10F700009091C00095FFFCCF8093C6003196F5CF55
:10F71000E091C011F0E0EE0FFF1FE45EFD4F01909D
:10F72000F081E02DE459FE4F0190F081E02D8491AD
:10F73000882341F09091C00095FFFCCF8093C600D4
:10F740003196F5CF8091D30F9091D40F20E6289F6A
:10F75000F001299FF00D1124E752F04F8191882389
:10F7600039F09091C00095FFFCCF8093C600F6CF92
:10F77000EFE8F8E48491882341F09091C00095FF70
:10F78000FCCF8093C6003196F5CF8091C00085FFF5
:10F79000FCCF8AE08093C600AFC783E50E945F5F1D
:10F7A000882309F4A9C70E944B5F0E9421DD709352
:10F7B0001E0B60931D0BA0C783E50E945F5F88232B
:10F7C00009F49AC70E944B5F0E9421DD6B017C0106
:10F7D00084E50E945F5F882381F08DED90E00E94B8
:10F7E000AA69811189C7E091B80FF0E0EE0FFF1F01
:10F7F000E75EF44FD182C0827FC7D0921C0BC092CB
:10F800001B0B7AC780E50E945F5F882309F474C7E9
:10F810000E944B5F0E9421DDD62E062F172F83E515
:10F820000E945F5F882331F00E944B5F0E9421DDC0
:10F830007B0103C0EE24EA94FE2CC70101960397D6
:10F8400008F05AC7E0EBFCE0819191918017910795
:10F8500009F452C73CE0E83EF307B1F717FD4CC787
:10F860000E94DBC0CD2C60E08D2D0E9463D68FEF0F
:10F87000E816F80631F0EA94EF2871F000E010E0A5
:10F880000DC08D2D0E94D1D631E020E0892B09F0EA
:10F8900030E0032F122F02C001E010E08C2D0E94F7
:10F8A000D1D68017910709F427C70E940F3B80E04B
:10F8B0000E94DD680E945A98F1CF83E50E945F5F45
:10F8C000882331F00E944B5F0E9421DD8B0102C032
:10F8D0000EE610E080E50E945F5F882331F00E9411
:10F8E0004B5F0E9421DDCB0102C088EE93E06C01EA
:10F8F000EE24D7FCE094FE2C101611067CF420E0D8
:10F9000030E0A901B8018EE40E940FD8C701B6010A
:10F910000E9472D78EE40E9420DBEEC6C701B601BA
:10F920000E9472D7E9C680E50E945F5F882351F08C
:10F930000E944B5F609318027093190280931A0221
:10F9400090931B0289E40E945F5F882361F00E940C
:10F950004B5F0E945444609314027093150280938D
:10F9600016029093170284E40E945F5F882361F07F
:10F970000E944B5F0E9460446093100270931102DA
:10F98000809312029093130283E40E945F5F8823A6
:10F9900051F00E944B5F60930C0270930D028093B4
:10F9A0000E0290930F020E94C23AE091C011F0E063
:10F9B000EE0FFF1FE45EFD4F0190F081E02DE65C4D
:10F9C000FE4F0190F081E02D8191882339F09091D4
:10F9D000C00095FFFCCF8093C600F6CFEEE9FCE0B7
:10F9E0008191882339F09091C00095FFFCCF8093DE
:10F9F000C600F6CF409118025091190260911A0288
:10FA000070911B0222E030E08BE295E10E945DB82C
:10FA1000E2EAFCE08191882339F09091C00095FFE3
:10FA2000FCCF8093C600F6CF60911402709115024E
:10FA300080911602909117020E945A44AB01BC01BA
:10FA400022E030E08BE295E10E945DB8E6EAFCE05E
:10FA50008191882339F09091C00095FFFCCF80936D
:10FA6000C600F6CF609110027091110280911202CF
:10FA7000909113020E946644AB01BC0122E030E089
:10FA80008BE295E10E945DB8EAEAFCE0819188236F
:10FA900039F09091C00095FFFCCF8093C600F6CF5F
:10FAA00040910C0250910D0260910E0270910F0274
:10FAB00022E030E08BE295E10E945DB88091C000C9
:10FAC00085FFFCCF8AE08093C60016C683E50E94BE
:10FAD0005F5F882319F00E944B5F03C060E070E015
:10FAE000CB010E9419D308C685E40E945F5F88237A
:10FAF00041F00E944B5F0E9421DD8B0177FF03C024
:10FB000009C000E010E0C12CD12CF6E1EF2EF3E4A7
:10FB1000FF2E06C0C12CD12CECE8EE2EE2E4FE2E26
:10FB200083E50E945F5F882321F00E944B5F6B0199
:10FB30007C0183E40E945F5F882331F00E944B5F69
:10FB40000E9421DD9B0102C025E030E0A801C70131
:10FB5000B6010E94F53DD0C50E94DBC0CDC50E9414
:10FB60008EB40E9460B0C8C50E948EB4C5C50E9404
:10FB700060B0C2C59091C00095FFFCCF8093C600D5
:10FB8000319684918111F6CFEFE7F8E484918823D0
:10FB900009F4B2C59091C00095FFFCCF8093C600D8
:10FBA0003196F4CF8AE50E945F5F882309F4D6C0BE
:10FBB0000E944B5F6B017C0120E030E040E751EC9C
:10FBC0000E94B5DE87FD57C020E030E040EA50ECEF
:10FBD000C701B6010E94B2DC18160CF44CC0F7FA4B
:10FBE000F094F7F8F094C0929C11D0929D11E0929D
:10FBF0009E11F0929F11EBE9F9E48491882341F082
:10FC00009091C00095FFFCCF8093C6003196F5CF50
:10FC1000E091C011F0E0EE0FFF1FE45EFD4F808128
:10FC20009181FC01E65CFE4F40815181E255F10972
:10FC30002EE738E465E07DE0808191810E941947DC
:10FC4000FC012491222341F03091C00035FFFCCF0C
:10FC50002093C6000196F4CF8091C00085FFFCCFB1
:10FC60008AE08093C6008091C00085FFFCCF8AE0C7
:10FC70008093C60041C5EBE9F9E48491882341F003
:10FC80009091C00095FFFCCF8093C6003196F5CFD0
:10FC9000E091C011F0E0EE0FFF1FE45EFD4F019018
:10FCA000F081E02DE851FF4F0190F081E02D84912B
:10FCB000882341F09091C00095FFFCCF8093C6004F
:10FCC0003196F5CFE091C011F0E0EE0FFF1FE45E3A
:10FCD000FD4F0190F081E02DE658FE4F0190F0813C
:10FCE000E02D8491882341F09091C00095FFFCCFD6
:10FCF0008093C6003196F5CF4AE050E061EF7FEF88
:10FD00008BE295E10E9487B7E091C011F0E0EE0F21
:10FD1000FF1FE45EFD4F0190F081E02DE458FE4F9F
:10FD20000190F081E02D8491882341F09091C000F2
:10FD300095FFFCCF8093C6003196F5CF4AE050E0A6
:10FD40006BEF7FEF8BE295E10E9487B78091C00057
:10FD500085FFFCCF8AE08093C600CEC4EBE9F9E4CE
:10FD60008491882341F09091C00095FFFCCF80934F
:10FD7000C6003196F5CFE091C011F0E0EE0FFF1F05
:10FD8000E45EFD4F0190F081E02DE851FF4F6AE7FE
:10FD900078E4808191810E94F846FC01249122231D
:10FDA00041F03091C00035FFFCCF2093C600019692
:10FDB000F4CF8091C00085FFFCCF8AE08093C6001D
:10FDC00040919C1150919D1160919E1170919F11D5
:10FDD000705822E030E08BE295E10E945DB880919E
:10FDE000C00085FFFCCF8AE08093C60085C4809167
:10FDF0001D0B90911E0B9093180B8093170BC090C6
:10FE0000AF11D090B011E090B111F090B211CF8E3F
:10FE1000D8A2E9A2FAA20091B3111091B4112091D5
:10FE2000B5113091B6110BA31CA32DA33EA3409195
:10FE3000B7115091B8116091B9117091BA114FA3D7
:10FE400058A769A77AA78091BB119091BC11A09186
:10FE5000BD11B091BE118BA79CA7ADA7BEA7C9824B
:10FE6000DA82EB82FC820D831E832F8338874987D9
:10FE70005A876B877C878D879E87AF87B88B85E491
:10FE80000E945F5F882359F00E944B5F9B01AC0189
:10FE90006BA57CA58DA59EA50E94D9DB0AC020E09C
:10FEA00030E040E050E46BA57CA58DA59EA50E94A6
:10FEB000D8DB6BA77CA78DA79EA79BE9C92E91E1F4
:10FEC000D92EE12CF12C08EC13E49E01255D3F4F67
:10FED000AE01495D5F4FBE016D5D7F4FCE014F9614
:10FEE0000E946EC88AE50E945F5F882349F00E94E5
:10FEF0004B5F9B01AC016FA178A589A59AA51EC097
:10FF000020E030E040E050E46FA178A589A59AA5F3
:10FF10000E94D9DB6B017C016FA378A789A79AA700
:10FF200020E030E040E251E40E94B2DC87FF0CC0E8
:10FF300020E030E040E251E4C701B6010E94D9DB85
:10FF40006FA378A789A79AA7BBE9CB2EB1E1DB2ED7
:10FF5000E12CF12C06E913E49E01255D3F4FAE0133
:10FF6000495D5F4FBE016D5D7F4FCE014F960E9490
:10FF70006EC888E50E945F5F882379F00E944B5F1E
:10FF80009B01AC016F8D78A189A19AA10E94D9DB58
:10FF90006F8F78A389A39AA308C080E090E0A3E5BF
:10FFA000B3E48F8F98A3A9A3BAA389E50E945F5FEA
:10FFB000882339F00E944B5F6BA37CA38DA39EA383
:10FFC00004C01BA21CA21DA21EA2FBE9CF2EF1E1C0
:10FFD000DF2EE12CF12C0CE812E49E01255D3F4F51
:10FFE000AE01495D5F4FBE016D5D7F4FCE014F9603
:10FFF0000E946EC88CE40E945F5F882359F00E94C3
:020000021000EC
:100000004B5F9B01AC016BA57CA58DA59EA50E94B5
:10001000D9DB0AC020E030E040EA52E46BA57CA5C1
:100020008DA59EA50E94D8DB6BA77CA78DA79EA758
:100030007BE9C72E71E1D72EE12CF12C08EC13E4FB
:100040009E01255D3F4FAE01495D5F4FBE016D5D75
:100050007F4FCE014F960E946EC80E94DBC0149A5B
:1000600064E670E080E090E00E9472D70E94E6A310
:1000700000E010E0F12C0E94429981111BC0F39422
:100080000E940F3B81E00E94DD68F110F4CF043F35
:10009000F1E01F0711F400E010E06A9A0115110564
:1000A00011F4729A04C00431110509F472980F5FBB
:1000B0001F4FE1CF729820E030E04CE852E46BA58E
:1000C0007CA58DA59EA50E94D9DB6BA77CA78DA7DB
:1000D0009EA74BE9C42E41E1D42EE12CF12C00EA7D
:1000E00011E49E01255D3F4FAE01495D5F4FBE01AA
:1000F0006D5D7F4FCE014F960E946EC820E030E0CC
:1001000048E452E46BA57CA58DA59EA50E94D9DB91
:100110006BA77CA78DA79EA7E12CF12C00E010E433
:100120009E01255D3F4FAE01495D5F4FBE016D5D94
:100130007F4FCE014F960E946EC81092C21110924E
:10014000C1110E947CA48091C1119091C2110197AC
:1001500009F47CC01092C2111092C1110E94CFA468
:100160008091C1119091C2118230910549F103979C
:1001700009F069C020E030E048E452E46BA57CA5BA
:100180008DA59EA50E94D9DB6BA77CA78DA79EA7F6
:10019000BBE9CB2EB1E1DB2EE12CF12C00E010E429
:1001A0009E01255D3F4FAE01495D5F4FBE016D5D14
:1001B0007F4FCE014F960E946EC80E9429A4C3CFE4
:1001C00020E030E04CE852E46BA57CA58DA59EA50F
:1001D0000E94D9DB6BA77CA78DA79EA79BE9C92EA0
:1001E00091E1D92EE12CF12C00EA11E49E01255D6C
:1001F0003F4FAE01495D5F4FBE016D5D7F4FCE0148
:100200004F960E946EC820E030E048E452E46BA5AF
:100210007CA58DA59EA50E94D9DB6BA77CA78DA789
:100220009EA7E12CF12C00E010E49E01255D3F4FDC
:10023000AE01495D5F4FBE016D5D7F4FCE014F96B0
:100240000E946EC87ECF0E9412A47DCF20E030E0D5
:1002500040EA50E46BA57CA58DA59EA50E94D9DB44
:100260006BA77CA78DA79EA75BE9C52E51E1D52E74
:10027000E12CF12C00E010E49E01255D3F4FAE0122
:10028000495D5F4FBE016D5D7F4FCE014F960E946D
:100290006EC8A80197016BA57CA58DA59EA50E949F
:1002A000D8DB6BA77CA78DA79EA7E12CF12C08ECCF
:1002B00013E49E01255D3F4FAE01495D5F4FBE01D6
:1002C0006D5D7F4FCE014F960E946EC8E12CF12CE0
:1002D0000CE812E49E01255D3F4FAE01495D5F4F82
:1002E000BE016B5F7F4FCE0101960E946EC8E12C6C
:1002F000F12C06E913E49E01255D3F4FAE01475FF7
:100300005F4FBE016B5F7F4FCE0101960E946EC8AA
:1003100020E030E040E050E46BA57CA58DA59EA5D3
:100320000E94D9DB6BA77CA78DA79EA7E12CF12C9F
:1003300008EC13E49E01255D3F4FAE01475F5F4F20
:10034000BE016B5F7F4FCE0101960E946EC8CE0149
:100350000D960E94F5D28091170B9091180B809307
:100360001D0B90931E0B9F938F9381E798E49F93AF
:100370008F938E01015D1F4F1F930F930E9476E4B0
:10038000C8010E943F5C0F900F900F900F900F904C
:100390000F90B2C188E50E945F5F882339F00E9408
:1003A0004B5F0E9421DD80E00E9405C28AE50E9429
:1003B0005F5F882339F00E944B5F0E9421DD81E05E
:1003C0000E9405C285E40E945F5F882309F494C1FE
:1003D0000E944B5F0E9421DD82E00E9405C28CC119
:1003E00083E50E945F5F811104C008EE1CE0F12CE0
:1003F00010C010E00E944B5F0E9426DD812F0E94FA
:10040000DBC21F5F1530B1F7F0CFF394F4E0FF16B5
:1004100079F0F80181918F010E945F5F8823A9F331
:100420000E944B5F0E9426DD8F2D0E94DBC2EDCF24
:1004300082E40E945F5F882339F00E944B5F0E9434
:1004400026DD84E00E94DBC20E94A1C355C183E582
:100450000E945F5F882309F453C00E944B5F0E9493
:1004600021DD6130710541F06230710509F048C04D
:1004700008EE1CE0F12C25C008EE1CE0F12CF80180
:1004800081918F010E945F5F882341F00E944B5F42
:100490000E9421DD4FEF8F2D0E949DC2F394F4E066
:1004A000FF12EDCF82E40E945F5F882349F10E9432
:1004B0004B5F0E9421DD4FEF20C0F394F4E0FF1664
:1004C00089F0F80181918F010E945F5F8823A9F371
:1004D0000E944B5F0E9421DD462F6FEF8F2D0E94FF
:1004E0009DC2EBCF82E40E945F5F882349F00E94A7
:1004F0004B5F0E9421DD462F6FEF84E00E949DC27A
:100500000E94A1C3F9C084E50E945F5F882309F4BB
:10051000A2C00E944B5F0E9426DD6093B80F662345
:1005200009F442C0EBE9F9E48491882341F0909109
:10053000C00095FFFCCF8093C6003196F5CFEEEA60
:10054000FCE08191882339F09091C00095FFFCCFA9
:100550008093C600F6CF40E050E06091B80F8BE288
:1005600095E10E94BEB7E091C011F0E0EE0FFF1FD1
:10057000E45EFD4F0190F081E02DE059FE4F0190C7
:10058000F081E02D8191882339F09091C00095FF92
:10059000FCCF8093C600F6CF8091C00085FFFCCFD2
:1005A0008AE08093C600A8C086E40E945F5F88232B
:1005B000D9F00E944B5F6B017C0160936A117093CC
:1005C0006B1180936C1190936D1120E030E0A901C4
:1005D0000E94B5DE181644F4C092E10AD092E20AF5
:1005E000E092E30AF092E40AEBE9F9E484918823CB
:1005F00041F09091C00095FFFCCF8093C6003196EA
:10060000F5CFE091C011F0E0EE0FFF1FE45EFD4F6B
:100610000190F081E02DE259FE4F0190F081E02D34
:100620008191882339F09091C00095FFFCCF809391
:10063000C600F6CF60919B1170E04AE050E08BE27B
:1006400095E10E9487B78091C00085FFFCCF8AE0CA
:100650008093C60051C0EBE9F9E48491882341F00E
:100660009091C00095FFFCCF8093C6003196F5CFE6
:10067000E091C011F0E0EE0FFF1FE45EFD4F01902E
:10068000F081E02DE459FE4F0190F081E02D84913E
:10069000882341F09091C00095FFFCCF8093C60065
:1006A0003196F5CF8091D30F9091D40F20E6289FFB
:1006B000F001299FF00D1124E752F04F819188231A
:1006C00039F09091C00095FFFCCF8093C600F6CF23
:1006D000EFE6F8E48491882341F09091C00095FF03
:1006E000FCCF8093C6003196F5CF8091C00085FF86
:1006F000FCCF8AE08093C6000E94865FCBC1C09089
:100700008611D0908711E0908811F0908911209186
:10071000BB113091BC114091BD115091BE11C70168
:10072000B6010E94D8DB2DEC3CEC4CEC5DE30E9462
:10073000B5DE181614F00C94806BC092BB11D092E9
:10074000BC11E092BD11F092BE118BEB91E10E94C1
:10075000F5D260E080E00E94F8619CC180E090E00A
:100760000E94AD5A0C94896C81E090E00E94AD5AD1
:100770000C94946C82E090E00E94AD5A0C94DD6C75
:100780000E940F3B80E00E94DD680E945A980C9402
:10079000D76F0E94545FAB01BC0140936C1450931F
:1007A0006D1460936E1470936F1487EB93E10E9445
:1007B000462FA2CF0E944B5F0E9421DD8B010C943B
:1007C00014720E9443D7681979098A099B09693E06
:1007D00073408105910508F479C0EFEBF8E484914A
:1007E000882341F09091C00095FFFCCF8093C60014
:1007F0003196F5CFE091B80F24E0E29FF00111248B
:10080000EA56F04F408151816281738121E030E0EE
:100810008BE295E10E945DB8EBEBF8E484918823CC
:1008200041F09091C00095FFFCCF8093C6003196B7
:10083000F5CF6091B80F70E04AE050E08BE295E1AF
:100840000E9487B7E7EBF8E48491882341F0909108
:10085000C00095FFFCCF8093C6003196F5CFF7FE20
:1008600003C0E3E9FCE025C00E9443D78B019C0153
:10087000C701B6016854744F8F4F9F4F601B710BB7
:10088000820B930BA30192010E9490E0BA01A9018F
:100890002AE030E08BE295E10E94B3B78091C0007E
:1008A00085FFFCCF0DC09091C00095FFFCCF8093D9
:1008B000C60081918111F7CF8091C00085FFFCCFE8
:1008C0003092C6000E9443D74B015C010E940F3B4F
:1008D00080E00E94DD680E945A98FFEFCF16DF0685
:1008E000EF06FF0609F046C08091B60FE091B80F01
:1008F000F0E08F01000F111F000F111F0A56104F5B
:10090000EE0FFF1FE256F04F608171818823C9F01E
:10091000882777FD8095982F0E9454DD20E030E0F5
:1009200040E85FE30E94D8DB9B01AC01F8016081E5
:100930007181828193810E94B5DE87FF50C00C9443
:10094000F673882777FD8095982F0E9454DD20E06C
:1009500030E040E85FE30E94D9DB9B01AC01F80185
:1009600060817181828193810E94B2DC1816BCF58E
:100970000C94F673F7FE02C00C94F673E091B80F76
:10098000F0E08F01000F111F000F111F0A56104FCA
:10099000EE0FFF1FE256F04F60817181882777FDCF
:1009A0008095982F0E9454DD9B01AC01F801608175
:1009B0007181828193810E94D8DB0E9421DD97FFA3
:1009C00007C090958095709561957F4F8F4F9F4F91
:1009D000663071058105910514F40C94F6730E943C
:1009E00043D76B017C010C94F673E091C011F0E0E9
:1009F000EE0FFF1FE45EFD4F0190F081E02DE45A01
:100A0000FE4F808191810E94BE978091D1118823F1
:100A100021F08CE49CE00E948E970E9443D7609363
:100A2000BD0F7093BE0F8093BF0F9093C00F0E94B5
:100A300043D76093C50F7093C60F8093C70F9093F1
:100A4000C80F5ACE0E94DBC088E50E945F5F8823F2
:100A500019F0179A1092A01189E50E945F5F882310
:100A600019F0169A1092A1118AE50E945F5F8823FF
:100A700019F0159A1092A21185E40E945F5F8823F5
:100A800009F43ACE149A38CE0E94DBC0149A0E9420
:100A900045C132CEE9960FB6F894DEBF0FBECDBF8A
:100AA000DF91CF911F910F91FF90EF90DF90CF904A
:100AB000BF90AF909F908F907F906F905F904F907E
:100AC0003F900895CF93DF938091CF0F9091D00FF7
:100AD000039714F40E94B86460E08FEC91E10E94E7
:100AE0009D518091CF0F9091D00F892B09F47EC03A
:100AF0008091CF118823E1F08091D30F9091D40F92
:100B000020E6289FE001299FD00D1124C752D04F25
:100B10006BE079E4CE010E94E9E3892B59F5BE012F
:100B20008FEC91E10E941F518091D011882319F020
:100B30000E94BA6A45C0E091C011F0E0EE0FFF1FBD
:100B4000E45EFD4F0190F081E02DE65CFE4F0190E8
:100B5000F081E02D8491882341F09091C00095FFB1
:100B6000FCCF8093C6003196F5CF8091C00085FF01
:100B7000FCCF23C060E08FEC91E10E949352E091A2
:100B8000C011F0E0EE0FFF1FE45EFD4F0190F08119
:100B9000E02DE45CFE4F0190F081E02D84918823EC
:100BA00041F09091C00095FFFCCF8093C600319634
:100BB000F5CF8091C00085FFFCCF8AE08093C6000E
:100BC0008091CF0F9091D00F01979093D00F809389
:100BD000CF0F8091D30F9091D40F019664E070E015
:100BE0000E947DE09093D40F8093D30F0E940F3B1F
:100BF00080E00E94DD680E947CB8DF91CF910C9468
:100C00005A988F929F92AF92BF92CF92DF92EF92BB
:100C1000FF920F931F93CF93DF938C018C519E4FC4
:100C20000E94E44A680189E8C80ED11C21F17801CC
:100C300081E4E81A8EEFF80AE70157018FE1A81A5C
:100C4000B10863E2862E6DE0962ECC15DD0599F095
:100C5000FE01EE19FF09EA0DFB1D91828082FE0163
:100C600078978081811102C06F97EFCFCE014B97AB
:100C70000E942930F9CFC80186599F4F0E94E44A4B
:100C8000C801875B9F4FDF91CF911F910F91FF901C
:100C9000EF90DF90CF90BF90AF909F908F900C948B
:100CA000E44A8FEC91E10C94F04A8FEC91E1A9CFEA
:100CB000FB016091300B7091310B70939F14609326
:100CC0009E146091A8147091A91470939D14609360
:100CD0009C1462E060932F0B6AE871EA7093310B09
:100CE0006093300B90939B1480939A14F093991413
:100CF000E0939814662757FD6095762F40939414DF
:100D0000509395146093961470939714C901AA2771
:100D100097FDA095BA2F841B950BA60BB70B80935C
:100D2000901490939114A0939214B0939314808193
:100D30009181AA2797FDA095BA2F841B950BA60B2E
:100D4000B70B8093A8149093A914A093AA14B093FE
:100D5000AB140895CF93DF93CDB7DEB7C054D1095C
:100D60000FB6F894DEBF0FBECDBF88E0E7E6FBE02C
:100D7000DE01D99601900D928A95E1F788E0EFE6C1
:100D8000FBE0DE01D19601900D928A95E1F788E0B3
:100D9000E7E7FBE0DE01999601900D928A95E1F775
:100DA00088E0EFE7FBE0DE01919601900D928A95D5
:100DB000E1F788E0E7E8FBE0DE01599601900D924B
:100DC0008A95E1F788E0EFE8FBE0DE0151960190BB
:100DD0000D928A95E1F788E0E7E9FBE0DE011996DC
:100DE00001900D928A95E1F788E0EFE9FBE0DE01E2
:100DF000119601900D928A95E1F7AE01475C5F4F25
:100E000060E083EB94E10E94B946AE014F5C5F4F16
:100E100061E083EB94E10E94B946AE01475D5F4F0C
:100E200062E083EB94E10E94B946AE014F5D5F4FF3
:100E300063E083EB94E10E94B946AE01475E5F4FE9
:100E400064E083EB94E10E94B946AE014F5E5F4FD0
:100E500065E083EB94E10E94B946AE01475F5F4FC6
:100E600066E083EB94E10E94B946AE014F5F5F4FAD
:100E700067E083EB94E10E94B946C05CDF4F0FB698
:100E8000F894DEBF0FBECDBFDF91CF9108950F93D1
:100E90001F93CF93DF93EB01142F022F482F60E0B5
:100EA00083EB94E10E941B45612F83EB94E10E9448
:100EB000D1DB11E1FE016491662311F0111117C01D
:100EC000112339F060E283EB94E10E94D1DB1150F1
:100ED000F7CF602F83EB94E10E94D1DB60E283EBDC
:100EE00094E1DF91CF911F910F910C94D1DB83EBB3
:100EF00094E10E94D1DB21961150DCCFEF92FF925A
:100F00000F931F93CF93DF93EB01E42E8901F90137
:100F100001900020E9F7F22EFE1A92E1F90E482F17
:100F200060E083EB94E10E941B456E2D83EB94E11E
:100F30000E94D1DBFE016491662311F0F11019C00B
:100F40006AE383EB94E10E94D1DBFF2039F060E299
:100F500083EB94E10E94D1DBFA94F7CFB80183EBE5
:100F600094E1DF91CF911F910F91FF90EF900C943E
:100F7000D0DB83EB94E10E94D1DB2196FA94DACFA7
:100F80008093C01191E09093320B682F88EF9FE01F
:100F90000E949AE680918714813019F482E0809350
:100FA00087140895109222158FEC91E10E94A657A4
:100FB0001092B11408958FEC91E10C94854E8FEC52
:100FC00091E10C948C4ECF9382E080932F0B0E9482
:100FD00043D76C507E4F8F4F9F4F6093AD147093EB
:100FE000AE148093AF149093B0146A9ACAE0729AC8
:100FF00084E690E00E9496D7729884E690E00E9482
:1010000096D7C150A1F7CF910895E091300BF091A0
:10101000310BE817F90771F09093310B8093300B87
:101020004093A8145093A9146093AA147093AB141E
:101030002111C9CF089521E040E050E0BA01E5CF89
:1010400021E040E050E0BA01E0CFCF92DF92EF9292
:10105000FF920F931F93CF93DF938091A8149091E9
:10106000A914A091AA14B091AB1481309048A105A5
:10107000B10540F01092A8141092A9141092AA146D
:101080001092AB148091A8149091A914A091AA1465
:10109000B091AB14B695A795979587954091B114EB
:1010A00050E060E070E084179507A607B70710F4DA
:1010B0008093B114D091B1141091B21412FB112786
:1010C00010F9C0E0B1E1CB2ED12CE12CF12C01E0E4
:1010D0004091A8145091A9146091AA147091AB1476
:1010E000D11138C080912F0B8823C1F0E091C0113D
:1010F000F0E0EE0FFF1FE45EFD4F0190F081E02D68
:101100008681978123E0423051056105710510F415
:1011100043E001C040E2BC018C2FB9DE112309F489
:101120009CC18091A8149091A914A091AA14B09187
:10113000AB140297A105B10508F08FC144DF8FE021
:1011400096EADF91CF911F910F91FF90EF90DF9082
:10115000CF9071CFD13051F580912F0B882389F03A
:10116000769567955795479523E041305105610580
:10117000710511F443E001C040E269EA7AE48C2F82
:1011800086DE112309F469C18091A8149091A914F5
:10119000A091AA14B091AB14B695A7959795879591
:1011A0000197A105B10509F058C1C8CFD230B9F5F2
:1011B00080912F0B8823F1F0E091C011F0E0EE0F49
:1011C000FF1FE45EFD4F0190F081E02DE854FE4FDB
:1011D00080819181769567955795479523E04230B8
:1011E00051056105710511F443E001C040E2BC0105
:1011F0008C2F4DDE112309F430C18091A8149091F9
:10120000A914A091AA14B091AB14B695A79597957F
:1012100087950297A105B10509F01FC18FCFD33083
:10122000B9F580912F0B8823F1F0E091C011F0E027
:10123000EE0FFF1FE45EFD4F0190F081E02DE654BC
:10124000FE4F80819181769567955795479523E06C
:10125000433051056105710511F443E001C040E2DE
:10126000BC018C2F14DE112309F4F7C08091A8145F
:101270009091A914A091AA14B091AB14B695A7951A
:10128000979587950397A105B10509F0E6C056CF5C
:10129000D430B9F580912F0B8823F1F0E091C01183
:1012A000F0E0EE0FFF1FE45EFD4F0190F081E02DB6
:1012B000E454FE4F808191817695679557954795C7
:1012C00023E0443051056105710511F443E001C08C
:1012D00040E2BC018C2FDBDD112309F4BEC08091FC
:1012E000A8149091A914A091AA14B091AB14B6952A
:1012F000A795979587950497A105B10509F0ADC00D
:101300001DCFD53051F580912F0B882389F076952C
:1013100067955795479523E045305105610571055F
:1013200011F443E001C040E26CE97AE48C2FAFDDB8
:10133000112309F492C08091A8149091A914A0914E
:10134000AA14B091AB14B695A79597958795059774
:10135000A105B10509F081C0F1CED63051F58091DB
:101360002F0B882389F0769567955795479523E04D
:10137000463051056105710511F443E001C040E2BA
:1013800065E97AE48C2F83DD112309F466C080912E
:10139000A8149091A914A091AA14B091AB14B69579
:1013A000A795979587950697A105B10509F055C0B2
:1013B000C5CED73041F580912F0B882389F07695E3
:1013C00067955795479523E04730510561057105AD
:1013D00011F443E001C040E26CE87AE48C2F57DD61
:1013E0001123D9F18091A8149091A914A091AA1465
:1013F000B091AB14B695A795979587950797A105DA
:10140000B10559F59BCED83041F580912F0B88233B
:1014100089F0769567955795479523E048305105B3
:101420006105710511F443E001C040E262E87AE42D
:101430008C2F2DDD112389F08091A8149091A9148F
:10144000A091AA14B091AB14B695A79597958795DE
:101450000897A105B10509F471CE8091A814909167
:10146000A914A091AA14B091AB144297A105B1059B
:1014700040F0C092A814D092A914E092AA14F0925D
:10148000AB144091A8145091A9146091AA147091C2
:10149000AB1476956795579547958091B11490E078
:1014A0000396242F30E0821793074CF48DEF840FBE
:1014B0008093B11400932F0BDCEFD40FCFEFCF5FED
:1014C000DF5FC43008F404CEDF91CF911F910F91FC
:1014D000FF90EF90DF90CF9008957F928F929F9230
:1014E000AF92BF92CF92DF92EF92FF920F931F9332
:1014F000CF93DF938091A8149091A914A091AA147E
:10150000B091AB1481309048A105B10540F0109224
:10151000A8141092A9141092AA141092AB148091DE
:10152000A8149091A914A091AA14B091AB14B695E7
:10153000A795979587954091B11450E060E070E0D1
:1015400084179507A607B70710F48093B114E090AD
:10155000B114D090B214D2FADD24D0F8F12CCC24FE
:10156000C3948091871481113BC0EE2019F0772439
:10157000739437C080912F0B882301F1E091C01143
:10158000F0E0EE0FFF1FE45EFD4F0190F081E02DD3
:10159000EA50FF4F608171818091A8149091A91445
:1015A000A091AA14B091AB1423E00297A105B10554
:1015B00010F443E001C040E28F2D69DCDD20B9F278
:1015C0008091A8149091A914A091AA14B091AB1481
:1015D0000297A105B10558F6F6DC8CEB94E951C0F1
:1015E000712C80918714823009F05AC07E1057C048
:1015F00080912F0B882359F1E091C011F0E0EE0F9C
:10160000FF1FE45EFD4F0190F081E02DE055FF4F9C
:101610000190F081E02D8091A8149091A914A091DF
:10162000AA14B091AB14B695A79597958795472DB9
:1016300050E060E070E023E084179507A607B70745
:1016400011F443E001C040E2BF018F2D20DCDD201A
:1016500031F18091A8149091A914A091AA14B0918D
:10166000AB14B695A79597958795472D50E060E008
:1016700070E084179507A607B70789F4A4DC83E216
:101680009DEADF91CF911F910F91FF90EF90DF9036
:10169000CF90BF90AF909F908F907F90CCCC739461
:1016A0000CE112E0C0E0D0E08E2C912CA12CB12CEA
:1016B0007E104AC080912F0B882319F1D801ED913B
:1016C000FC91EC54FE4F608171818091A81490913F
:1016D000A914A091AA14B091AB14B695A7959795AB
:1016E0008795272D30E040E050E082179307A4074C
:1016F000B50719F420E24EE302C020E240E28F2D4C
:10170000C6DBDD2009F18091A8149091A914A09165
:10171000AA14B091AB14B695A7959795879588159F
:101720009905AA05BB0581F44EDC8C2FDF91CF9182
:101730001F910F91FF90EF90DF90CF90BF90AF90EF
:101740009F908F907F901CCC739421960E5F1F4FBB
:10175000C530D10509F0ACCF4091A8145091A9141F
:101760006091AA147091AB1476956795579547953B
:10177000872D90E0A0E0B0E0481759076A077B0783
:1017800088F0872D90E0880F991F0197AA2797FD71
:10179000A095BA2F8093A8149093A914A093AA148B
:1017A000B093AB144091A8145091A9146091AA145D
:1017B0007091AB1476956795579547958091B114C4
:1017C00090E00396242F30E0821793075CF48DEFAE
:1017D000840F8093B114C0922F0BDCEFED2EE40E3A
:1017E000FF24FA94F394E394B3E0BF1508F0B9CE64
:1017F000DF91CF911F910F91FF90EF90DF90CF90ED
:10180000BF90AF909F908F907F9008950F931F93FC
:10181000CF93DF938091A8149091A914A091AA145A
:10182000B091AB1481309048A105B10540F0109201
:10183000A8141092A9141092AA141092AB148091BB
:10184000A8149091A914A091AA14B091AB14B695C4
:10185000A795979587954091B11450E060E070E0AE
:1018600084179507A607B70710F48093B114D09199
:10187000B1141091B21412FB112710F9C0E001E06D
:101880008091A8149091A914A091AA14B091AB14BE
:10189000D11134C020912F0B2223C1F0E091C0114F
:1018A000F0E0EE0FFF1FE45EFD4F0190F081E02DB0
:1018B000EA50FF4F6081718123E00297A105B105D5
:1018C00010F443E001C040E28C2FE1DA112309F467
:1018D00082C08091A8149091A914A091AA14B091EB
:1018E000AB140297A105B10508F075C06CDB8CEB59
:1018F00094E9DF91CF911F910F919DCBD130A9F544
:1019000020912F0B2223D1F0E091C011F0E0EE0FD7
:10191000FF1FE45EFD4F0190F081E02D62AD73ADDD
:10192000B695A795979587952EE70197A105B105DF
:1019300011F44EE301C040E28C2FA9DA112309F41F
:101940004AC08091A8149091A914A091AA14B091B2
:10195000AB14B695A795979587950197A105B10505
:10196000D1F531DB86ED92EABFC0D230A1F52091EE
:101970002F0B2223D1F0E091C011F0E0EE0FFF1FFA
:10198000E45EFD4F0190F081E02D64AD75ADB6953C
:10199000A795979587952EE70297A105B10511F4B4
:1019A0004EE301C040E28C2F72DA1123A1F0809146
:1019B000A8149091A914A091AA14B091AB14B69553
:1019C000A795979587950297A105B10521F4FBDAB4
:1019D0008DED92EA89C020E030E040E251E4609170
:1019E00083147091841480918514909186140E94C0
:1019F000B2DC87FF7EC08091A8149091A914A091B9
:101A0000AA14B091AB14D330B1F520912F0B22233F
:101A1000D1F0E091C011F0E0EE0FFF1FE45EFD4F4A
:101A20000190F081E02D66AD77ADB695A7959795BD
:101A300087952EE70397A105B10511F44EE301C088
:101A400040E28C2F24DA111102C025E053C08091AE
:101A5000A8149091A914A091AA14B091AB14B695B2
:101A6000A795979587950397A105B10571F7ABDA0F
:101A700084EE92EA39C0D43041F720912F0B222313
:101A8000E1F0E091C011F0E0EE0FFF1FE45EFD4FCA
:101A90000190F081E02DE05CFF4F60817181B6958F
:101AA000A795979587952EE70497A105B10511F4A1
:101AB0004EE301C040E28C2FEAD9112331F240916C
:101AC000A8145091A9146091AA147091AB14769542
:101AD000679557954795443051056105710509F0A3
:101AE000B4CF71DA80E191EADF91CF911F910F912C
:101AF000A7CA23E04091A8145091A9146091AA1498
:101B00007091AB147695679557954795822F90E025
:101B1000A0E0B0E0481759076A077B0788F0822FDA
:101B200090E0880F991F0197AA2797FDA095BA2FDB
:101B30008093A8149093A914A093AA14B093AB1403
:101B40004091A8145091A9146091AA147091AB14FB
:101B500076956795579547958091B11490E00396D7
:101B6000242F30E0821793074CF48DEF840F80937D
:101B7000B11400932F0BDCEFD40FCFEFCF5FDF5FFB
:101B8000C43008F47DCEDF91CF911F910F9108955D
:101B900080E090E0A0E8BFE38093831490938414E6
:101BA000A0938514B093861431CE20E044E064E124
:101BB00083EB94E10E944E45CDD883EB94E10C94E5
:101BC0000F45F3DF20E040E050E0BA0183E29DEAF8
:101BD0001CCA10929F0F10929E0F10929D0F109290
:101BE0009C0F10929A1110929911EBCF83EB94E114
:101BF0000C940F4580911F159091201590939F0F85
:101C000080939E0F80911D1590911E1590939D0FAE
